:020000040800F2
:20300000102B0020013100080720010885CA0008051F0108354B00088162010800000000F3
:20302000000000000000000000000000673B0108516F00080000000069230108C94A01086C
:203040001B3100081B3100081B3100081B3100081B3100081B3100081B3100081B310008D0
:203060009D7500081B3100081B3100084D5C00081B3100081B3100081B3100081B3100088D
:203080001B3100081B310008C54200081B310008C15B0108394B00081B3100081B310008CC
:2030A0001B310008F54B01081B3100081B3100081B3100081B3100081B3100081B3100087B
:2030C0001B3100081B3100081B3100081B3100081B3100081B3100081B310008D55A01086C
:2030E000917500081B3100081B310008DFF80CD001F098F800480047A1420008102B002011
:203100000648804706480047FEE7FEE7FEE7FEE7FEE7FEE7FEE7FEE7FEE7FEE79D4B010822
:20312000ED3000082DE9FF1F002000210022002300240025002600275FF000085FF000096B
:203140005FF0000A5FF0000B5FF0000C002001210222032304240525062607275FF00808CA
:203160005FF009095FF00A0A5FF00B0B5FF00C0C00281DD101291BD1022A19D1032B17D167
:20318000042C15D1052D13D1062E11D1072F0FD1B8F1080F0CD1B9F1090F09D1BAF10A0FDA
:2031A00006D1BBF10B0F03D1BCF10C0F00D101E004F000BDBDE8FF1F7047000073B40020B2
:2031C00000210124002501262046A04226D1A94224D12846A84221D1A9421FD14FEA440498
:2031E00006F10106202EEFDD5FF0FF305FF0FF317FF000445FF0FF3501262046A0420DD137
:20320000A9420BD12846A84208D1A94206D14FEA740406F10106202EEFDD01E004F0CABCD0
:2032200073BC7047E7B40021002000220125002601272946A94230D1B0422ED1B2422CD1F9
:203240003146B14229D1B04227D1B24225D14FEA450507F10107202FEBDD5FF0FF315FF0CE
:20326000FF305FF0FF327FF000455FF0FF3601272946A94211D1B0420FD1B2420DD13146E8
:20328000B1420AD1B04208D1B24206D14FEA750507F10107202FEBDD01E004F08BBCE7BC41
:2032A00070472DE9CE01002200210023012600275FF001083246B24233D1B94231D1BB42FC
:2032C0002FD13A46BA422CD1B9422AD1BB4228D14FEA460608F10108B8F1200FEADD5FF014
:2032E000FF325FF0FF315FF0FF337FF000465FF0FF375FF001083246B24212D1B94210D1E0
:20330000BB420ED13A46BA420BD1B94209D1BB4207D14FEA760608F10108B8F1200FEADD79
:2033200001E004F047BCBDE8CE0170472DE99C0300230022002401275FF000085FF0010994
:203340003B46BB4233D1424531D144452FD1434643452CD142452AD1444528D14FEA470740
:2033600009F10109B9F1200FEADD5FF0FF335FF0FF325FF0FF347FF000475FF0FF385FF09B
:2033800001093B46BB4212D1424510D144450ED1434643450BD1424509D1444507D14FEA0A
:2033A000770709F10109B9F1200FEADD01E004F001BCBDE89C0370472DE9381C00240023AD
:2033C00000255FF0010A5FF0000B5FF0010C5446544533D15B4531D15D452FD15C465C45FA
:2033E0002CD15B452AD15D4528D14FEA4A0A0CF1010CBCF1200FEADD5FF0FF345FF0FF335D
:203400005FF0FF357FF0004A5FF0FF3B5FF0010C5446544512D15B4510D15D450ED15C46D1
:203420005C450BD15B4509D15D4507D14FEA7A0A0CF1010CBCF1200FEADD01E004F0BABB67
:20344000BDE8381C70472DE9701C0025002400265FF0010A5FF0000B5FF0010C5546554566
:2034600033D15C4531D15E452FD15D465D452CD15C452AD15E4528D14FEA4A0A0CF1010CF1
:20348000BCF1200FEADD5FF0FF355FF0FF345FF0FF367FF0004A5FF0FF3B5FF0010C5546C7
:2034A000554512D15C4510D15E450ED15D465D450BD15C4509D15E4507D14FEA7A0A0CF1BA
:2034C000010CBCF1200FEADD01E004F073BBBDE8701C70472DE9E01C0026002500275FF07E
:2034E000010A5FF0000B5FF0010C5646564533D15D4531D15F452FD15E465E452CD15D45A2
:203500002AD15F4528D14FEA4A0A0CF1010CBCF1200FEADD5FF0FF365FF0FF355FF0FF374D
:203520007FF0004A5FF0FF3B5FF0010C5646564512D15D4510D15F450ED15E465E450BD1AA
:203540005D4509D15F4507D14FEA7A0A0CF1010CBCF1200FEADD01E004F02CBBBDE8E01CAC
:2035600070472DE9C01D002700265FF000085FF0010A5FF0000B5FF0010C5746574533D1B0
:203580005E4531D1D8452FD15F465F452CD15E452AD1D84528D14FEA4A0A0CF1010CBCF12B
:2035A000200FEADD5FF0FF375FF0FF365FF0FF387FF0004A5FF0FF3B5FF0010C57465745AF
:2035C00012D15E4510D1D8450ED15F465F450BD15E4509D1D84507D14FEA7A0A0CF1010C2A
:2035E000BCF1200FEADD01E004F0E4BABDE8C01D70472DE9801F5FF0000800275FF00009F1
:203600005FF0010A5FF0000B5FF0010CD046D04533D15F4531D1D9452FD1D846D8452CD16F
:203620005F452AD1D94528D14FEA4A0A0CF1010CBCF1200FEADD5FF0FF385FF0FF375FF040
:20364000FF397FF0004A5FF0FF3B5FF0010CD046D04512D15F4510D1D9450ED1D846D845C9
:203660000BD15F4509D1D94507D14FEA7A0A0CF1010CBCF1200FEADD01E004F09BBABDE8C1
:20368000801F70472DE970075FF000095FF000085FF0000A012400250126A146A14530D100
:2036A000A8452ED1AA452CD1A946A94529D1A84527D1AA4525D14FEA440406F10106202EC4
:2036C000EBDD5FF0FF395FF0FF385FF0FF3A7FF000445FF0FF350126A146A14511D1A84594
:2036E0000FD1AA450DD1A946A9450AD1A84508D1AA4506D14FEA740406F10106202EEBDD14
:2037000001E004F057BABDE8700770472DE9700E5FF0000A5FF000095FF0000B0124002507
:203720000126A246A24530D1A9452ED1AB452CD1AA46AA4529D1A94527D1AB4525D14FEADA
:20374000440406F10106202EEBDD5FF0FF3A5FF0FF395FF0FF3B7FF000445FF0FF35012618
:20376000A246A24511D1A9450FD1AB450DD1AA46AA450AD1A94508D1AB4506D14FEA740403
:2037800006F10106202EEBDD01E004F013BABDE8700E70472DE9701C5FF0000B5FF0000A44
:2037A0005FF0000C012400250126A346A34530D1AA452ED1AC452CD1AB46AB4529D1AA45C5
:2037C00027D1AC4525D14FEA440406F10106202EEBDD5FF0FF3B5FF0FF3A5FF0FF3C7FF06B
:2037E00000445FF0FF350126A346A34511D1AA450FD1AC450DD1AB46AB450AD1AA4508D106
:20380000AC4506D14FEA740406F10106202EEBDD01E004F0CFB9BDE8701C70472DE9701838
:203820005FF0000C5FF0000B012400250126A446A44526D1AB4524D1AC46AC4521D1AB45EE
:203840001FD14FEA440406F10106202EEFDD5FF0FF3C5FF0FF3B7FF000445FF0FF3501266F
:20386000A446A4450DD1AB450BD1AC46AC4508D1AB4506D14FEA740406F10106202EEFDD7F
:2038800001E004F097B9BDE8701870472DE9F0030024002546594E51445105F10405182DB6
:2038A000F8DB04255FF0000801245FF0010944514659B4425FD105F10407C659B0455AD19D
:2038C0002F1FC659B04556D140F805804659B04551D105F10407C659B0454CD12F1FC6594D
:2038E000B04548D14FEA440409F10109B9F1200FDDDD05F10405142DD6DB5FF0FF3400250A
:20390000445105F10405182DFADB04255FF0FF387FF000445FF0010944514659B4422AD119
:2039200005F10407C659B04525D12F1FC659B04521D140F805804659B0451CD105F10407E9
:20394000C659B04517D12F1FC659B04513D14FEA740409F10109B9F1200FDDDD05F10405DE
:20396000142DD5DB00254E59465105F10405182DF9DB012000E00020BDE8F00370472DE955
:20398000F00300240025445105F104058D42FADB00255FF0000801245FF001094451465985
:2039A000B44268D1002D03D02F1FC659B04562D105F104078F4202DAC659B0455BD140F81D
:2039C00005804659B04556D1002D03D02F1FC659B04550D105F104078F4202DAC659B04562
:2039E00049D14FEA440409F10109B9F1200FD5DD05F104058D42CEDB5FF0FF3400254451EA
:203A000005F104058D42FADB00255FF0FF387FF000445FF0010944514659B4422BD1002DF9
:203A200003D02F1FC659B04525D105F104078F4202DAC659B0451ED140F805804659B04559
:203A400019D1002D03D02F1FC659B04513D105F104078F4202DAC659B0450CD14FEA7404E6
:203A600009F10109B9F1200FD5DD05F104058D42CDDB012000E00020BDE8F0037047202A87
:203A800004DB203A21FA02F00021704721FA02F3D040C2F12002914008431946704740EAB7
:203AA00001039B0703D009E008C9121F08C0042AFAD203E011F8013B00F8013B521EF9D249
:203AC0007047D2B201E000F8012B491EFBD270470022F6E710B513460A4604461946FFF7AF
:203AE000F0FF204610BD10B5044604E00B7800F8013B03B1491C521EF8D2204610BD421C16
:203B000010F8011B0029FBD1801A704730B505460020034600E05B1C934205D2EC5CC85C33
:203B2000201A01D1002CF6D130BD2DE9F0410546002090460E46044600E0641C44450BD2AD
:203B4000285D00F083FA0746305D00F07FFA381A02D1295D0029F0D1BDE8F081F0B480EA77
:203B60000102D40F4200B2EB410F02D20246084611464A0042D0C30DDDB2C1F3C752AD1A20
:203B8000202D35DAC1F3160141F4000204B15242C5F1200602FA06F12A411044B3EBD05F23
:203BA00023D0C4B1012DA0EBC35009DCF0BC4FF0004202EAC352DBB200F5000000F055BA3D
:203BC000400000F1807000EBC350A0F1807040EAD170490009E0490841EAC071A0EBC3505D
:203BE00000F50000400800EBC350F0BC00F034BA6142012202EB4101001BF6E7F0BC7047B0
:203C000081F00041AAE780F00040A7E780EA010210B502F00043400022D04A001FD0010E42
:203C200001EB1261C0F35600C2F3560240F4000042F40002A0FB022000047F39140400D042
:203C4000401C50EA124001D44000491EC2B20C0604EBD010401C4008802A02D003E0002088
:203C600010BD20F00100002900DA0020184310BD2DE9FE4F804681EA0300C00F0C460090D3
:203C800021F0004123F00045B8EB0200A94105D24046214690461C460B46024623F0004003
:203CA000104347D0270DC7F30A00C3F30A510290401A019040286BDAC3F3130040F4801BCF
:203CC0000098924620B10023D2EB030A63EB0B0B01985946C0F14002504600F096F90646C6
:203CE0000D4650465946019A00F09EF910EB08006141002487EA115284EAE7731A4340D048
:203D0000009A62B3019A012A4FEA075215DC001B61EB02014FF0004202EA0752CDE9004283
:203D2000001C41F5801132462B4600F0DBF903B0BDE8F08F40462146F9E7001B61EB0201E5
:203D4000001C41F5801300185B412018A2F5001747EB030140EAD570B6196D4111E06D085C
:203D60004FEA360645EAC0754FEA0752001B61EB0201001C41F5801149084FEA30000019B8
:203D8000514132462B4603B0BDE8F04F00F09BB90098012240000023D0EB020263EBE0734F
:203DA000009821464FEAE074B8EB000061EB0401E9E783F000435BE781F0004158E72DE9B4
:203DC000F04D81EA030404F0004B21F0004514464FF0000A23F0004150EA050220D054EA39
:203DE00001021DD0C5F30A570246C5F31303C1F31300C1F30A5640F4801543F48013A7EBA4
:203E00000608101BD64608F2FD3873EB050002D308F1010801E092185B41B8F1000F03DA28
:203E200000200146BDE8F08D00204FF48011064684460EE0171B73EB050705D3121B63EB12
:203E4000050306434CEA010C49084FEA300092185B4150EA0107EDD152EA030012D082EA41
:203E6000040083EA0501084305D0101BAB4106D20122002306E000224FF0004302E06FF0AB
:203E8000010253101AEB06004CEB085110EB0A0041EB0B01BDE8F04D00F015B99623002269
:203EA000114600F0E2B80EB5C10F80EAE0700844CA07002140F233438DE80E000A460B46CA
:203EC00000F010F903B000BD0EB540F2334102910021CDE900110A460B4600F003F903B055
:203EE00000BD00F0004220F00040C10DC0F3160040F400007F2901DA00207047962903DCC0
:203F0000C1F19601C84001E096398840002AF4D04042704720F00040C10DC0F3160040F496
:203F200000007F2901DA00207047962903DCC1F19601C840704796398840704770B5C1F35A
:203F40000A5201F000450024C1F3130140F2FF3341F480119A4201DA002070BD40F233430D
:203F60009A42A2F2334203DC5242FFF788FD00E090402C43F1D0404270BDC1F30A5210B50A
:203F8000C1F3130140F2FF3341F480119A4201DA002010BD40F233439A42A2F2334203DC1F
:203FA0005242FFF76CFD10BD904010BD00F0004230F000400AD0C10D01F56071C0F31600DA
:203FC00042EA0151C20840071143704700200146704701F0004330B421F0004150EA010282
:203FE00006D00A0DA2F56072C1F31301002A02DC30BC00207047440F44EAC104C100E018D9
:2040000030BC00EBC25000F027B8202A04DB203A00FA02F1002070479140C2F1200320FAE0
:2040200003F3194390407047202A06DBCB17203A41FA02F043EAE07306E041FA02F3D0406D
:20404000C2F120029140084319467047A0F14101192900D8203070470029A8BF7047401CC2
:20406000490008BF20F00100704710B4B0FA80FC00FA0CF050EA010404BF10BC704749B109
:20408000CCF1200421FA04F411FA0CF118BF012121430843A3EB0C01CB1D4FEA00614FEA26
:2040A000102042BF002010BC704700EBC35010440029A4BF10BC7047401C490008BF20F04F
:2040C000010010BC704710B5141E73F1000408DA401C41F1000192185B411A4301D120F007
:2040E000010010BD2DE9F04D92469B4611B1B1FA81F202E0B0FA80F220329046FFF785FF66
:2041000004460F4640EA0A0041EA0B0153465A46084313D0114653EA010019D0C8F14002B5
:204120005046FFF7ACFC05460E46504659464246FFF76BFF084305D0012004E02046394685
:20414000BDE8F08D0020054346EAE0762C4337430A986305E40AA0EB08000022FD0A44EA84
:2041600047540A3002D500200146E9E7010510196941DDE9084500196941BDE8F04DA2E742
:204180002DE9F04D00231A461B1A8A4103DB00200146BDE8F08DC1F30A52C1F3130141F4D5
:2041A00080154FF0000BD10702D100186D41521E0027044640F2FF11384601EB620A3E4632
:2041C0008046024600204FF48011FFF758FCC2197141BB1846EB0100B4EB030C75EB000CE7
:2041E00004D3E41A65EB000517460E46241908F101006D4180463428E3DDF91946EB0600D4
:20420000091BA84103D24FF0FF32134601E0002213461BEB070046EB0A51BDE8F04DFFF726
:2042200052BF0000064C074D06E0E06840F0010394E8070098471034AC42F6D3FEF75AFFBA
:204240000C7F01082C7F010870B58C1810F8015B15F0070301D110F8013B2A1106D110F8AA
:20426000012B03E010F8016B01F8016B5B1EF9D12B0705D40023521E0DD401F8013BFAE77E
:2042800010F8013BCB1A921C03E013F8015B01F8015B521EF9D5A142D8D3002070BD00008F
:2042A00010B572B606480079AA2801D00FF05CFB00200349087162B612F0FCFC10BD00008D
:2042C0000030024010B5024805F054F810BD0000381F002070B5044600252068806800F0E4
:2042E0000100F0B12068806820F001002168886006F0FAFC05460EE006F0F6FC401B022898
:2043000009D9A06A40F01000A062E06A40F00100E062012070BD2068806800F001000028DB
:20432000EAD10020F6E770B505466C6AA06A00F05000E0B9A06A40F40070A062206880687C
:2043400000F46020B0F5602F0DD1E06858B9A06A20F48070A062A06A00F4805018B9A06AC5
:2043600040F00100A062204604F0DCFC03E0206A016B2846884770BD70B505466C6AA06A45
:2043800040F04000A062E06A40F00400E062204604F0EFFF70BD70B50446656A284604F0D6
:2043A000E7FF70BD38B504460025002000902068806800F0010080BB2068806840F00100A1
:2043C00021688860164800681649B0FBF1F0009002E00098401E009000980028F9D106F043
:2043E00083FC054613E006F07FFC401B02280ED9A06A40F01000A062E06A40F00100E0621A
:2044000000BF002084F8240000BF012038BD2068806800F001000028E5D00020F6E700000D
:204420000000002040420F0070B505460E4606F05BFC22490968401A02283DD3002418E02E
:204440001F4850F824001F4931F81410C0EB81201B4951F8241001EBE010194941F824000C
:20446000084650F82400C0F38F2025F81400601CC4B20B2CE4DB002418E0134850F8240024
:20448000124931F81410C0EB81200F4951F8241001EBE0100C4941F82400084650F824000B
:2044A000C0F38F2026F81400601CC4B2032CE4DB06F01AFC0149086070BD00007805002000
:2044C000AC1F0020DC1E0020D81F00202405002010B5154804F0EAF8144804F0E7F81248F6
:2044E00005F0FEF8114805F0FBF8104804F0EEFA0B220F490C4805F08BF90B48006A0068E5
:20450000006820F004000849096A09680860094807F041FC0C21074807F0B4FE0C2105485E
:2045200007F05AFB10BD0000081F0020381F0020DC1E00201C1E0020014600226648814256
:204540000DD1664848604A68824201D000207047634848604A68824201D00020F7E76148C8
:2045600081420DD1604848604A68824201D00020EDE75E4848604A68824201D00020E6E78D
:2045800040F2555048614A69824201D00020DEE740F6AA2048614A69824201D00020D6E7A0
:2045A00040F2555088618A69824201D00020CEE740F6AA2088618A69824201D00020C6E7A0
:2045C00040F25550C861CA69824201D00020BEE740F6AA20C861CA69824201D00020B6E7A0
:2045E00040F2555008620A6A824201D00020AEE740F6AA2008620A6A824201D00020A6E79C
:2046000040F2555048624A6A824201D000209EE740F6AA2048624A6A824201D0002096E79B
:2046200040F2555088628A6A824201D000208EE740F6AA2088628A6A824201D0002086E79B
:204640002B48C862CA6A824201D000207FE72948C862CA6A824201D0002078E726480863B2
:204660000A6B824201D0002071E7244808630A6B824201D000206AE71F4848634A6B8242DB
:2046800001D0002063E71D4848634A6B824201D000205CE71A4888638A6B824201D000202B
:2046A00055E7184888638A6B824201D000204EE700204860C860086148618861C861086216
:2046C00040F6FF70486200208862C86208634863886301203BE700000024014055554500BF
:2046E000AAAA8A000028014055554000AAAA800055555500AAAAAA0055555515AAAAAA2A7C
:2047000055551500AAAA2A0088B001460022086800904868019088680290CB6803930B69BB
:2047200004934B690593552008600A68552A02D0002008B07047AA2008600A68AA2A01D01E
:204740000020F6E745F2555048604A68824201D00020EEE74AF6AA20486048684AF6AA232D
:2047600000EA03021846824201D00020E1E745F2555088608A68824201D00020D9E742F60C
:20478000AA2088608A68824201D00020D1E745F25553CB60CA681846824201D00020C8E70A
:2047A00042F6AA23CB60CA681846824201D00020BFE745F255530B610A691846824201D02D
:2047C0000020B6E742F6AA230B610A691846824201D00020ADE745F255534B614A691846F5
:2047E000824201D00020A4E742F6AA234B614A691846824201D000209BE7009808600198E7
:20480000486002988860039BCB60049B0B61059B4B6101208DE70246002004E0002322F830
:204820001030431C98B28842F8DB70472DE9F04704460E46924699466527844800780128A0
:204840007AD106F051FA40F6C411884202D20020BDE8F0877E480088401C7D490880608A05
:204860007C49096808447B49086079480088012801DC1920ECE776480088032801DC32208F
:20488000E6E773480088052801DC4B20E0E770480088072801DC6420DAE700206B490870EF
:2048A000B9F1180F0AD16B480068C0F3CF0000EB80004000072190FBF1F011E0B9F1300F96
:2048C0000AD164480068C0F3CF0000EB800040000D2190FBF1F003E05E480068C0F3CF00AF
:2048E00080B25D490880002523E0781EA84205DC4FF00008C4F804800020A9E7B01C30F8A4
:2049000015005549098888420EDC30886843642190FBF1F03188A1EB0008C4F80480781B2B
:20492000401EC0B294E707E04FF00008681C80B20546BD42D9DB86E0484880F800A00078C4
:2049400047490870607C00287AD143F698216069B0FBF1F081B2434802780078401C414B21
:20496000187004F11C0020F81210184600780C2827DBB9F1180F0BD10C2104F11C0003F07A
:20498000DFFD00EB80004000072190FBF1F013E0B9F1300F0BD10C2104F11C0003F0D0FD46
:2049A00000EB800040000D2190FBF1F004E00C2104F11C0003F0C4FD274908800020294952
:2049C0000870002524E0781EA84207DC4FF00008C4F804800020224908701BE0B01C30F85A
:2049E00015001D49098888420EDC30886843642190FBF1F03188A1EB0008C4F80480781B83
:204A0000401E1749087005E04FF00008681C85B2BD42D8DB00BF1248007810490978884292
:204A20000ADD0F4801780D4800781430814203DA0A4800780A4908700020606101206074A3
:204A40000748007804E700BF02E700007E0300207A03002084030020800300207D030020D4
:204A60007C0300207F03002030B51E2A04DB0CDB64280ADA0A2908DA9C891C809C89DC813A
:204A80009C895C8000245C6030BD40F6EB244C43B4EB002F01D2040202E040F6EB244C4317
:204AA000950405EB85056D00B5FBF4F41C801C88B4F5FA7F02DA4FF4FA7407E01C88B4F5BB
:204AC000FA5F02DD4FF4FA5400E01C881C801D885C68C4EB85245D6805EB64145C605C687F
:204AE000C4F38F245C805C88DC8100BFCCE7000038B504460B48012300220A2100900A48E0
:204B000008F0BAF90948012300220A210090084808F0B2F90348007804490978084020703C
:204B200038BD0000520400207C1D002053040020901D002000BFFEE710B5024804F0C8FF9F
:204B400010BD00004424002000B58BB0002006900790012008904CF2200001900020029069
:204B60004DF2E01003904FF6FF700490002005900120099001A9244804F00AFF20B140F2A6
:204B8000491122A011F02CFE0120069000200790012008904FF460400190002002904CF243
:204BA000E01003904FF6FF700490002005900120099001A9144804F0EBFE20B14FF4AF71A4
:204BC00012A011F00DFE0220069000200790012008904FF240500190002002904FF6C07066
:204BE00003904FF6FF70049001200590099001A9054804F0CDFE20B140F2731103A011F0AA
:204C0000EFFD0BB000BD0000442400202E2E5C436F72655C5372635C63616E2E63000000C4
:204C20002DE9F04104460D46002700260DB9666B00E0A66B206800F5D87000EB051000688E
:204C400000F00400B060B06858B9206800F5D87000EB0510006840F2FF7101EA505030603D
:204C60000AE0206800F5D87000EB051000686FF0604101EAD0007060206800F5D87000EBE2
:204C80000510006800F00200F060206800F5D87000EB0510406800F00F0030613562206839
:204CA00000F5D87000EB05104068C0F30720F061206800F5D87000EB05108068307520680A
:204CC00000F5D87000EB05108068010A7175206800F5D87000EB05108068010CB175206856
:204CE00000F5D87000EB05108068000EF075206800F5D87000EB0510C0683076206800F50C
:204D0000D87000EB0510C068010A7176206800F5D87000EB0510C068010CB176206800F593
:204D2000D87000EB0510C068000EF0764DB920202168C8602068406920F00A00216848611B
:204D400008E02020216808612068406920F050002168486194F83C70222F01D0322F05D1E5
:204D60002068406920F40F4021684861EDB994F83C00422804D0622806D072280CD107E003
:204D8000122084F83C000BE0322084F83C0007E0522084F83C0003E0012084F83C0000BFA8
:204DA00000BF204605F01CF91CE094F83C00522804D0622806D072280CD107E0122084F846
:204DC0003C000BE0222084F83C0007E0422084F83C0003E0012084F83C0000BF00BF204611
:204DE00005F0C6F80020BDE8F08100002DE9F34F83B0044660790B287EDB0021204611F008
:204E000039FE00906449009808700121204611F031FE8246604981F801A0009855286CD179
:204E2000BAF1AA0FFBD12088000A88702078C8700221204611F01EFE064657490E71112E78
:204E400003D0162E01D00C2E7ED10321204611F011FE8046504880F805800521204611F05F
:204E600009FE83460421204611F004FE0BEB00201FFA80F94FEA19204749887181F8079021
:204E80000521204611F0F6FD0546A8EB0500022872D1617908F10900814217DA207C0128ED
:204EA00004D105F021FFE0600020207405F01CFFE168411A0498814205D96179204611F0E2
:204EC00095FD0120207405B0BDE8F08F0120207400270EE0B81DC1B2204611F0CBFD2F49F9
:204EE000C8550846C15D07F108002B4A1154781C87B2AF42EEDB01E04CE047E0A81DC1B25C
:204F0000204611F0B7FD4FEA006BE81DC1B2204611F0B0FD0BEB004B05F10800C1B220462E
:204F200011F0A8FD0BEB002B05F10900C1B2204611F0A0FD0BEB0001019105F1080116484E
:204F400000F038F9029000E01BE0DDE90110081A0CD12088114B4A46314600F0FFFE08F1FC
:204F60000900C1B2204611F041FDACE70121204611F03CFD0EE0FFE70121204611F036FD2B
:204F800008E00121204611F031FD03E00121204611F02CFD00BF96E73F0D0020400C0020C9
:204FA00030B50A4600211CE00F4B5B6B14335B5CC57884686355C3785B1CDBB2C370847832
:204FC000A34201DB0023C37043795B1CDBB243718478A34203DD83784371012383714B1C57
:204FE000D9B29142E0DB30BD442400202DE9F047824688461446002C5FDD2046E11704EB31
:205000005171C910A4EBC1018FB237B90827E11704EB5171C1F3CF0907E02046E11704EBDB
:205020005171C910491C1FFA81F92548006BC0F800A000202249096BC8602149096B8860C0
:2050400000261CE008201E49096B086100250AE0082000FB065018F800101948006B14300A
:205060004155681C85B2082DF2DB0A21144805F027F8012801D10CF035FD701C86B2A9F1BB
:205080000100B042DEDC0E48006B076100250AE0082000FB065018F800100948006B143092
:2050A0004155681C85B2BD42F2DB0A21044805F007F8012801D10CF015FDBDE8F087000043
:2050C0004424002010B504462068406920F001002168486194F83C00122805D120684069BC
:2050E00020F40F402168486194F83C00422804D0522806D072280CD107E0222084F83C006D
:205100000BE0322084F83C0007E0622084F83C0003E0012084F83C0000BF00BF204605F0E4
:2051200027F9002010BD000010B5014600224C69CB69552008600A68552A01D0002010BDBF
:20514000A82008600A6802F0A802A82A01D00020F5E70A4848614A69824201D00020EEE73A
:20516000074848614A69824201D00020E7E74C61CB614FF4004008600120E0E755050100FA
:205180002A8A020030B503460C460021002200BF09E0985C80EA1120C0B2054D35F810005E
:2051A00080EA0121521CA242F3D388B230BD000004800108F0B502460B460025681E00218D
:2051C0000FE0565C7040002407E0060E064F57F8265000026840661CB4B2042CF5DB4E1C49
:2051E000B1B29942EDDBF0BD0482010800B585B000BF1848806940F00400164988610846B1
:20520000806900F00400009000BF00BF00BF0846806940F0080088610846806900F008005D
:20522000009000BF00BF08200190002002900120039001A9084805F0B7FB4FF4004001908C
:20524000002002900120039001A9044805F0ACFB05B000BD00100240000C014000080140FC
:205260002DE9F84F04460D4616461F4600F0FAF8009000F0F7F8804600F0F4F88146009821
:20528000404504D1C84502D16A4880F800906A48007830B9674800786649487001206649A9
:2052A00008706448007863494978884238D0614840786049097801F00301604A515C884272
:2052C00009D1002060705E4908805E4908806068401C606024E0574840785649097801F056
:2052E0000301594A515C88420DD155480088401C5349088008460088042811DB012060702E
:20530000002008800CE04F480088401C4D490880084600880A2803DD0120607000200880DF
:205320004FF0020A4348007800F001004149497801F0010188422DD005F0D6FC4349096865
:20534000401A4FF47A71B1FBF0F04149088005F0CBFC3E49086017B94FF0010A00E0B2468A
:20536000607858B93B480078401C3A49087008460078504504DB0120A07001E00020A07076
:2053800035490888012111F0B5FE208105F0ACFC32490860324800682D490988C0EB8120D3
:2053A0002F49096801EB20202D49086008460068C0F3872020704FF0640B2548008814287B
:2053C00002DA4FF496700DE021480088282801DD642007E01E48008800EB80004FF4FA712A
:2053E000A1EB40001FFA80FB0BFB05F0642190FBF1F085B205F078FC18490968401AA842AB
:2054000011D90020A070022060700020207010490880134908600F4908700F490888002152
:2054200011F068FE20810348007802494870BDE8F88F0000C0030020C2030020FE7E010825
:20544000C4030020C6030020027F0108C8030020D0030020D203002032050020D4030020D1
:20546000CC03002070B54FF40041084805F02AFC05462C460821064805F024FC064644EA66
:205480004600C4B204F0030070BD000000080140000C014000BF084A1268526A91B201EB20
:2054A000810292004FF47A7392FBF3F202800022014B1B685A6270475C1E002010B54FF4AD
:2054C000FA710948FFF792FC4FF4FA710748FFF78DFC4FF4FA710648FFF788FC4FF4FA71EC
:2054E0000448FFF783FC10BDA0050020B4050020C8050020DC050020F0B58DB007460E460F
:20550000154618A103C9CDE90B0118A103C9CDE9070109AB002231460BA811F015FB05ABE5
:205520000022314607A811F00FFB002405E009A8005D01A90855601CC4B2082CF7DB0024DE
:2055400007E005A8015D01AA04F108001154601CC4B2082CF5DB294601A801F000FD0DB093
:20556000F0BD000039FF6C063454333029270957FFFFFFFF30B502460B460021002400BFBB
:205580000EE0481C84B207E0505C155DA84201D1002030BD601C84B29C42F5DB481C81B2BE
:2055A0009942EEDB0120F4E731B581B0BDF80400ADF80000BDF9040044F6E61500FB05F1F6
:2055C000C913BDF9060000FB05F2D2130C4613466042C01AC01A00B2ADF8020000983CBD71
:2055E00070B504460AB9084670BD081B800290FBF2F086B2934202DD0D462846F4E706FB63
:2056000003F004EBA02085B22846EDE710B510224F4950480DF0E4FA044624B910224C497F
:205620004D48FEF73CFA102249494A4814300DF0D7FA04462CB91022454947481030FEF78F
:205640002EFA20224249434828300DF0C9FA044624B920223E494148FEF721FA10223C4972
:205660003C484C300DF0BCFA044624B9102238493B48FEF714FA10223549364860300DF05C
:20568000AFFA044624B9102231493648FEF707FA10222F492F4874300DF0A2FA044624B995
:2056A00010222B493048FEF7FAF920222849294888300DF095FA044624B9202224492B4833
:2056C000FEF7EDF92948007829490870202220492048AC300DF084FA044624B920221C49E4
:2056E0002448FEF7DCF9102219491A48D0300DF077FA044624B9102215491F48FEF7CFF935
:20570000082213491348E4300DF06AFA04462CB91A480F490A68026049684160CC220C49E1
:205720000C48F0300DF05CFA044624B9CC2208491348FEF7B4F92022054912480DF050FA0E
:20574000044624B9202202490F48FEF7A8F910BD7C17002008FC01081C090020400B00206B
:20576000600B0020700B0020800B0020B00A0020B9010020D00A0020F00A0020C0040020AC
:20578000B4090020C8FD01089001002010B50446684B0C220421204602F01AFF401C28B9EA
:2057A000644B0C220421204602F012FF624B01221221204602F00CFF401C28B95E4B01220F
:2057C0001221204602F004FF5B4B183B18221521204602F0FDFE401C30B9574B183B18220B
:2057E0001521204602F0F4FE544B01222F21204602F0EEFE401C28B9504B01222F21204622
:2058000002F0E6FE4D4B183B18223221204602F0DFFE401C30B9494B183B182232212046E6
:2058200002F0D6FE464B01224C21204602F0D0FE401C28B9424B01224C21204602F0C8FEE3
:205840003F4B183B18224F21204602F0C1FE401C30B93B4B183B18224F21204602F0B8FED4
:20586000384B30226921204602F0B2FE401C28B9344B30226921204602F0AAFE3148006848
:20588000401C304908600B463022692120460EF028FD401C28B92B4B3022692120460EF022
:2058A00020FD294B10229B21204602F091FE401C28B9254B10229B21204602F089FE234B9A
:2058C0001022AD21204602F083FE401C28B91F4B1022AD21204602F07BFE1D4B0822C32101
:2058E000204602F075FE401C28B9194B0822C321204602F06DFE174B1022CD21204602F091
:2059000067FE401C28B9134B1022CD21204602F05FFE114B0222DF21204602F059FE401C27
:2059200028B90D4B0222DF21204602F051FE002010BD0000C40B00200816002022160020F1
:205940003C160020000B0020300B0020200C0020BB010020300C0020120400201CB5334948
:20596000334801F0C9FD10223249314808300EF055FC10222F4910312D481C300EF04EFC54
:2059800020222D492A4830300EF048FC10222B49274854300EF042FC1022294924486830BE
:2059A0000EF03CFC1022274921487C300EF036FC202225491E4890300EF030FC202223491C
:2059C0001B48B4300EF02AFC102221491848D8300EF024FC08221F491548EC300EF01EFC17
:2059E000CC221D491248F8300EF018FC20221B491B480EF013FC1B480078000619494978A5
:205A000000EB01401749897800EB01201549C9780844009004211348FFF7CCFB0190022280
:205A20006946034801F03AFF1CBD0000FFFF010800FC01081C090020400B0020600B002022
:205A4000700B0020800B0020B00A0020D00A0020F00A0020C0040020B409002090010020A0
:205A6000C8FD0108067F010838B50546002410F055FE10F02DFE284601F0C8FB284601F06F
:205A800081FB1F48008800909DF800200021284601F0A8FC401C28B99DF8002000212846B1
:205AA00001F0A0FC9DF801200121284601F09AFC401C28B99DF801200121284601F092FC8A
:205AC00002216846FFF75EFB044622120221284601F088FC401C20B922120221284601F037
:205AE00081FCE2B20321284601F07CFC401C20B9E2B20321284601F075FC002038BD0000C8
:205B00000A7F010810B5094A0949A2F10C00FFF7F3FC064B0C22042106480EF0E2FB0648EA
:205B2000006820F400100449086010BDC40B0020BB010020400400208C01002070B505460B
:205B4000002639480078C8B9002404E03748C0880644601C84B20A2CF8DB0A20B6FBF0F016
:205B60003349088005F0C0F83249086005F0BCF83149086001202C4908704FE005F0B4F828
:205B80002D490968401AB0F5FA7F03D905F0ACF8284908602868C0F3804000283ED105F029
:205BA000A3F824490968401AB0F5FA6F36D9002404E01E48C0880644601C84B20A2CF8DB3A
:205BC0000A20B6FBF0F01A49088008460088B0F57A7F05DB0846008840F6B831884219DD16
:205BE000286820F4802000F5802028600720134948800F4800888880084601F051FD002065
:205C00000F4908700F484089401C0E49488102200D49087005F068F80649086005F064F8CB
:205C20000549086070BD000040000020DC1E0020480500204400002048000020980700200F
:205C400091030020300B0020BA01002010B5024804F010FC10BD0000681F00203FB5044699
:205C600000252068009060680190A0680290E06803900020206045F25550206025688542C9
:205C800002D0002004B030BD0020206042F6AA2020602568854201D00020F3E70020206090
:205CA00045F25550606005200DF04EFF656845F25550854201D00020E4E74AF6AA206060E3
:205CC00005200DF041FF65684AF6AA20854201D00020D7E74FF05530A060A568B5F1553F0A
:205CE00001D00020CEE74FF0AA30A060A568B5F1AA3F01D00020C5E74FF05530E060E5685B
:205D0000B5F1553F01D00020BCE74FF0AA30E060E568B5F1AA3F01D00020B3E7019860609C
:205D20000298A0600398E060009820600120A9E730B590F840500124AC40C56B6C600468AF
:205D400063604468102C04D10468A2600468E16003E00468A1600468E26030BD2DE9F84F60
:205D60000746884615461C4605F0FF0A40F23171781A8F4274D00CDCA7F25160002801F087
:205D80009B80CF280ED0D0280DD0DF2841F0AD8065E00F287ED010287DD01F287CD02028AF
:205DA000F4D1A0E300BF41F20C61681A8D4236D00BDCA5F58050A0F1100070B1B0F53E7F70
:205DC00023D0B0F5806F45D123E0B0F5807F2CD0A0F5C850F93878BB2FE052462146FE481E
:205DE000FDF75DFEFC48407AFC49C8730020FC49887604F079FFFA49C8610020F9490870C1
:205E000004F072FFF749486025E001200CF0CCFB21E052462146F448FDF741FE1BE052464A
:205E20002146F248FDF73BFE15E052462146EF480C30FDF734FE0EE00CE052462146ECA0A2
:205E4000FDF764FE28B9EC48007820F00100EA49087000E000BF00BF01F048B800E000BFB5
:205E6000B5F5545F7ED025DC43F20511A5EB01008D4279D014DCA5F58050A0F10800B0B32C
:205E8000B0F5017F38D0B0F5417F3BD0A0F5F850FA3802E01FE21FE224E3002871D138E0E9
:205EA000A0F2031000286FD0F8287ED0B0F5007FF4D1B0E0B5F5824F74D00DDCA5F5585005
:205EC000A0F1050000286ED0A0F2FB2000286BD0B0F5E16FE2D13EE1A5F584400838002829
:205EE0007ED0F8287DD0B0F5067FD7D1D3E1FFE701200CF059FBECE152462146BF48FDF743
:205F0000CEFDE6E152462146BC480C30FDF7C7FDDFE1BB48007801280DD052462146B948B7
:205F2000FDF7BDFDB7480078C043B7490870B5484078C0434870B3480078A8494873B14839
:205F4000407888730B464FF481520C214FF4E2600EF066FA0020AD49087004F0C5FEAB49DE
:205F60004860B6E191E0FFE752462146A0A0FDF7CDFD28B9A048007820F002009E490870DC
:205F8000A7E1A5E100E010E052462146A048FDF786FDA0A345F203320C2140F213700EF036
:205FA0003FFA96E1E5E079E0ACE0202221469A480CF016FE202221469848FDF770FD974823
:205FC000007B207095484078607094480079A0709248C07EE070012020710F20607101E0F1
:205FE000CEE0E0E02022A11D8B4824300CF0F8FD2022A11D8A48FDF752FD8948007CA071A8
:206000000020E071234645F208420C2140F213700EF006FA5DE1207840B28049C876084628
:2060200090F91B000A2801DD0A20C8767B4890F91B0010F10A0F02DAF6207849C8766078FA
:2060400076494870207940B275490874084690F91000002802DD0020087408E0704890F951
:20606000100010F1140F02DAEC206D49087400206C49087001F068FF66A345F203320C218B
:2060800040F213700EF0CCF923E1674B41F210520C214FF4E2600EF0C3F91AE152462146D7
:2060A00062A0FDF733FD60BB00205F498860C8600922604960A0FDF729FD80B15A4800689E
:2060C000B0F57A7F03D20020574908604860092259A15848FDF707FD002052490870524BF0
:2060E0001022AD2157480EF0FCF84AA345F203320C2140F213700EF093F90020374908831F
:206100004883E6E05048007820BB10224F49424888380CF065FD10224C4910313E48743857
:206120000CF05EFD0C214A48FFF744F806464748C66203464FF492520C214FF4E2600EF0F4
:206140006FF9444B4FF4B9520C214FF4E2600EF067F900BFBDE0524621463F48FDF79FFC79
:206160002CA345F203320C2140F213700EF058F9AFE03A4A3A493B48007802F02BF9A8E084
:20618000524621463648FDF78AFC00202549087001F0DAFE1FA345F203320C2140F2137029
:2061A0000EF03EF995E0202221461B480CF018FD202221461948FDF772FC202221461648A5
:2061C00024300CF00DFD202221461548FDF767FC12480E30016847E07C090020DC08002037
:2061E00008030020E8010020A40900208C0900205245414459000000B0010020800A0020F9
:20620000D8000020DA000020DC000020D8010020B101002041434B0090FC0108B00A002087
:20622000D00A002039040020200C0020434C454152000000600B0020434C4541525F4F4470
:206240004F00000040040020FE0100201C090020B80B00205C090020B80400209804002027
:20626000C0040020C904002021604168616000892081F7480168C4F80A104168C4F80E1037
:2062800000896082234645F220620C2140F213700EF0C6F81DE0EF4821680160616841604B
:2062A00021890181EA48D4F80A100160D4F80E104160618A01810020E7490870AFF2AC0329
:2062C00045F203320C2140F213700EF0A9F800E000BF00BFC0E500BFB5F5445F5ED010DCA8
:2062E000A5F58050A0F58670C8B1B0F5807F1CD0B0F57F7F20D0A0F5F050F438002872D1A1
:2063000022E0A5F548500838F0B3FD286CD0B0F5FC7F6AD0A0F2FD200028F0D1A7E05246F4
:206320002146CE48FDF7BBFBDAE052462146CB480C30FDF7B4FBD3E00020C949087004F03A
:20634000D3FCC7494860CBE0C648007828BB1022C549C6480CF044FC1022C3491031C3488E
:2063600014300CF03DFC0C21C148FEF723FF0646BD48C66203464FF492520C214FF4E260BC
:206380000EF04EF8BB4B00E030E04FF4B9520C214FF4E2600EF044F800BFA1E020222146A0
:2063A000B24888300CF01CFC20222146A9480E38FDF775FBA7480E38007B2070A5480E3860
:2063C00040786070A3480E380079A070A1480E38C07EE070234647F208320C2140F21470FF
:2063E0000EF01EF87CE07AE02AE037E0207840B298490E39C876084690F91B000A2801DDC0
:206400000A20C87693480E3890F91B0010F10A0F03DAF6208F490E39C87660788D490E39F0
:20642000487000208C49087001F08EFDAFF21C2347F203420C2140F214700DF0F1FF4FE05E
:2064400052462146AFF25820FDF760FB28B98A48007820F004008849087041E0874B41F227
:2064600010520C214FF4E2600DF0DAFF38E052462146AFF24820FDF749FB78BB00207F49BF
:206480008860C86009227E49AFF25420FDF73EFB88B17A480068B0F57A7F03D20020774902
:2064A000086048600922AFF270217548FDF71BFB002069490870714B1022AD2171480DF0EC
:2064C00010FFAFF2B02347F203420C2140F214700DF0A6FF00206C490883488300BF00BF8D
:2064E00000BFB9E400BF42F20561681A8D4276D05ADCB5F5D95F73D02EDCB5F5A85F70D0FA
:2065000015DCB5F5905F6DD008DCB5F5805F6AD0A5F58850083800286FD1E1E0B5F5985F91
:206520006CD0A5F5A05010380028F5D131E141F61001681A8D426ED008DCA5F58050A0F593
:20654000C260002868D0F028E6D155E1F12879D0B0F5F87FE0D18CE1B5F5045F73D013DCD9
:20656000B5F5F05F70D008DCB5F5E05F6DD0A5F5E85010380028CFD1B5E1B5F5F85F65D02A
:20658000B5F5005FC8D1E0E1A5F50850103800285DD0B0F5807F79D0B0F5047F77D0A0F21B
:2065A000F5200028B8D113E240F6FB12811A90426ED032DC40F2FC52A0EB0201904268D00C
:2065C0001DDC40F2FB22A0EB0201904276D00BDCA0F20310002872D0FA289DD15AE212E217
:2065E00056E1E8E09AE06CE0A1F20110002867D0A0F2011000288FD1B4E2EEE3B6E0A1F218
:20660000071100297DD0E8297CD0F8297BD0B1F5FC7F8AD141E3FEE0DCE040F60912881AF6
:20662000914271D03DDC40F20132A1EB020091426BD02FDCB1F5907F68D0A1F20121002956
:2066400088D153E3F9E081E15FE13DE16EE186E1E20A0020BE0A002039040020980A002049
:20666000E0010020FE0100201C09002008FC0108B80B00205C090020B0010020200C002023
:20668000600B002040040020DC0800207BE18DE10CE37CE2A0F20110002876D0FE289CD14C
:2066A0009CE3A0F2C310002870D044286FD0B0F59A7F6DD0B0F5157F8FD1E8E350E2CDE1A4
:2066C0004FE2FE4B0822C321FD4801F081FFFB4B4AF208420C2140F215700DF0A1FEE9E364
:2066E00052462146F548FDF7DAF9F44B0822C321F3480DF0F6FDAFF2E4434AF603120C21D5
:2067000005E048E279E2BFE277E31DE3DCE24FF4E2600DF085FEFFF7F5F9CBE3E948007816
:2067200018BB1022E849E9480CF05AFA1022E6491031E64814300CF053FA0C21E448FEF7F7
:2067400039FD0646E048C66203464FF492520C214FF4E2600DF064FEDE4B4FF4B9520C2142
:206760004FF4E2600DF05CFE00BFA3E31022DA49D6484C300CF034FAD74B4AF210620C21E2
:2067800040F215700DF04CFE94E3F3E24AE35BE36FE352462146D048FDF781F90020CF4935
:2067A0000870AFF290534AF603120C214FF4E2600DF036FE7EE31022C949C44860300CF068
:2067C0000FFAC74B4AF210720C2140F215700DF027FE6FE352462146C148FDF760F9002013
:2067E000BE490870AFF2D4534AF603120C214FF4E2600DF015FE5DE31022BA49B348743027
:206800000CF0EEF9B74B4AF610020C2140F215700DF006FE4EE352462146B248FDF73FF906
:206820000020AE490870AFF214634AF603120C214FF4E2600DF0F4FD3CE32078AA4908709A
:2068400008460078C043A9490870A748007878B1A748006820F48060A5490860084600681E
:2068600020F4805008600846006820F40060086020E320222146954888300CF0B1F92346EA
:206880004AF220020C2140F215700DF0C9FD11E3524621469748FDF702F9964800789649FD
:2068A000087000208D4908709249487B0FF086FA01F04AFBAFF2A4634AF603120C2140F243
:2068C00015700DF0ADFDF5E2102221467F48D0300CF086F923464AF210120C2140F215702F
:2068E0000DF09EFDE6E2524621468448FDF7D7F800207A490870AFF2E4634AF603120C21E5
:2069000040F215700DF08CFDD4E27D4B4AF230220C2140F215700DF083FD7A4B4AF6104276
:206920000C2140F215700DF07BFDC3E220227649664828300CF054F9734B4AF220520C2170
:2069400040F215700DF06CFDB4E2B3E26F4B41F201420C214FF4E2600DF062FDAAE252468D
:2069600021465948FDF79BF800205C490870AFF25C734AF603120C214FF4E2600DF050FD8A
:20698000FFF7C0F896E2524621464F481030FDF786F8002051490870AFF288734AF6031266
:2069A0000C214FF4E2600DF03BFD83E2524621465548FDF774F8002048490870AFF2AC73A6
:2069C0004AF603120C214FF4E2600DF029FD71E2524621464EA0FDF799F898B9AFF2CC7397
:2069E0004AF603120C2140F215700DF019FD00200BF0DAFD642003F091FE01200FF0C8FF6C
:206A000004F094FA56E252462146AFF2E070FDF77DF810BBFF2304220021294800F084FB4F
:206A2000FF236D226921264800F07EFB3A492748083800F061FD3949394800F05DFDAFF6D2
:206A40002C034AF603120C2140F215700DF0E8FC01200FF09DFF04F069FA2BE252462146CE
:206A600030A0FDF753F8A0B90FF058FE144800F0CDFBFEF773FFAFF664034AF603120C2150
:206A800040F215700DF0CCFC01200FF081FF04F04DFA0FE2524621462548FDF700F82448EA
:206AA0000078C0432349087021484078C043487000202149087004F017F93FE0BB0100209A
:206AC00040040020FE0100201C09002008FC0108B80B00205C090020600B00203904002091
:206AE000700B0020800B0020D8000020D90000208C010020B00A0020B9010020F00A0020E4
:206B0000000B0020300B0020400B0020B00100205245534554000000FFFF0108FFF301082E
:206B200000F001085245434F5645525900000000DA000020DC000020D8010020ED49486020
:206B4000ED480078ED494873EB48407888730B464FF481520C214FF4E2600DF061FCA9E1B4
:206B6000A8E1A7E152462146E548FCF798FFE44B0222DF21E3480DF0B4FBAFF668134AF6C4
:206B800003120C2140F215700DF04AFC92E12078DD4908708EE100BF20790006617900EB7E
:206BA0000140A17900EB0120E179084421780906627801EB0241A27801EB0221E27811443F
:206BC000401A461C20780006627800EB0240A27800EB0220E2788118324604F10800FCF7D2
:206BE0005EFF4AF60830304482B223460C2140F215700DF015FC00BF5CE100BF2078000664
:206C0000617800EB0140A17800EB0120E178461820790006617900EB0140A17900EB0120C8
:206C2000E17900EB010BABEB060000F10109B6F1005F0FD94A4604F108013046FCF72FFF59
:206C4000AFF630234AF603120C2140F215700DF0E7FB17E0AD48864214D906F2FF313046E5
:206C600000F04AFC09F0FF0204F1080130460DF0D5FAAFF660234AF603120C2140F2157043
:206C80000DF0CEFB00BF00BFA14B41F210520C214FF4E2600DF0C4FB0CE19E4B41F208624E
:206CA0000C214FF4E2600DF0BBFB03E12022214699480BF095FF23464AF620520C2140F2F8
:206CC00015700DF0ADFBF5E0524621469348FCF7E6FE002092490870AFF6C8234AF60312AC
:206CE0000C2140F215700DF09BFBE3E02078401E00EB4002C2EB40101530C1B2631C1822C9
:206D0000804801F065FC2078012804D0022807D003280FD109E08348C08AA4F8170009E01E
:206D20008148C08AA4F8170004E08048C08AA4F8170000BF00BF23464AF61A620C2140F2E2
:206D400015700DF06DFBB5E02078401E00EB4002C2EB40101230C1B2631C0122694801F09B
:206D600037FC23464AF602720C2140F215700DF057FB9FE0207801280AD16078694908766D
:206D800001F11803012212215E480DF0AAFA1AE0207802280AD160786349087601F11803A3
:206DA00001222F2157480DF09CFA0CE02078032809D160785D49087601F1180301224C210C
:206DC00050480DF08EFAAFF6B4334AF603120C2140F215700DF024FB6CE06AE02346022292
:206DE000DF21484801F0F4FB23464BF202020C2140F215700DF014FB5CE0524621464CA062
:206E0000FCF784FE68B90FF063FC3E4800F0BAF9AFF600434AF603120C2140F215700DF037
:206E2000FFFA47E0524621464448FCF738FE00203B490870AFF624434AF603120C2140F2A2
:206E400015700DF0EDFA35E0524621463048FCF726FE2F4B1022AD212A480DF042FAAFF65C
:206E60004C434AF603120C2140F215700DF0D8FA20E02022324933480BF0B2FE304B4BF6DC
:206E800020320C2140F215700DF0CAFA12E0524621462B48FCF703FE002021490870AFF6FC
:206EA0008C434AF603120C214FF4E2600DF0B8FA00E000BF00BF19E0A5F51450053820B1EA
:206EC000A0F5F840063828B900E000BF02201E49087000E000BF00BF2B46424640F25161EB
:206EE0001A4800940DF0E8FA00E000BF00BFBDE8F88F0000D8010020DA000020DC0800203C
:206F00001204002040040020CF01002000300008200C0020F0010020B4FC0108D00A00209F
:206F200039040020F01500200A160020241600204C4F4720434C454152000000B4090020EF
:206F400090010020C8FD01085D00002000060020704700BF0100A0F10100FBD1704710B5BE
:206F60000246002016E0135C041D145D63400B54031DD35C00F10804145D6340041D0B55CF
:206F8000231DD35C0834145D634000F108040B55431CD8B20428E6DB10BD000010B503F07A
:206FA000A3FE14490968401AB0F5FA7F21D303F09BFE104908601048007858B90FA343F2E1
:206FC0000902112140F212700DF02AFA01200A4908700EE00848007801280AD107A345F218
:206FE0000902112140F213700DF01AFA00200249087010BDD0000020D400002048414E44DF
:207000005348414B450000001FB54FF46040009011200190022003906946194803F0C4FC83
:207020004FF4E060009011200190022003906946144803F0B9FC00224FF48071114803F071
:207040004DFE00224FF400710E4803F047FE00224FF480610B4803F041FE00224FF4005100
:20706000074803F03BFE00224FF48041044803F035FE00224FF40041014803F02FFE1FBD12
:20708000000C01400008014010B500210D4805F019F904210B4805F015F90821094805F02E
:2070A00011F90021074804F0ADFD0421054804F0A9FD0821034804F0A5FD0C21014805F037
:2070C000E1F810BD1C1E0020F8B50446002000906A460021204600F02FF90DF10102012197
:2070E000204600F029F902216846FEF74BF806466A460221204600F01FF90DF1010203215D
:20710000204600F019F99DF801009DF8001000EB012085B2A81B03D12046FEF737FBF8BDB0
:207120002046FEF7A1FCFAE72DE9F04780460C4616461F46301B00F0FF09002507E0601988
:20714000C1B23A46404600F04DF9681CC5B24D45F5DBBDE8F08700001FB504460220009037
:207160000120019003906946054803F01DFC01220221034803F0B2FD204605F0AFFC1FBDAD
:20718000000C014010B504461C4B3022692120460DF0A7F8401C28B9184B3022692120466C
:2071A0000DF09FF8164B10229B2120460DF099F8401C28B9124B10229B2120460DF091F884
:2071C000104B1022AD2120460DF08BF8401C28B90C4B1022AD2120460DF083F80A4B102275
:2071E000CD2120460DF07DF8401C28B9064B1022CD2120460DF075F810BD0000000B002053
:20720000300B0020200C0020300C002010B50446424B0C22042142480DF063F8401C28B95D
:207220003E4B0C2204213E480DF05BF83D4B0122122120460DF055F8401C28B9394B01222A
:20724000122120460DF04DF8364B183B1822152120460DF046F8401C30B9324B183B18221F
:20726000152120460DF03DF82F4B01222F2120460DF037F8401C28B92B4B01222F21204635
:207280000DF02FF8284B183B1822322120460DF028F8401C30B9244B183B182232212046FA
:2072A0000DF01FF8214B01224C2120460DF019F8401C28B91D4B01224C2120460DF011F8A9
:2072C0001A4B183B18224F2120460DF00AF8401C30B9164B183B18224F2120460DF001F8E8
:2072E000134B0822C32120460CF0FBFF401C28B90F4B0822C32120460CF0F3FF0D4B022251
:20730000DF2120460CF0EDFF401C28B9094B0222DF2120460CF0E5FF10BD0000C40B002068
:207320004004002008160020221600203C160020BB010020120400202DE9F04106460F46E7
:2073400015460024304605F03CFCA021304605F07DFC00BF00BF601C84B240F6B830844252
:2073600003DD4FF0FF30BDE8F081304605F096FB0028F0D13946304605F068FC002400BF93
:20738000601C84B240F6B830844202DD4FF0FF30E9E7304605F082FB0028F1D1304605F0FD
:2073A00010FCA121304605F051FC002400BF601C84B240F6B830844202DD4FF0FF30D2E7C8
:2073C000304605F06BFB0028F1D12946304605F0A2FB304605F0D2FB304605F012FC0020AA
:2073E000C1E700002DE9F04106460F461546002400220221294803F071FC304605F0E1FB21
:20740000A021304605F022FC00BF00BF601C84B240F6B830844203DD4FF0FF30BDE8F081AA
:20742000304605F03BFB0028F0D13946304605F00DFC002400BF601C84B240F6B830844256
:2074400002DD4FF0FF30E9E7304605F027FB0028F1D12946304605F0F9FB002400BF601C6B
:2074600084B240F6B830844202DD4FF0FF30D5E7304605F013FB0028F1D1304605F0C1FB5F
:207480000A2003F04BF901220221044803F026FC034803F057FC0020C0E70000000C01403F
:2074A00004080020F8B50E480468001D0568200E8DF80000200C8DF80100200A8DF8020091
:2074C000E0B28DF8030004216846FDF773FE0646701B02D1FEF79AF801E0FEF73FFAF8BD65
:2074E00000FC010810B50446207818B9FEF736FA0120207010BD000038B504460D460020C2
:207500000C49086008468460281B401C800AC86003F0D2F900BF34200749C86000BF694674
:20752000044803F00FF903F065F9642003F0F6F838BD00006C1700200020024010B5042269
:207540000E490F480BF04CFB0446A4B904220B490CA0FCF7DBFA70B928220849084808305A
:207560000BF03EFB044634B9282204490748FCF796FA002010BD0120FCE700007C17002093
:2075800000E80108464C414700000000900B002010B54FF4805003F0F9F910BD10B50420B2
:2075A00003F0F4F910BD00001FB54FF4604000900220019003906946064803F0F5F94FF470
:2075C000E06000900220019003906946024803F0EBF91FBD000C01400008014010B500216D
:2075E000104804F04FFE04210E4804F04BFE08210C4804F047FE0C210A4804F043FE0021AF
:20760000084804F0E9FA0421064804F0E5FA0821044804F0E1FA0C21024804F0DDFA0BF07C
:207620004FF810BD1C1E00202DE9F04107460C46207860BB384600F057F846B2701C48B109
:207640001448402101FB06054022394628460CF01BFE1AE00F49491E0F48FFF74DFFF0229E
:207660000C4940310C4800F019F90C490948FFF743FFF0220849074800F010F9074D3F3D95
:207680004022394628460CF0FFFD01202070BDE8F081000000F0010800EC0108FFF30108F3
:2076A00010B504460B480068A0600B484068E06020220A4904F11000FCF7F1F90848016895
:2076C00021634068606307480168A1634068E06310BD00008C010020000B0020DC0800206B
:2076E000F0010020DE00002010B50246002116E00F4C04EB811003884FF6FF7083420CD19B
:2077000011B90120108006E04020C0EB8110084C035B581C1080084610BD481C41B210290B
:20772000E6DB04480388581C10804FF0FF30F3E700F00108C0F301080021074AD1610749BC
:20774000096941F00401054A11611146096941F040011161704700003007002000200240A3
:207760000021074AD1610749096941F00201054A116111464861096941F0400111617047A1
:2077800030070020002002400022054BDA61054A126942F00102034B1A6101807047000083
:2077A000300700200020024000201E49C96801F0100139B11C49C96941F002011A4AD1610B
:2077C00040F010001749C96801F0040139B11649C96941F00101144AD16140F00400114916
:2077E000C96901F0010169B10F49C96941F004010D4AD16100BF0B49C96921F00101094A56
:20780000D16100BF00BF40F20111884206D10549C96921F00101034AD16101E00149C8606E
:2078200000BF7047002002403007002070B5044603F05AFA054609E0601C38B124B103F002
:2078400053FA401BA04201D9032070BD1248C06800F001000028EFD10F48C06800F020008A
:2078600020B100BF20200C49C86000BF0A48C06800F0100048B90848C06900F0010020B93E
:207880000548C06800F0040018B1FFF78DFF0120DBE70020D9E70000002002402DE9F041C8
:2078A00004460E461746002503F006F800BF0FE056F825C0624600232146022002F0A4FFED
:2078C00008B9241D03E002F095FFBDE8F0816D1CBD4202D203488442EAD902F08BFF00BFBC
:2078E000F3E70000FBFF0108022005490870002004490880488004490880488070470000B2
:2079000030000020280000202C0000200120014908707047300000202DE9FF4704460E469F
:2079200017464FF0000A0CF0CBFB03900398FDF73BFE029039B202980AF0D0FC00908B4844
:2079400000990160B0F9000089490968C1EB80208749096801EBA02085490860084600681C
:20796000801200B2834908808048B0F9020082490968C1EB80208049096801EBA0207E49C7
:20798000086008460068801200B27C4908807C48007C002849D17B480078042845D17A4877
:2079A000408840F6B831884210DA784804607848006810F1040F05DA75480068001D7449EE
:2079C000086077E000207249086073E06E48408840F68A41884221DA6B484088A0F6B83015
:2079E00000EB800040F21A41081A6A49086008460068844201DA204601E0664800686349F2
:207A0000086063480068801E614908600846006810F5D27F4EDA604808604BE000205B4908
:207A200008605D485A49086044E05748408840F61C41884210DA554804605548006810F155
:207A4000040F05DA52480068001D5149086031E000204F4908602DE04B48408840F6EE4115
:207A6000884221DA48484088A0F61C4000EB800040F21A41081A4749086008460068844269
:207A800001DA204601E0434800684049086040480068801E3E4908600846006810F5D27F57
:207AA00008DA3D48086005E00020384908603A4837490860394A2F48B0F9001033480088E9
:207AC00000B20AF0CBFB054635480068C0EB45203349096801EBE000314908603148408818
:207AE000B7214843C0F3CF1947F698107043B9F57A7F02DA4FF47A7100E0494690FBF1FA5A
:207B0000274800680AEB602547F69810854200DD00E02846054628B223490880234A174858
:207B2000B0F900101A48008800B20AF097FB80461F480068C0EB48201D49096801EBE00019
:207B40001B49086008460068401200B21649488008460BF07BF81448006800900BF09CF8D9
:207B6000019001980CF000F8BDE8FF87280000200C00002020000020100000202200002096
:207B8000D8070020DE000020DC1E00200400002008000020240000205CFEFFFF540600206C
:207BA00018000020F00A00202C000020780600201C00002005F098F809F0DCFF0AF07CF886
:207BC00062B60020124981F83C0009F08BFF72B60AF052F80AF07CFDFFF716FA00200D497F
:207BE00008600846006820F4005000F5005008600DE0084B41F204120C214FF4E2600CF01F
:207C00000FFCC8200BF090FF034803F09BF8F0E7442400208C0100200408002070B505466E
:207C20000E46049CAC4208DAFF2E01D100210DE0281B7043C0F5806108E0944202DA4FF40A
:207C4000806103E0A01A5843C0F58061002901DC002000E00846014688B270BD87B00146F5
:207C600000220868009048680190C86803903D4881423AD04FF0553008600A68B2F1553FB7
:207C800002D0002007B070474FF0AA3008600A68B2F1AA3F01D00020F4E74FF055304860CD
:207CA0004A68B2F1553F01D00020EBE74FF0AA3048604A68B2F1AA3F01D00020E2E745F228
:207CC0005550C860CA6890B245F25553984201D00020D7E74AF6AA20C860CA6890B24AF615
:207CE000AA23984235D00020CCE700986FF30B0000F2555008600A68C2F30B0040F25553F5
:207D0000984201D00020BDE700986FF30B0000F6AA2008600A68C2F30B0040F6AA239842B8
:207D200001D00020AEE7039820F00700C01DC860CA6802F00700072801D00020A2E7039897
:207D400020F00700C860CA6802F0070008B1002098E700980860019848600398C86001203C
:207D600090E70000001401402DE9F04104460E46154629480078012812D1284801780078A1
:207D8000401C264A1070264820F8116010460078322810DB002020490870114608700AE0D3
:207DA00032221F4930460AF013F9643087B22088B84200DD00BF2888C0F3C03050BB20887A
:207DC00040F2DC51884203DC02F08EFF1549086002F08AFF13490968401A42F21071884235
:207DE00018D9286820F4004000F50040286001200D494880208888800846FFF751FC002051
:207E00000A4908700A488088401C09498880022008490870BDE8F0818B0400208C04002027
:207E2000B81D0020900400209807002091030020300B0020BA010020B1F5967F03DA012235
:207E4000044B1A7002E00022024B1A7001F16402028070478A04002010B502460020B2F55B
:207E6000FA7F01DC01200EE0B2F5E16F01DB084609E040F2145393FBF1F4A2F5FA7393FBF5
:207E8000F4F35B1CD8B210BD10B50446207800284DD12749087002F027FF25494860608842
:207EA00040F2AA71884236D120792249087060794870A0798870E079C870617A207A01EB94
:207EC00000201C4988801C48807EEE2811D10846808820B94FF6FF701849886009E0154849
:207EE00080884EF6602191FBF0F0144988600020C870A07A0F498871E07AC8710846807967
:207F0000C0F3401018B100200D4908700DE001200B49087009E0608840F2AB71884204D10F
:207F2000084861680160A16841600120207010BDB0040020EC070020B00A0020E4030020D7
:207F4000C90400209404002010B500BF2A480078052803DA05202849087006E0264800782A
:207F6000182802DD18202449087023480078401E43F2C82191FBF0F084B218211F48FCF731
:207F80004AFC00200BE000FB04F10A2291FBF2F101F5FA71194A22F81010411CC8B21649D1
:207FA0000978491E8142EEDC4FF4E16112480078401E124A22F8101000BF00BF1048807932
:207FC00000EB4000C0000A2190FBF1F00D4908700B48C07948700A48007B0949C97E08445B
:207FE00064380849487104484078887002488078C87000BF10BD0000C0040020CA04002007
:20800000B00A00209C04002010B502F06DFE40F6B831884206D9C1480078F02802D1C04967
:20802000C87710BDBF48FFF72FFFBF48007858B902F05AFEBC494968401A40F6B831884236
:2080400002D90120B8490870B4480078202823D040285CD080285BD0F02875D1AF480078C8
:20806000AF49C87700BF02F03FFEB0490968401AC82809D90120AE490870084600F086F9F8
:2080800002F032FEA949086000BFA748007810B92020A24908703DE1A048007800F0E00084
:2080A0009F49C87700BFA3480078052800DB16E002F01AFEA0490968401AC8280ED99F4AFB
:2080C0009F49A048007800F085F902F00DFE9A49086098480078401C9649087000BF00BF19
:2080E0009948007890B198480078032803D140208A4908700AE094480078042803D09248CD
:208100000078082802D180208449087002E100BF8D480078082805D18549087000204880DC
:20812000888054E088480078032829D140207B49087003207E49087083484078012804DA0E
:2081400082480088488017E0E3E07F4840787C490978884208DD7A480078401E7B4931F852
:2081600010007349488007E077484078401E774931F810006E49488000206D49888026E053
:2081800071480078042822D18020644908700420674908706C48407869494978884204DAF7
:2081A00067484078624988800EE06748407864498978884204DD624880785D49888003E0C4
:2081C000614840785A49888000205949488056480078012803D1F0205149C87725E04F4871
:2081E0000078402812D1564A1178594A5278642302FB03F0FFF730FE00F01F00474909786B
:2082000001F0E00108444649C8770EE04348007880280AD14148007800F0E0004C494978D7
:2082200001F01F0108443E49C87700BF02F05CFD48490968401AB0F57A7F39D94248007803
:2082400008280FD144480078052807DA384800F09DF841480078401C3F49087000203F49F2
:20826000087021E03D480078012808DA3C4800F07DF83A480078401C3849087011E03748D5
:20828000007805280DDA2A4800F080F833480078401C3249087008460078052801DB002047
:2082A000087000202C49087002F01EFD2949086000BF00BF022402F017FD2A490968401A6A
:2082C000B0F57A7F23D91F480078012809D100BF1A4A1B49204600F07DF8002022490870CD
:2082E00011E01848007870B900241F480078052809DA124A1249204600F06CF81A4800782E
:20830000401C1949087002F0EFFC1649086000BF00E000BF00BF00BF83E60000C804002052
:20832000DC080020A4040020B0040020FC040020F607002004050020000500209804002056
:20834000C0040020C9040020B8040020CA040020EC070020080500200D0500200C050020DF
:208360009C04002010050020140500201CB5044600200090019020680090606801900822D8
:20838000694640F2AC70FCF731FE1CBD1CB5044600200090019020788DF800006088001272
:2083A0008DF80100A0788DF80200A08800128DF8030020798DF8040000208DF805008DF885
:2083C00006008DF807000822694640F2AD70FCF70DFE1CBD7FB506460C461546002000902F
:2083E0000190029003908DF800602088ADF80100A0788DF8030028788DF804006B4645F2E3
:2084000010520C2140F213700CF00AF87FBD000038B5044601234FF47A720A21024800944B
:2084200004F02AFD38BD0000A41D002030B503460024002204E033F812502C44551CAAB229
:208440008A42F8DBB4FBF1F5A8B230BD70B505462C480078012811D100202A49087002F03D
:2084600043FCB0F5E16F05D902F03EFCC8302649088003E04FF4FA602349088002F034FC39
:208480002149098888423BD920480078012837D11F48007858B11F480088C82807DC40F216
:2084A000C27085420CDD40F63E00854208DA00201949C8720A2219A11B48FBF714FB1CE0BB
:2084C00001201549C872002415E0184830F81400A8420EDB0A2216A11348FBF704FB1748CD
:2084E000015D1148203880F8271000200749087070BD601CC4B2092CE7DB002003490870DC
:2085000000BFF5E79403002092030020FE010020D0010020CC010020D807002054544B5A0B
:2085200030313044343800003C090020C27E010854544B5A3031394134380000D47E01085D
:2085400010B502460B460020002107E032F81140844201DD32F811004C1CA1B29942F5DBD5
:2085600010BD10B502460B464FF6FF70002107E032F81140844201DA32F811004C1CA1B202
:208580009942F5DB10BD00000246002108E0064830F81100904201DC08467047481CC1B200
:2085A000C829F4DB0020F8E7048601080246002108E0064830F81100904201DC08467047DD
:2085C000481CC1B2BF29F4DB0020F8E7948701082DE9F84F82460D4614461F4600260EE09F
:2085E0001C488219A819C1B25046FEF7A5FE401C18B94FF0FF30BDE8F88F701CC6B2A64267
:20860000EEDB21461348FCF7BDFD81462819C1B26A465046FEF790FE2819401CC1B20DF1D0
:2086200001025046FEF788FE9DF801009DF8001000EB01201FFA80F8B8EB090006D1224663
:2086400004493846FBF72BFA0020D4E74FF0FF30D1E700007C1C00202DE9FC5F8046894679
:208660004FF0000A002549464046FFF7DFFE8346002407E038F81400ABEB000505FB05AA42
:20868000601C84B24C45F5DB5046FBF70CFC06460F46304639460EF007FDCDE90001FBF7F6
:2086A0004DFC05462846BDE8FC9F0000F8B5044600260020009000BF94F82400012801D141
:2086C0000220F8BD012084F8240000BF2046FBF701FE0646002E62D1A06A20F4885040F019
:2086E0000200A062022002F043FC30490968B1FBF0F04000009002E00098401E00900098DD
:208700000028F9D12046FBF74DFE2068806840F008002168886002F0E7FA054611E002F0AA
:20872000E3FA401B0A280CD9A06A20F0020040F01000A06200BF002084F8240000BF01202D
:20874000BFE72068806800F008000028E7D12068806840F004002168886002F0C5FA05461A
:2087600011E002F0C1FA401B0A280CD9A06A20F0020040F01000A06200BF002084F824000C
:2087800000BF01209DE72068806800F004000028E7D1A06A20F0020040F00100A06200BF23
:2087A000002084F8240000BF30468AE70000002038B50246002300200090906800B100BFC3
:2087C00000BF92F82400012801D1022038BD012082F8240000BF906890B94868012809D1A8
:2087E0001068806B6FF315000C6840EAC4301468A06338E0906A40F020009062012332E004
:208800000C694868A0421ED84C680869001BC0F1030000EB80041F20A04040F440141068D9
:20882000806BA0434D680C69641BC4F1030404EB84050C68AC400D8A6D1E44EA0554204321
:208840001468A0630FE04C680869001BC0F1030000EB80041F20A04040F440141068806B3D
:20886000A0431468A0631068806800F0010040B91068806847F20104A043CC6920431468B7
:20888000A060886901280FD1C869B0F5E04F06D11068406840F480601468606004E0906AB4
:2088A00040F0200090620123486901280DD1886930B91068406840F480501468606004E07C
:2088C000906A40F020009062012308680A2812D31068C0680C780A3C04EB44050724AC40F8
:2088E000A0430D780A3D05EB45058C68AC4020431468E0600FE0106800690C7804EB440504
:208900000724AC40A0430D7805EB45058C68AC402043146820610868102802D0086811283B
:2089200005D11068806840F400001468A0604868012806D002280DD0032814D004281BD174
:208940001BE0106840696FF30B00CC682043146860611BE0106880696FF30B00CC6820435A
:208960001468A06112E01068C0696FF30B00CC6820431468E06109E000BF1068006A6FF33A
:208980000B00CC6820431468206200BF00BF0868102802D00868112827D1174C1068A042E1
:2089A0001ED11068806800F40000F0B91068806840F400001468A0600868102815D10F48D6
:2089C00000680F4CB0FBF4F000EB80004000009002E00098401E009000980028F9D104E034
:2089E000906A40F020009062012300BF002082F8240000BF1846E9E6002401400000002029
:208A000040420F0010B504460121204600F044F84FF6FF7101EA00101A494880022120469E
:208A200000F03AF84FF6FF7101EA0010154988800321204600F030F84FF6FF7101EA0010AC
:208A400010490880104800880988401A00B20F4908800D4840880B494988401A00B20B4936
:208A600048800948808807498988401A00B2074988800749054809F079FC0120054908701E
:208A800010BD000024050020360500203C05002042050020300500200246002001290FD0D7
:208AA000022909D0032904D0042908D11368986C09E01368586C06E01368186C03E000BF7E
:208AC0001368D86B00BF00BF7047000070B50446002500BF94F82400012801D1022070BD56
:208AE000012084F8240000BF2046FBF75BFC0546002D5BD1A06A42F20101884340F4805094
:208B0000A0622E492068884208D12D48006800F4702008B9012002E0002000E0012020B19A
:208B2000A06A20F48010A06203E0A06A40F48010A062A06A00F4807008B90020E06200BF02
:208B4000002084F8240000BF401F216808602068406840F08000216848602068406800F411
:208B6000806010BB2068806800F4E040B0F5E04F15D112492068884208D11148006800F4D1
:208B8000702008B9012002E0002000E0012030B12068806840F40210216888600BE02068E5
:208BA000806840F400402168886004E000BF002084F8240000BF284691E700000028014077
:208BC0000424014038B5024600230020009000BF92F82400012801D1022038BD012082F80A
:208BE000240000BF4868072812D21068406B0C79641E04EB84051F24AC40A0430D796D1E0A
:208C000005EB85050C68AC4020431468606327E048680D2812D21068006B0C79E41F04EBAE
:208C200084051F24AC40A0430D79ED1F05EB85050C68AC4020431468206311E01068C06A38
:208C40000C790D3C04EB84051F24AC40A0430D790D3D05EB85050C68AC4020431468E062F1
:208C600008680A2812D31068C0680C780A3C04EB44050724AC40A0430D780A3D05EB4505CB
:208C80008C68AC4020431468E0600FE0106800690C7804EB44050724AC40A0430D7805EBDA
:208CA00045058C68AC402043146820610868102802D00868112827D1174C1068A0421ED163
:208CC0001068806800F40000F0B91068806840F400001468A0600868102815D10F4800683A
:208CE0000F4CB0FBF4F000EB80004000009002E00098401E009000980028F9D104E0906A7F
:208D000040F020009062012300BF002082F8240000BF184661E70000002401400000002086
:208D200040420F002DE9F0410746FE480068401CFC49086008460068B0F5967F01D90020ED
:208D40000860F9480078012805D14120F74948758875C87599E0F648C07A012808D1F5482B
:208D60000078012804D10020F249087008F062FDF1480088F14909680844F0490860EE48C4
:208D80008088EF4909680844ED490860EA48408AEC4909680844EB490860EB480088401C97
:208DA000E94908800846008840F6B83188426CDBDF48C07A012822D1E0480068B0FBF1F05A
:208DC00086B23046FFF7F2FBD8494875DC48006840F6B831B0FBF1F086B23046FFF7E6FB68
:208DE000D2498875D748006840F6B831B0FBF1F086B23046FFF7DAFBCC49C8753CE0CF482B
:208E0000006840F6B831B0FBF1F086B23046FFF7BBFBC6494875CA48006840F6B831B0FBD5
:208E2000F1F086B23046FFF7AFFBC0498875C748007801280ED10846407DC5490870C148D4
:208E4000006840F6B831B0FBF1F0C24908800020BE490870BB48006840F6B831B0FBF1F0B7
:208E6000BC490988081A00EB40008001B849097801EBA020AD49C8750020B3490880AF4991
:208E80000860AF490860AF490860AB484088B2490968C1EB8020B049096801EB6020AE496A
:208EA000086008460068801244F2CE714843C0F38F209E49C8800846C0880989C91101EB83
:208EC000C10202EB011108449849C880A348007803280BD10846C088A0F5F850A43840F270
:208EE0007A514843C0F38F209049C8809C48407C01281FD101F0F8FEB0F5FA6F1AD38B482B
:208F0000C0880A2190FBF1F09549488208464069498A08449249486108468069401C8861B4
:208F20000846806943F69821884203D300208C49886148747E48C07A012815D17E48C088B1
:208F400088490988401A49F6192148438512002D01DC002006E049F61920854201DB401E31
:208F600000E02846054613E07348C0887D490988401A4CF250314843C512002D01DC002066
:208F800005E04CF25030854200DB00E02846054675480068C0EB85207349096801EB6020E5
:208FA0007149086008460068C0F38F205F4908816E48007807287DD2DFE800F0045592F701
:208FC000FEF5F4005C4800896949C98A401A642148436749097E90FBF1F004B2002C01DCAC
:208FE000002000E0204604461C2094FBF0F04F4908772546504840895E49C98A401A64215A
:2090000048435C49097E90FBF1F004B2002C01DC002000E0204604461C2094FBF0F0434987
:2090200048772544444880895349C98A401A642148435149097E90FBF1F004B2002C01DCCE
:20904000002000E0204604461C2094FBF0F0374988772544002D01DC002002E0032095FB0E
:20906000F0F0054630E1344840894249C98A401A642148433F49097E90FBF1F004B2002CCA
:2090800001DC002000E0204604461C2094FBF0F0264948772546284880893749C98A401A59
:2090A000642148433449097E90FBF1F004B2002C03DC00E006E1002000E0204604461C20BC
:2090C00094FBF0F01949887728190546002D01DC002103E0284600EBD07149100D46F3E00D
:2090E000154800892249C98A401A642148432049097E90FBF1F004B2002C01DC002000E047
:20910000204604461C2094FBF0F0084908772546094880891849C98A401A642148431649E2
:20912000097E2BE04C050020FE010020DC080020D807002074050020DC1E002060050020D2
:209140005C050020640500205805002068050020690500206A05002050050020F801002050
:2091600028030020480500205405002010040020F01500200A1600202416002090FBF1F05F
:2091800004B2002C01DC002000E0204604461C2094FBF0F06B49887728190546002D05DC68
:2091A000002107E075E05BE006E040E0284600EBD07149100D4687E0634800896349C98A31
:2091C000401A642148436149097E90FBF1F004B2002C01DC002000E0204604461C2094FB4E
:2091E000F0F0584908772546574840895849C98A401A642148435649097E90FBF1F004B2F6
:20920000002C01DC002000E0204604461C2094FBF0F04C49487728190546002D01DC0021DF
:2092200003E0284600EBD07149100D464CE0464880894849C98A401A642148434549097EDF
:2092400090FBF1F004B2002C01DC002000E0204604461C2094FBF0F03A498877254633E088
:20926000394840893A49C98A401A642148433849097E90FBF1F004B2002C01DC002000E031
:20928000204604461C2094FBF0F02E49487725461AE02D4800892D49C98A401A64214843A7
:2092A0002A49097E90FBF1F004B2002C01DC002000E0204604461C2094FBF0F02149087745
:2092C000254601E0002500BF00BF23490D8023480078D8B91C48008A21490988451A002DBD
:2092E00001DC002000E0284605461E480068C0EB85201C49096801EB20201A49086008469F
:209300000068C0F38F201449488002E00020124948800D48C08914490968C1EB8020124926
:20932000096801EB60201049086008460068C0F38F200E4908800449488809F0F7F8BDE8EE
:20934000F0810000DC080020DC1E0020F01500200A16002024160020320500208A040020BA
:20936000880400206C05002070050020FC0100207047704710B504462068406800F0200041
:2093800020282FD12068006800F00200022829D1A06A00F0100018B9A06A40F40070A062F4
:2093A0002068806800F46020B0F5602F13D1E06888B92068406820F0200021684860A06A8D
:2093C00020F48070A062A06A00F4805018B9A06A40F00100A0622046FFF7A4FC6FF012003E
:2093E000216808602068406800F0800080283BD12068006800F00400042835D1A06A00F018
:20940000100018B9A06A40F40050A0622068806800F4E040B0F5E04F0DD02068406800F482
:209420008060D0B92068806800F46020B0F5602F13D1E06888B92068406820F080002168F5
:209440004860A06A20F48050A062A06A00F4807018B9A06A40F00100A0622046FFF7D2FA50
:209460006FF00C00216808602068406800F0400040280FD12068006800F0010050B1A06AFC
:2094800040F48030A062204600F0A8F86FF001002168086010BD00002DE9F041044600271A
:2094A00000250026A84614B90120BDE8F081A06810B1606900B100BFA06A30B90020E06218
:2094C00084F82400204600F08BF82046FAF702FF0746A06A00F01000002873D1002F71D187
:2094E000A06A20F4885040F00200A062E16960680843E16840EA41000643A068B0F5807F3C
:2095000002D0A068012802D14FF4807000E0002005436069012811D1E06838B9A069401E86
:209520004FF4006141EA4030054307E0A06A40F02000A062E06A40F00100E0622068406874
:2095400020F469402843216848602068806821490840304321688860A068B0F5807F02D02E
:20956000A068012802D14FF4807000E00020B0F5807F03D1208A401E4FEA00582068C06AF1
:2095800020F4700040EA08002168C8622068806811490840B04208D10020E062A06A20F009
:2095A000020040F00100A06211E0A06A20F0020040F01000A062E06A40F00100E062012742
:2095C00005E0FFE7A06A40F01000A062012738466BE70000FDF7E1FFFE0E1FFF70470000C7
:2095E00010B586B004463249206888423CD100BF3048806940F400702E49886108468069F1
:2096000000F40070019000BF00BF3F2002900320039002A9284801F0C7F9B02002900320DF
:20962000039002A9254801F0BFF9254825490860002048600021234881608021C160490053
:20964000016189004161202181610021C16100F0DFFF20B14FF497711BA00DF0C1F800BFFD
:2096600018482062446221E01C49206888421DD100BF1048806940F480600E49886108461A
:20968000806900F48060019000BF00BF0E2002900320039002A9094801F086F901221146A2
:2096A000122001F0F0FB122001F0E0FB06B010BD00240140001002400010014000080140CA
:2096C00008000240681F00202E2E5C436F72655C5372635C6164632E630000000028014056
:2096E00070B50446002500BF94F82400012801D1022070BD012084F8240000BF2046FAF746
:2097000051FE0546002D77D1A06A40F20121884340F48070A0623C492068884208D13B48B8
:20972000006800F4702008B9012002E0002000E0012078B1A06A20F48010A062206840684F
:2097400000F4806000B3A06A20F4005040F48050A06219E0A06A40F48010A0622B49091FA9
:209760002068884203D028492068884204D12748006800F4806000E0002028B1A06A20F48A
:20978000005040F48050A062A06A00F4805020B1E06A20F00600E06201E00020E06200BF30
:2097A000002084F8240000BFC01E216808602068806800F46020B0F5602F16D11249206879
:2097C000884208D11148006800F4702008B9012002E0002000E0012038B12068806840F42F
:2097E000A000216888600CE006E02068806840F480102168886004E000BF002084F824007E
:2098000000BF284675E7000000280140042401402DE9F04104460D4616460027574920685E
:20982000884203D056492068884205D15348001D006800F4702000E0002000287ED100BFEA
:2098400094F82400012802D10220BDE8F081012084F8240000BF2046FAF7A4FD0746002F30
:209860006DD1A06A40F60161884340F48070A06243492068884209D14048001D006800F45E
:20988000702008B9012002E0002000E0012078B1A06A20F48010A0622068406800F4806076
:2098A00000B3A06A20F4005040F48050A06219E0A06A40F48010A06230492068884203D01A
:2098C0002F492068884205D12C48001D006800F4806000E0002028B1A06A20F4005040F4A0
:2098E0008050A062A06A00F4805020B1E06A20F00600E06201E00020E06200BF002084F8B7
:20990000240000BF1F48216A88621F48216AC8621E48216A08636FF0020021680860206836
:20992000806840F4807021688860226802F14C0133462A46206A00F0A3FE01E01AE014E00D
:209940002068806800F46020B0F5602F06D12068806840F4A000216888600CE02068806807
:2099600040F480102168886005E000BF002084F8240000E00127384667E700000024014015
:209980000028014027430008974300087943000830B5024600230C7D012000FA04F31068E3
:2099A000D0F8000220F47C5001254C6A45EA042420431468C4F800021068D0F81C029843F4
:2099C0001468C4F81C02C869E8B91068D0F80C0298431468C4F80C02888880B28C8940EA6F
:2099E0000444106800F510704D6940F83540088880B20C8940EA0444106800F510704D6963
:209A000000EBC5004460C86901281DD11068D0F80C0218431468C4F80C02888880B20C88E5
:209A200040EA0444106800F510704D6940F83540888980B20C8940EA0444106800F510702D
:209A40004D6900EBC5004460886938B91068D0F8040298431468C4F8040206E01068D0F895
:209A6000040218431468C4F80402086938B91068D0F8140298431468C4F8140206E0106808
:209A8000D0F8140218431468C4F81402086A012806D11068D0F81C0218431468C4F81C02BE
:209AA0001068D0F8000220F001001468C4F80002002030BD0168496941F0020102685161A1
:209AC0000168496941F0100102685161704700002DE9F0410446002500260027A8462068DD
:209AE000C068C0F3001520684069C0F3C0062DB126B148F4007810202168C8602068006991
:209B0000C0F3001520684069C0F380162DB126B148F480681020216808612068406900F0E7
:209B2000010000283BD0206880687A490840884201D1012000E0002005462068806876493F
:209B40000840884201D1012000E0002006462068806872490840884201D1012000E0002084
:209B600007460DB906B9D7B120688068C0F3400520688068C0F340262068806800F0010732
:209B80000DB906B91FB12046FBF79CFA01E048F4006820688068624908432168886020689E
:209BA000C06800F0030520684069C0F3400625B11EB100212046FBF733F82068006900F031
:209BC000030520684069C0F3001625B11EB101212046FBF725F8206C40EA0800206420687D
:209BE000806900F0010520684069C0F3002620684069C0F3C0372DB126B11FB1206C40F060
:209C00000100206420688069C0F3400520684069C0F3402620684069C0F3C0372DB126B17C
:209C20001FB1206C40F00200206420688069C0F3800520684069C0F3802620684069C0F3FB
:209C4000C0372DB126B11FB1206C40F0040020642068806900F0700008B9012000E0002091
:209C6000054620684069C0F3C02620684069C0F3C03795BB8EB387B32068806900F0700553
:209C8000402D1BD006DC102D09D0202D0CD0302D24D10EE0502D16D0602D1FD118E0206CA7
:209CA00040F0080020641AE0206C40F01000206415E0206C40F02000206410E0206C40F09D
:209CC000400020640BE0206C40F08000206406E0206C40F48070206401E007E000BF00BFB5
:209CE0002068806920F0700021688861206C78B1042021684860012084F83C0020684069ED
:209D000048F65B718843216848612046FFF7D2FEBDE8F081010000040001000800000110DB
:209D2000090501002DE9F041044600270026002514B90120BDE8F08194F83C0028B9002044
:209D400084F83D00204600F0A5F8022084F83C002068006820F0020021680860206800689A
:209D600040F001002168086000F0BEFF06460EE000F0BAFF801B0A2809D9032084F83C00A7
:209D800000BF002084F83D0000BF0320D2E72068406800F001000028EAD02068406800F06D
:209DA0000100002867D0A069012802D145F0800501E025F08005E069012802D145F040054A
:209DC00001E025F04005206A012802D145F0200501E025F02005606A012802D145F010053D
:209DE00001E025F01005A06A012802D145F0080501E025F00805E06A012802D145F0040589
:209E000001E025F004052068006820F0FC00284321680860D4E90201084321690843616941
:209E200008436168491E08432168C8612068006820F001002168086000F056FF06460EE039
:209E400000F052FF801B0A2809D9032084F83C0000BF002084F83D0000BF03206AE72068E4
:209E6000406800F001000028EAD12068406800F0010000B90127012F06D100202064012098
:209E800084F83C00002055E7042084F83C00012050E7000010B586B004462D49206888426D
:209EA00054D100BF2B48C06940F000702949C8610846C06900F00070019000BF00BF881564
:209EC000029000200390049002A9234800F06CFD4FF400700290022003900320059002A9DD
:209EE0001D4800F061FD00BF1C49486820F4C04040F0E06040F48040486000BF0122114682
:209F0000142000F0C0FF142000F0B0FF01221146152000F0B8FF152000F0A8FF104820638E
:209F2000104860631048A063FAF70EFE0F480068406940F002000D49096848610B480068E9
:209F4000406940F0100009490968486106B010BD0064004000100240000C014000000140A5
:209F6000E41F0020002000202420002044240020816B896811B9416B096941B91649096803
:209F8000496941F01001144A126851617047816B0968A1F2AA7111B1012911D100E000BF14
:209FA000816B096908290AD100210C4A1170816B09885180816B4B6953608969916000E0DB
:209FC00000BF00BF04490968496941F01001024A1268516100BFD9E744240020A40400200A
:209FE00010B50446606B806810B9606B006940B92E480068406940F002002C490968486161
:20A0000010BD606B006840F23172811A904214D009DCA0F2516080B3CF2818D0D02817D001
:20A02000DF2837D108E00F291CD010291BD01F2924D020292ED122E000BF606B00881C49E4
:20A040000880606B017C1A48FAF7AAFF23E000BF606B008817490880606B017C1548FAF7A1
:20A060009FFF18E000BF606B008813490880606B017C1148FAF794FF0DE001E000BF00BFE3
:20A08000606B00880D490880606B017C0B48FAF787FF00E000BF00BF04480068406940F092
:20A0A000020002490968486100BFA9E744240020A0050020B4050020C8050020DC050020D6
:20A0C0002DE9F04104460E46042500272068806800F08060B0F1806F0DD02068806800F03E
:20A0E0000060B0F1006F06D02068806800F08050B0F1805F7ED100BF94F83D00012802D197
:20A100000220BDE8F081012084F83D0000BF94F83C00222804D0322806D062280CD107E00A
:20A12000422084F83C000BE0522084F83C0007E0722084F83C0003E0122084F83C0000BF33
:20A1400000BF2068806800F0806008B1002507E02068806800F0006008B1012500E0022595
:20A16000206800F5C07000EB0510006800F00101206800F5C07000EB05100160206B806857
:20A1800098B9206800F5C07000EB05100068216BC968226B128841EA42510843216801F5ED
:20A1A000C07101EB0511086015E0206800F5C07000EB05100068216B8968226B526841EA0B
:20A1C000C201226BD26811430143206800F5C07000EB05100160206B007C00F00F00216BBD
:20A1E0000861206800F5C07000EB0510406820F00F0100E0B1E0206800F5C07000EB051063
:20A200004160206800F5C07000EB05104068216B09690843216801F5C07101EB05114860A5
:20A22000206BC07D0106206B807D41EA0041206B407D41EA0020216B097D0843216801F5EC
:20A24000C07101EB05118860206BC07E0106206B807E41EA0041206B407E41EA0021206BFE
:20A26000007E0143206800F5C07000EB0510C160206800F5C07000EB0510006840F0010107
:20A28000206800F5C07000EB0510016000F02CFD074620E0701CF0B126B100F025FDC01B59
:20A2A000B04218D9032084F83C001DB980202168886009E0012D03D1E8032168886003E0CF
:20A2C0004FF400002168886000BF002084F83D0000BF032015E74DB920688068214908402C
:20A2E000884201D1012016E0002014E0012D09D1206880681C490840884201D101200AE0CB
:20A30000002008E02068806818490840884201D1012000E000200028BCD094F83C00422879
:20A3200004D0522806D072280CD107E0222084F83C000BE0322084F83C0007E0622084F8C7
:20A340003C0003E0012084F83C0000BF00BF00BF002084F83D0000BFD3E6042084F83C009B
:20A360000120CEE6010000040001000800000110704710B504460CB9012010BD607920B9BE
:20A3800000202071204600F005F8012060710020F3E7000008B5094A016891420DD100BFE4
:20A3A0000749496941F04001054A51611146496901F04001009100BF00BF08BD00300240A7
:20A3C0000010024070B50446002594F82100022803D00420A063012548E02068006820F078
:20A3E0000E00216808602068006820F00100216808601F492068884201D1012026E01C4954
:20A4000014312068884201D110201FE0184928312068884201D1801518E015493C312068E6
:20A42000884201D1801411E0114950312068884202D14FF4803009E00D49643120688842E2
:20A4400002D14FF4801001E04FF08070084908394860012084F8210000BF002084F82000D3
:20A4600000BF606B10B12046616B8847284670BD0800024070B50446E06B0568206806688E
:20A4800094F84010042088402840002846D006F00400002842D02068006800F0200028B939
:20A4A0002068006820F004002168086057492068884201D1042027E0544914312068884284
:20A4C00001D1402020E0514928312068884201D1001519E04D493C312068884202D14FF4BA
:20A4E000804011E0494950312068884202D14FF4802009E0454964312068884202D14FF41C
:20A50000800001E04FF08060404908394860E06A00287AD02046E16A884776E094F84010DB
:20A52000022088402840A0B306F0020088B32068006800F0200040B92068006820F00A0040
:20A5400021680860012084F8210030492068884201D1022028E02D4914312068884201D1A6
:20A56000202021E0294928312068884201D140151AE026493C312068884202D14FF40050C8
:20A5800012E0224950312068884203D14FF400300AE017E01D4964312068884202D14FF400
:20A5A000001001E04FF0007018490839486000BF002084F8200000BFA06A30B32046A16A19
:20A5C000884722E094F84010082088402840E0B106F00800C8B12068006820F00E002168D7
:20A5E000086094F8401001208840E16B48600120A06384F8210000BF002084F8200000BF3F
:20A60000206B10B12046216B884770BD080002400146002209B901207047184B0868C01A06
:20A620001423B0FBF3F08000086414480838C863022081F821000868026843F6F0708243AE
:20A64000D1E901031843CB6818430B6918434B6918438B691843CB69184302430868026080
:20A6600000208862C862086348638863012081F82100002081F8200000BFCDE70800024074
:20A680002DE9F04104460D4616461F464FF0000800BF94F82000012802D10220BDE8F0812F
:20A6A000012084F8200000BF94F8210001282CD1022084F821000020A0632068006820F069
:20A6C0000100216808603B46324629462046FBF72FFBE06A30B12068006840F00E002168BC
:20A6E00008600BE02068006820F00400216808602068006840F00A00216808602068006807
:20A7000040F001002168086006E000BF002084F8200000BF4FF002084046BFE770B5044613
:20A7200000F0E2FA06462546681C10B104480078054400BF00F0D8FA801BA842FAD370BD44
:20A74000580000202DE9F04104460E460127002500BF2648007E012802D10220BDE8F08170
:20A7600001202249087600BF2068022813D14CF25030FDF75BF890BB0120FCF7DDFF4CF2FC
:20A780005030FDF753F807461948006920F004001749086123E04CF25030FDF747F8F0B969
:20A7A0004FF0FF303060A56812E02846FCF7D8FF4CF25030FDF73AF807460D48006920F065
:20A7C00002000B4908610FB1356007E005F58065D4E9021001EB8020A842E6D800BF00BF1E
:20A7E00000200249087600BF3846B7E730070020002002400348006940F0800001490861C5
:20A8000000207047002002402DE9FE4F05468B4617469846012600240020029000BF24481D
:20A82000007E012802D10220BDE8FE8F01202049087600BF4CF25030FCF7F8FF064686BB4E
:20A84000012D02D10120029006E0022D02D10220029001E00420029000241EE02201B946CD
:20A86000C24648465146F9F70AF980B20190022000FB04B000900199FCF786FF4CF25030C4
:20A88000FCF7D4FF06460B48006920F001000949086106B104E0601CC4B202988442DDDB79
:20A8A00000BF00BF00200249087600BF3046BBE7300700200020024000200849096901F0CD
:20A8C000800151B10649054A5160064951601146096901F0800101B101207047002002407F
:20A8E00023016745AB89EFCD10B50446042C3BD100202149C8700846807840B900F0F4F96F
:20A900001D494860601F88600120887011E000F0EBF919494968401A1749886008468068F9
:20A920004B2802D215480068886000F0DDF91249486011488068114908600F4880684B28A5
:20A9400018D30F480068401C0D4908600D48007E08B9012001E00B48007E09490968B1FB5D
:20A96000F0F00549C86005E0B4F5805F02D101200549087010BD0000E40300209C050020C5
:20A9800098050020B00A0020CC02002010B5044604480068204020B1024804602046FFF734
:20A9A000A3FF10BD140401402DE9F84703460024002000258446002700226EE14FF001081E
:20A9C00008FA02F4D1F8008008EA0400A0427DD1DFF8D0A2D1F80480A8EB0A09D0453AD0B5
:20A9E00014DCB8F1030F50D009DCB8F1000F31D0B8F1010F1CD0B8F1020F49D120E0B8F1CC
:20AA0000110F18D0B8F1120F42D11EE0B9F5881F25D006DCB9F5803F20D0B9F5801F37D175
:20AA20001AE0B9F5001F18D0B9F5041F30D117E0D1F80CC02DE0D1F80C8008F1040C28E096
:20AA4000D1F80C8008F1080C23E0D1F80C8008F10C0C1EE000BF00BF00BF00BF00BF00BFB3
:20AA6000D1F80880B8F1000F02D14FF0040C0BE0D1F80880B8F1010F03D14FF0080C1C6112
:20AA800002E04FF0080C5C6103E04FF0000C00E000BF00BFFF2801D8984601E003F1040879
:20AAA0004646FF2802D84FEA820803E0A2F108084FEA88084746D6F800804FF00F0909FAC2
:20AAC00007F928EA09080CFA07F900E088E048EA0908C6F80080D1F8048008F08058B8F1BE
:20AAE000805F7DD100BFDFF8C081D8F8188048F00108DFF8B491C9F81880C846D8F81880BE
:20AB000008F00108CDF8008000BF00BF4FEAB9384FEA920958F829504FEA82784FEA1879AD
:20AB20004FF00F0808FA09F825EA0805DFF87C81434502D14FF0000816E0DFF874814345E0
:20AB400002D14FF001080FE0DFF86881434502D14FF0020808E0DFF86081434502D14FF04D
:20AB6000030801E04FF004084FEA82794FEA197908FA09F848EA0505DFF840814FEA9209F4
:20AB800048F82950D1F8048008F48038B8F5803F0AD1DFF82C81D8F8008048EA0008DFF8CF
:20ABA0002091C9F8008009E0DFF81481D8F8008028EA0008DFF80891C9F80080D1F80480E6
:20ABC00008F40038B8F5003F10D1DFF8F48008F10408D8F8008048EA0008DFF8E49000E06F
:20ABE0005AE009F10409C9F800800DE0DFF8D08008F10408D8F8008028EA0008DFF8C09029
:20AC000009F10409C9F80080D1F8048008F48018B8F5801F0ED1DFF8A88008F10808D8F808
:20AC2000008048EA0008DFF8989009F10809C9F800800DE0DFF8888008F10808D8F80080EA
:20AC400028EA0008DFF8789009F10809C9F80080D1F8048008F40018B8F5001F0ED1DFF8CC
:20AC6000608008F10C08D8F8008048EA0008DFF8509009F10C09C9F800800DE0DFF84080D2
:20AC800008F10C08D8F8008028EA0008DFF8309009F10C09C9F80080521C102AFFF48EAE7F
:20ACA000BDE8F887000011100010024000080140000C014000100140001401400800014078
:20ACC00000040140024693680B400BB1012000E000207047C2684A40C26070470AB1016163
:20ACE00001E00B040361704701480068704700005000002070B504460CB9012070BD4CF6AD
:20AD0000CC402168086045F2555021680860D4E9001048602168A0688860FFF7E5FF054656
:20AD200006E0FFF7E1FF401B302801D90320E5E72068C0680028F4D14AF6AA202168086043
:20AD40000020DBE701464AF6AA200A681060002070470000034800680349097808440149F1
:20AD600008607047500000205800002010B50848006840F0100006490860032000F0C2F88B
:20AD8000002000F007F800F02BF8002010BD00000020024070B504460E4800784FF47A71D7
:20ADA000B1FBF0F00C490968B1FBF0F5284600F083FE08B1012070BD102C07D2002221462C
:20ADC000501E00F060F80548046001E00120F2E70020F0E75800002000000020540000202E
:20ADE00008B500BF1F48806940F001001D4988610846806900F00100009000BF00BF0320AE
:20AE000000F080F8002211466FF00B0000F03BF8002211466FF00A0000F035F8002211464C
:20AE20006FF0090000F02FF800221146501F00F02AF800221146101F00F025F8002211466B
:20AE4000901E00F020F800221146501E00F01BF800BF0549486820F0E06040F000704860FD
:20AE600000BF08BD001002400000014000BF00F01F02012191404209920002F1E022C2F86C
:20AE8000001100BF70472DE9F05F80460D461646002707F0B9F8074639462A46334601F0DC
:20AEA0000700C0F1070ABAF1040F02D94FF0040A01E0C0F1070AD14600F1040ABAF1070F69
:20AEC00002D24FF0000A01E0A0F1030AD4464FF0010A0AFA09FAAAF1010A0AEA020A0AFAC1
:20AEE0000CFA4FF0010B0BFA0CFBABF1010B0BEA030B4AEA0B042146404607F08DF8BDE8F9
:20AF0000F09F000000BF00F00702064B19684FF6FF031940044B0B4343EA0221014B1960C6
:20AF200000BF70470CED00E00000FA0500BF00BF00BF00BF00BFBFF34F8F00BF00BF00BF3B
:20AF40000948006800F4E06008490843001D0649086000BF00BF00BFBFF34F8F00BF00BF49
:20AF600000BF00BF00BFFDE70CED00E00000FA052DE9F04385B006463DA30FCB01AC0FC4D4
:20AF80003FA0006800904FF00008002500270024A146012E30D0022E58D0102E61D13948C4
:20AFA0004468006800F0807000B301A8C4F38341475C04F4803070B132484068C0F3404005
:20AFC0001DF8008004F4803040B12F48B0FBF8F000FB07F502E02D4807FB00F529484068DB
:20AFE00000F48000B0F5800F01D1A94603E068000321B0FBF1F935E02248046A04F440704F
:20B00000B0F5807F05D104F0020010B14FF400491BE004F44070B0F5007F07D11948406AC9
:20B0200000F0020010B149F640490EE004F44070B0F5407F07D11348006800F4003010B11B
:20B040004FF2244901E04FF000090BE000F0A0F90C494968C1F38131491C4900B0FBF1F9F6
:20B0600000E000BF00BF484605B0BDE8F083000002030405060708090A0B0C0D0E0F101080
:20B08000010200000010024000127A0000093D00F8B5044600260025207800F00100002896
:20B0A0006BD000274348C06900F0805070B900BF4048C06940F080503E49C8610846C069FA
:20B0C00000F08050009000BF00BF01273A48006800F48070B0B93848006840F480703649B8
:20B0E0000860FFF701FE064606E0FFF7FDFD801B642801D90320F8BD2F48006800F4807035
:20B100000028F2D02B48006A00F440752DB3A08800F44070A84220D02648006A20F4407598
:20B12000012026490860002008602248056205F0010090B1FFF7D8FD064608E0FFF7D4FDC1
:20B14000801B41F28831884201D90320D3E71948006A00F002000028F0D01648006A20F466
:20B1600040706168084313490862012F04D10846C06920F08050C86100BF207800F0020077
:20B18000022807D10B48406820F44040A168084308494860207800F01000102807D10548DC
:20B1A000406820F48000E1680843024948600020A1E700000010024000700040400442425A
:20B1C00070B504460D4600266248006800F00700A8420ED25F48006820F0070028435D497D
:20B1E00008600846006800F00700A84201D0012070BD207800F00200022807D1564840685F
:20B2000020F0F000A168084353494860207800F0010000285DD06068012806D14E480068F2
:20B2200000F4003090B90120E2E76068022806D14948006800F0007040B90120D8E746482E
:20B24000006800F0020008B90120D1E74248406820F00300616808433F494860FFF744FD3A
:20B2600006466068012810D108E0FFF73DFD801B41F28831884201D90320B9E73648406884
:20B2800000F00C000428F0D123E06068022810D108E0FFF729FD801B41F28831884201D9C0
:20B2A0000320A5E72C48406800F00C000828F0D10FE008E0FFF718FD801B41F288318842A3
:20B2C00001D9032094E72448406800F00C000028F0D12048006800F00700A8420ED91D4800
:20B2E000006820F0070028431A4908600846006800F00700A84201D0012079E7207800F028
:20B300000400042807D11448406820F4E060E168084311494860207800F00800082808D19E
:20B320000D48406820F46050216940EAC1000A49486000F03DF808494968C1F30311074A9C
:20B34000515CC840064908600020FFF723FD00204EE7000000200240001002404072010887
:20B360000000002001480068704700000000002000B5FFF7F7FF04494968C1F30221034A62
:20B38000515CC84000BD0000001002405072010800B5FFF7E7FF04494968C1F3C221034AAB
:20B3A000515CC84000BD00000010024050720108F0B585B00FF26C0C9CE8E01001A8A0E806
:20B3C000E0101CA52D68009500210022002300240020194D696801F00C05F5B1042D02D006
:20B3E000082D19D101E0154819E001ADC1F38346AC5D01F4803555B10F4D6D68C5F34045A5
:20B400001DF805200D4D6543B5FBF2F302E00C4D04FB05F3184602E000BF084800BF00BF5C
:20B4200005B0F0BD02030405060708090A0B0C0D0E0F1010010200000010024000127A0032
:20B4400000093D00F8B504460025207800F00100002878D0F848406800F00C0004280CD0A5
:20B46000F548406800F00C00082811D1F248406800F48030B0F5803F0AD1EF48006800F481
:20B48000003000285FD0606800285CD10120F8BD00BF6068B0F5803F06D1E748006840F4A5
:20B4A0008030E549086028E0606858B9E248006820F48030E04908600846006820F4802014
:20B4C00008601AE06068B0F5A02F0BD1DA48006840F48020D84908600846006840F4803071
:20B4E00008600AE0D448006820F48030D24908600846006820F48020086000BF606888B19D
:20B50000FFF7F2FB054606E0FFF7EEFB401B642801D90320BBE7C848006800F400300028EE
:20B52000F2D010E0FFF7E0FB054606E0FFF7DCFB401B642801D90320A9E7BF48006800F4B3
:20B5400000300028F2D1207800F00200022857D1B948406800F00C0050B1B748406800F0B7
:20B560000C00082818D1B448406800F4803098B9B148006800F0020020B12069012801D066
:20B58000012084E7AC48006820F0F800616940EAC100A949086033E02069E8B10120A74966
:20B5A0000860FFF7A1FB054606E0FFF79DFB401B022801D903206AE79F48006800F00200BE
:20B5C0000028F2D09C48006820F0F800616940EAC1009949086013E0002098490860FFF7DC
:20B5E00083FB054606E0FFF77FFB401B022801D903204CE79048006800F002000028F2D15A
:20B60000207800F0080008282DD1A069B8B101208B490860FFF768FB054606E0FFF764FBBE
:20B62000401B022801D9032031E78348406A00F002000028F2D0012007F066F813E0002096
:20B640007F490860FFF750FB054606E0FFF74CFB401B022801D9032019E77748406A00F030
:20B6600002000028F2D1207800F00400042873D100267148C06900F0805070B900BF6E487B
:20B68000C06940F080506C49C8610846C06900F08050009000BF00BF01266A48006800F429
:20B6A0008070B0B96748006840F4807065490860FFF71AFB054606E0FFF716FB401B6428B6
:20B6C00001D90320E3E65F48006800F480700028F2D000BFE068012806D15748006A40F087
:20B6E00001005549086227E0E06858B95248006A20F00100504908620846006A20F00400FD
:20B70000086219E0E06805280BD14B48006A40F00400494908620846006A40F001000862F5
:20B720000AE04548006A20F00100434908620846006A20F00400086200BFE068A0B1FFF79D
:20B74000D3FA054609E0FFF7CFFA401B41F28831884202D903209AE622E03748006A00F0BF
:20B7600002000028EFD012E0FFF7BEFA054608E0FFF7BAFA401B41F28831884201D9032055
:20B7800085E62D48006A00F002000028F0D1012E05D12948C06920F080502749C86100BFAD
:20B7A000E069C8B32448406800F00C00082860D0E069022848D1002020490866FFF794FA4E
:20B7C000054606E0FFF790FA401B022801D903205DE61948006800F000700028F2D1206A55
:20B7E000B0F5803F07D11448406820F40030A168084311494860D4E9080108430E49496856
:20B8000021F4741108430C49486001200B490866FFF76AFA054607E02DE0FFF765FA401B1A
:20B82000022801D9032032E60348006800F000700028F2D01FE000000010024000004242F7
:20B84000800442420070004000200C490866FFF74BFA054606E0FFF747FA401B022801D94B
:20B86000032014E60648006800F000700028F2D101E001200BE6002009E600000000424224
:20B8800000100240042808D14FF0E021096941F004014FF0E022116107E04FF0E02109691D
:20B8A00021F004014FF0E022116170470EB563480078012800D10EBD6148407E08B9022013
:20B8C00001E05F48407E02465D48418801235D48F9F7C6FC5C48007830B95C4A11885C4A07
:20B8E00010885C4A03F04EFD5B485C490978CDE900105B480278564800680290594803786C
:20B9000051480078029903F06FFA53480078C0435549087050488079C04388714E48B0F927
:20B920000200C04348804C48B0F90400C04388804E480078D0B94E48027E4E480189454B91
:20B940004B48163009F03CFC4B48027E49484189404B4948163009F095FC4848027E4548E6
:20B9600081893C4B4548163009F0EEFC4448007828B94048018A374A4248FCF7F5F9424911
:20B980004248F8F751FD424805F0F4FD41480088401C4049088008460088052801DB0020F3
:20B9A00008803D480088401C3B490880084600880A2809DB00200880244B1A88997A5B88EF
:20B9C00098B2364BF9F750F835480088401C3449088008460088322804DB002008803148CE
:20B9E000F9F758FD30480088401C2F49088008460088642809DB00200880124908780A22B1
:20BA00002A4906F0E5FA1149887229480088401C2749088008460088C82801DB00200880F3
:20BA200024480088401C2349088008460088B0F57A7F01DB0020088000BF3CE75C0000206C
:20BA4000B00A0020B4030020D8000020DC080020320500208C010020DE00002051040020C2
:20BA6000DA00002050040020E600002014040020F0150020DC1E00200A1600202416002041
:20BA80008A040020880400202A050020F21E0020D00B00205E0000206000002004020020AE
:20BAA00062000020CC0100206400002064150020660000206800002070B504462546681E8C
:20BAC000B0F1807F01D301200FE0681E4FF0E02148610F214FF0FF3006F09EFA00204FF0E8
:20BAE000E021886107200861002070BD10B5FFF7DDFE10BD7047704710B50346002200BFBF
:20BB000093F83C00012801D1022010BD012083F83C0000BF22F0FF00CC6840EA040222F452
:20BB200040708C6840EA040222F480604C6840EA040222F400600C6840EA040222F4805057
:20BB40000C6940EA040222F400504C6940EA040222F480408C6940EA040222F400408C69AF
:20BB600040EA04021868426400BF002083F83C0000BF00BFC9E7024600BF92F83C000128B5
:20BB800001D102207047012082F83C0000BF022082F83D001068406820F0700013685860B8
:20BBA000106840680B681843136858601068806820F0800013689860106880684B68184393
:20BBC00013689860012082F83D0000BF002082F83C0000BF00BFD5E770B504460D46042263
:20BBE0002946206809F056F82068406C40F40040216848642068006840F001002168086018
:20BC0000002070BD70B504460D4600222946206809F040F800BF2068006A41F2111108407D
:20BC200050B92068006A8910084028B92068406C20F400402168486400BF00BF2068006A1A
:20BC400041F21111084050B92068006A8910084028B92068006820F001002168086000BFD9
:20BC6000002070BD10B504460CB9012010BD94F83D0028B9002084F83C00204600F00CF8D9
:20BC8000022084F83D00211D206808F0BBFF012084F83D000020E9E710B586B004463249C7
:20BCA0002068884233D100BF3048806940F400602E4988610846806900F40060019000BF3F
:20BCC00000BF8814029000200390049002A92848FEF76AFE4FF460400290022003900590F9
:20BCE00002A92348FEF760FE4FF47060029002200390059002A91F48FEF756FE0122114617
:20BD00001920FFF7C0F81920FFF7B0F829E02068B0F1804F25D100BF1448C06940F00100F9
:20BD20001249C8610846C06900F00100019000BF00BF00BF0846806940F0040088610846A7
:20BD4000806900F00400019000BF00BF012002900020039004900220059002A90548FEF759
:20BD600023FE06B010BD0000002C014000100240000C0140000801400146022081F83D00AB
:20BD80000868006840F001000A681060012081F83D000020704701460868C06840F00100FA
:20BDA0000A68D0600868006840F001000A681060002070472DE9F04104460D46002600BF56
:20BDC00094F83C00012802D10220BDE8F081012084F83C0000BF022084F83D00206886687E
:20BDE00026F0770626F47F4620688660286850283BD00CDC202860D004DC002853D010288D
:20BE000065D155E030285DD0402860D141E0602835D070280DD0B0F5805F03D0B0F5005F1B
:20BE200055D115E02068806820F00700216888604EE0D5E902136A68206808F039FF2068DC
:20BE4000866826F0770646F07706206886603FE0D5E902136A68206808F02AFF2068806863
:20BE600040F480402168886032E0EA686968206808F0FCFF5021206808F026FF28E0EA683D
:20BE80006968206809F007F86021206808F01CFF1EE0EA686968206808F0E8FF40212068C4
:20BEA00008F012FF14E00021206808F00DFF0FE01021206808F008FF0AE02021206808F086
:20BEC00003FF05E03021206808F0FEFE00E000BF00BF012084F83D0000BF002084F83C00DF
:20BEE00000BF00BF71E7704710B5044620680069C0F34000D8B12068C068C0F34000B0B135
:20BF00006FF0020021680861012020772068806900F0030018B12046FFF7E5FF05E020465E
:20BF200000F0D6F8204600F0ABF90020207720680069C0F38000D8B12068C068C0F3800002
:20BF4000B0B16FF0040021680861022020772068806900F4407018B12046FFF7C4FF05E090
:20BF6000204600F0B5F8204600F08AF90020207720680069C0F3C000D8B12068C068C0F3DE
:20BF8000C000B0B16FF0080021680861042020772068C06900F0030018B12046FFF7A3FF01
:20BFA00005E0204600F094F8204600F069F90020207720680069C0F30010D8B12068C0685E
:20BFC000C0F30010B0B16FF0100021680861082020772068C06900F4407018B12046FFF7A3
:20BFE00082FF05E0204600F073F8204600F048F9002020772068006900F0010058B1206859
:20C00000C06800F0010030B16FF0010021680861204600F095F920680069C0F3C01058B173
:20C020002068C068C0F3C01030B16FF08000216808612046FFF75EFD20680069C0F3801030
:20C0400058B12068C068C0F3801030B16FF0400021680861204600F077FA20680069C0F307
:20C06000401058B12068C068C0F3401030B16FF02000216808612046FFF73DFD10BD0000FF
:20C080001FB504460E492068884218D140200090022001900320039069460A48FEF784FC21
:20C0A00000BF0949486820F4406040F0E06040F44060486000BF0021044800F00BF81FBD24
:20C0C0000004004000100140000001409C1E00207047000030B504460D460122294620685D
:20C0E00008F0CAFD0A492068884201D1012000E0002028B12068406C40F400402168486433
:20C100002068006840F0010021680860002030BD002C014070B504460D46164600BF94F82A
:20C120003C00012801D1022070BD012084F83C0000BF022084F83D0036B1042E1BD0082ECC
:20C1400031D00C2E5ED145E02946206808F0C6FD2068806940F00800216888612068806912
:20C1600020F004002168886120688069296908432168886147E02946206808F0E1FD2068FD
:20C18000806940F40060216888612068806920F480602168886120688069296940EA01208B
:20C1A000216888612FE02946206808F001FE2068C06940F008002168C8612068C06920F0B4
:20C1C00004002168C8612068C069296908432168C86118E02946206808F020FE2068C069B3
:20C1E00040F400602168C8612068C06920F480602168C8612068C069296940EA012021688B
:20C20000C86100E000BF00BF012084F83D0000BF002084F83C0000BF00BF85E710B504462D
:20C220000CB9012010BD94F83D0028B9002084F83C00204600F00CF8022084F83D00211D56
:20C24000206808F0DFFC012084F83D000020E9E708B5094A016891420DD100BF0749C9694E
:20C2600041F00201054AD1611146C96901F00201009100BF00BF08BD000400400010024022
:20C280007047000030B504460D4601222946206808F0F2FC0A492068884201D1012000E0ED
:20C2A000002028B12068406C40F40040216848642068006840F0010021680860002030BD89
:20C2C000002C014030B504460D4600222946206808F0D2FC19492068884201D1012000E009
:20C2E000002090B100BF2068006A41F21111084050B92068006A8910084028B92068406C9E
:20C3000020F400402168486400BF00BF2068006A41F21111084050B92068006A89100840AB
:20C3200028B92068006820F001002168086000BF012084F83D00002030BD0000002C014017
:20C3400038B5044670480088401C6F49088008460088B0F5967F01DB002008806B4840784B
:20C360006B4B0090DA79997958796A4B1B7800F05BFE69480078401C67490870084600783D
:20C3800005280ADB65480068806840F0010063490968886000206049087061480068401CAA
:20C3A0005F49086000F04CFA5D48C08842F6FF7188420CDA5A480089594989880844584927
:20C3C00008810846C088898808445549C880544A917A108905F098FD524948805249534896
:20C3E00004F0F0FA52480078524909784840FF281AD14F4880794F4989794840FF2813D1DA
:20C400004B4880884B498988484080B24FF6FF71884209D14648408846494988484080B259
:20C420004FF6FF7188420AD0FEF75EFC42490968401AC82807D902204049087003E0FEF733
:20C4400053FC3D4908603D480078012802D0022856D151E03648807901284CD13848007870
:20C46000012804D1FBF7A0F800203549087030480078012811D0022804D003280ED00428F1
:20C4800037D116E0264B1A89264BB3F90210284BB3F90200FBF740FA2CE000BF204B1A8935
:20C4A000204BB3F90210224BB3F90400FBF734FA20E02448007800F0010050B9184B1A8932
:20C4C000184BB3F902101A4BB3F90400FBF724FA0EE01C48007800F0010048B1104B1A8964
:20C4E000104BB3F90210124BB3F90200FBF714FA00E000BF00BF04E001201149087000E003
:20C5000000BF00BF38BD000020050020DA000020D00A00205004002018050020081F002077
:20C52000D8070020DC0800208C010020CC020020DE000020E60000201C05002030000020C8
:20C5400019050020B9010020704770472DE9F0470446206805682068C668206847694FF09C
:20C560000008C14605F00F08B8F1000F0AD105F0200038B106F0200020B1204609F030F9A0
:20C58000BDE8F087B8F1000F6DD007F0010018B906F49070002866D005F0010030B106F498
:20C5A000807018B1E06B40F00100E06305F0040030B107F0010018B1E06B40F00200E063A8
:20C5C00005F0020030B107F0010018B1E06B40F00400E06305F0080030B107F0010018B161
:20C5E000E06B40F00800E063E06B68B305F0200028B106F0200010B1204609F0F1F820687A
:20C600004069C0F38019E06B00F0080010B9B9F1000F22D0204609F074F82068406900F082
:20C620004000B0B12068406920F0400021684861606B50B11748616B4863606BFDF7C2FE85
:20C6400010B1606B416B88470CE02046FFF77DFF08E02046FFF779FF04E02046FFF775FF9F
:20C660000020E0638CE705F0800030B106F0800018B1204609F0FAF982E705F0400030B17E
:20C6800006F0400018B1204609F04BF878E700BF76E70000B155010810B504460CB901207A
:20C6A00010BDA06900B100E000BF94F8390028B9002084F83800204600F028F8242084F8A4
:20C6C00039002068C06820F400502168C860204609F0E8F82068006920F490402168086156
:20C6E0002068406920F02A00216848612068C06840F400502168C8600020E063202084F899
:20C70000390084F83A000020CAE7000010B586B004462B49206888424FD100BF2948C069D5
:20C7200040F480202749C8610846C06900F48020019000BF00BF08150290022003900120ED
:20C7400004900320059002A91F48FEF72DF94FF400600290002003900120049002A91A48B6
:20C76000FEF722F900BF1949486820F0300040F0E06040F01000486000BF012211462720C0
:20C78000FEF781FB2720FEF771FB11480068C06840F480700E490968C8600D48006840691D
:20C7A00040F001000A490968486109480068C06840F0200006490968C86006B010BD00003F
:20C7C00000480040001002400010014000000140882600207047704710B500F011F90549A4
:20C7E00031F8100041F255510844034908810020086010BDEE7E0108D807002000B585B053
:20C8000000BF0D48806940F010000B4988610846806900F01000009000BF00BF4FF4607046
:20C820000190002002900120039001A90348FEF7BBF805B000BD000000100240001001404F
:20C84000F8B500F0DDF8064600F0DAF8044600F0D7F80546A64203D1AC4201D15E4805706D
:20C860005E48007830B95C4800785B49487001205A4908705848007857494978884210D0DA
:20C88000FEF732FA564908605648007828B155480078401C5349087017E00120524988724F
:20C8A00013E0FEF721FA4E490968401AC8280CD900204D4988724B4908704B498881C8819C
:20C8C0004A4908700120484908744748807A10B9002047490870404800783F494978454ACD
:20C8E000515C884245D14048006840B13E48006842F6AA21B1FBF0F03B49888002E00120BE
:20C90000394988803A480078401C394908700846007802280DDD3448006844F63E11B1FB4A
:20C92000F0F03149888100203049087001202E4908742F4800780F280CDA274800782E4905
:20C9400031F8100041F255510844274908810020888009E00F20264908701F48007826490B
:20C9600031F810002049088100201F490860C88026E019484078184909781E4A515C884274
:20C980001ED100201A4908701749888012480078194931F8100041F25551084412490881CF
:20C9A0004FF6FF70086011480078401CC0B20F490870052804DD0620087000200A49087451
:20C9C000054800680D49009003F092F80248007801494870F8BD0000980300209A0300204E
:20C9E0009C0300209B030020D8070020A0030020A1030020DE7E0108EE7E01088C010020AD
:20CA000010B51E48C07AA8B94FF400711C48FEF759F904464FF480711948FEF753F944EAA3
:20CA20004000C4B280211648FEF74CF944EA8000C4B220E04FF400711148FEF743F908B9E4
:20CA4000012000E0002004464FF480710C48FEF739F908B9012000E0002044EA4000C4B2F6
:20CA600080210748FEF72EF908B9012000E0002044EA8000C4B204F0070010BDD8070020DD
:20CA80000010014007E0044803F0D1FE002005F02BFDFAF7B9FAF6E70001002070B5044602
:20CAA000204609F05CFFA1890122A068FEF716F90120FAF74EFAA1882068FEF703F905461C
:20CAC000A1890022A068FEF709F90120FAF741FA012D01D1012070BD0020FCE71FB504464F
:20CAE000A06809F0B9FE206809F0B6FEA089009001200390112001906946A068FDF754FF1C
:20CB0000A0880090012003901120019069462068FDF74AFF1FBD2DE9F04704460F464FF06C
:20CB200000084FF08009204609F019FF00251CE0A1890122A068FEF7D1F83220FAF709FA34
:20CB4000A1882068FEF7BEF80646012E03D149FA05F040EA0808A1890022A068FEF7BEF8B9
:20CB60003220FAF7F6F9681CC5B2082DE0DB87F800800120FAF7EDF9BDE8F08710B5044676
:20CB8000204609F0F4FEA18801222068FEF7A6F80120FAF7DEF9A1890122A068FEF79EF814
:20CBA0003220FAF7D6F9A1890022A068FEF796F8A18800222068FEF791F80120FAF7C9F967
:20CBC00010BD10B50446204609F0D1FEA1890122A068FEF783F8A18801222068FEF77EF847
:20CBE0003220FAF7B6F9A18800222068FEF776F83220FAF7AEF9A1890022A068FEF76EF874
:20CC000010BD10B50446204609F0B1FEA18800222068FEF763F8A1890122A068FEF75EF867
:20CC20003220FAF796F9A18801222068FEF756F83220FAF78EF9A18800222068FEF74EF833
:20CC4000A1890022A068FEF749F810BD2DE9F04104460D46A8468026204609F088FE0027F9
:20CC600036E006EA0800C0B1A18801222068FEF735F83220FAF76DF9A1890122A068FEF74C
:20CC80002DF83220FAF765F9A1890022A068FEF725F83120FAF75DF917E0A1880022206806
:20CCA000FEF71CF83220FAF754F9A1890122A068FEF714F83220FAF74CF9A1890022A068A9
:20CCC000FEF70CF83120FAF744F97610781CC7B2082FC6DBA18801222068FDF7FFFF01208A
:20CCE000FAF737F9BDE8F08101480249086070470030000808ED00E00120294909780529FB
:20CD000010D12749103109789B290BD1244914310978522906D1224918310978052901D1A6
:20CD200003203BE01E49097804291BD11C4910310978C32916D11A4914310978B42911D1D2
:20CD40001749183109780B290CD116490988802901D1022022E013490988B1F5807F1DD189
:20CD600005201BE00E49097881B90D491031097810290BD10A4914310978042906D10849E6
:20CD8000183109780A2901D1012007E006490968064A914201D1042000E00020704700002C
:20CDA000D0FF0FE0E0F7FF1F002004E01004031300B585B000BF2B48806940F010002949DB
:20CDC00088610846806900F01000009000BF00BF254826490860401488800846808801909E
:20CDE0000020029001200390086801A9FDF7DCFD00201E4988714872C860C87108721A486F
:20CE00001B4908604FF4804088800846808801900020029001200390086801A9FDF7C4FD1F
:20CE20000020134988714872C860C87108720E48104908604FF4004088800846808801905F
:20CE40000020029001200390086801A9FDF7ACFD0020084988714872C860C871087205B001
:20CE600000BD000000100240001001407C1D0020901D0020A41D00202DE9F04104460F4605
:20CE800016469846069DB8F1000F04D10121204609F046FD03E00221204609F041FDE07968
:20CEA00000F0010020B101206072FDF71DFFE060607A01281BD1207A50B9FDF715FFE06093
:20CEC000FDF712FF206100206072012028700EE0FDF70AFFE168401AB84208D9FDF704FFC1
:20CEE000E060002060722870FDF7FEFE2061287868B966B1FDF7F8FE2169401AB04206D980
:20CF0000FDF7F2FE20610020607201202870BDE8F0812DE9F04105460E4617469846B8F121
:20CF2000F10F13D100240EE0BC4201D1012300E000231A4605EBC403998855F83400FDF757
:20CF4000CDFE601CC4B2B442EEDB0DE0002409E005EBC402918855F834000022FDF7BEFE39
:20CF6000601CC4B2B442F3DBBDE8F08110B586B000BF2A48806940F00400284988610846F4
:20CF8000806900F00400019000BF00BF00BF0846806940F0080088610846806900F008005F
:20CFA000019000BF00BF002433E01D4A02EBC40291881B4A52F834000022FDF78FFE184812
:20CFC00000EBC400808802900120039002200590134951F8340002A9FDF7E6FC114A02EBFB
:20CFE000C40291880F4A52F834000022FDF776FE0C4800EBC400808802900120039002207E
:20D000000590084951F8340002A9FDF7CDFC601CC4B2032CC9DB06B010BD000000100240AB
:20D02000540400206C0400202DE9F0470746894692461C46DDF82080FDF756FEB0F5FA6F7A
:20D040000DD2F0232A4603219848FFF762FFF023324603219648FFF75CFFBDE8F087B9F16F
:20D06000060F06D0B9F10C0F05D0B9F1FF0F06D103E0002505E0012503E0022501E0002579
:20D0800000BF00BFBAF1060F06D0BAF10C0F05D0BAF1FF0F06D103E0002605E0012603E059
:20D0A000022601E0022600BF00BF07F0F000102802D0202807D107E0F1232A4603217B485E
:20D0C000FFF727FF07E000BF43462A4603217748FFF71FFF00BF00BF07F00F00072843D2D6
:20D0E000DFE800F04204436F7AA6AD004CB9F123324603216E48FFF70CFF00206D490880EA
:20D1000031E0B8F1F10F22D16B48408969490988884206DDF123324603216548FFF7F9FEAC
:20D120000FE06548808963490988884206DDF023324603215E48FFF7ECFE02E000205D4983
:20D1400008805C480088401C5A4908800BE0B8F1F00F08D1F023324603215548FFF7D9FE0F
:20D160000020544908809DE000BF04BB51480088B0F5167F06DAF123324603214C48FFF7FA
:20D18000C8FE0EE04B480088B0F5966F06DAF023324603214648FFF7BCFE02E000204549B9
:20D1A000088044480088401C4249088008E04346324603213E48FFF7ACFE00203D49088003
:20D1C00070E00CB9F12000E0F0200346324603213748FFF79EFE65E004BB36480088B0F594
:20D1E000167F06DAF123324603213148FFF791FE0EE030480088B0F5966F06DAF023324609
:20D2000003212B48FFF785FE02E000202949088028480088401C2749088008E0F023324643
:20D2200003212348FFF775FE00202249088039E0F123324603211E48FFF76BFE32E01F48DC
:20D2400000881D490989884222DB1B48408919490988884206DDF123324603211448FFF7B9
:20D2600058FE0FE01448808912490988884206DDF023324603210E48FFF74BFE02E0002025
:20D280000C4908800B480088401C0A49088008E0002008490880F023324603210448FFF7CD
:20D2A00038FE00BF00BF00BFD7E60000540400206C04002084040020D00A0020E40300208D
:20D2C0007CB504460D46094903C9CDE90001084803F0A0FA01208DF8060003208DF800007A
:20D2E00000982060019860607CBD000060780108000100202DE9FF4F85B0804691461D46E9
:20D300004FF0000AFE4903C9CDE90301FD48008800B2FD490880FD48B0F9020064286DDDE4
:20D320000846B0F90000002868DDF848B0F9020064214843F449B1F90010B0FBF1F000B259
:20D34000F34908800846B0F90040F2480068C0EB0420F049096801EBA010EE49086008462E
:20D360000068001200B2EC490880E748B0F90000EA49B1F90010401A052811DDE348B0F9B6
:20D380000200E749B1F90010401A002804DDE048B0F90000E3490880DC484088E04908801C
:20D3A000D948B0F90000DD490880DF48007820BBDE48B0F90400192829DDDD480088401C58
:20D3C000DB49088008460088282820DB00200880D1480088D749D84A128821F81200D64812
:20D3E0000088401CD44908800846008832280EDB002008800120CC49087008E0C248B0F99A
:20D400000000C6490880C1484088C5490880CB48408800B2CA490880A9F16404B4F5006FCC
:20D4200002DD4FF4006000E02046044604FB04F0C11700EB5151CC12C24800780521B1EB60
:20D44000D00F17DBB14AD17BBF4A1279012383EAD21003F0B1F9BC490979BC4A92F91020C8
:20D460001144B84A127801EBD2010A314843C0F3872A16E0A54AD17BB34A1279012383EA98
:20D48000D21003F099F9B0490979B04A92F910201144AC4A127801EBD20115394843C0F3D5
:20D4A000872A0AF10100604332214843A849C98990FBF1F000B2A74908800AEB8A001621AF
:20D4C00001EB40009049B1F90010884202DA0020A04908809B480078C0F3800038B18A480D
:20D4E000B0F900003C2802DC00209A4908809948B0F90000002803DD9648B0F9000000E0BD
:20D500000020944908800846B0F900008C49B1F90010884203DA8F48B0F9000002E0884827
:20D52000B0F900008B4908809DF81800C0F34000B0B305F00F00012806D002280FD00328AC
:20D5400018D004282DD120E04FF4FA6201217C48B0F9000007F0B2FA7F4908602CE040F27A
:20D56000DC5201217648B0F9000007F0A7FA7A49086021E04FF47A7201217148B0F900007D
:20D5800007F09CFA7449086016E04FF4FA7201216B48B0F9000007F091FA6F4908600BE029
:20D5A0000BE04FF47A7201216548B0F9000007F085FA6949086000BF09E04FF4FA720121D0
:20D5C0005F48B0F9000007F079FA634908604FF47A7201215A48B0F9000007F06FFA5F49D9
:20D5E00008605248807968B94848B0F90200642808DD464840885A49088008460088000408
:20D60000584908609DF81800C0F34000F0B305F00F00012806D0022814D0032824D0042862
:20D6200042D134E04B49B1F9001001EBC10108114C4B4A490A684849096809F0B5F94849D8
:20D6400008803EE04349B1F9001001EB410202EBC1010811434B41490A683F49096809F06B
:20D66000A3F93F4908802CE03A49B1F9001001EB810202EBC10108113A4B38490A68364987
:20D68000096809F091F9364908801AE01AE0354B32480268304801682E48B0F9000009F03E
:20D6A00083F92F4908800CE02E4B2C4802682A4801682848B0F9000009F076F92849088056
:20D6C00000BF0BE0274B25480268234801682148B0F9000009F068F9214908806FF0C700FF
:20D6E0002149086140F6340048612048C08901B21D4A1B48B0F9000004F0B0FD1C4939E04E
:20D7000048780108E403002026010020DC0800202C010020080100202E0100202A010020DE
:20D72000280100200C01002010010020DE00002012010020140800200E010020F00A00208C
:20D7400030010020B9010020B00A0020D00A002004020020320100203401002038010020A3
:20D760003C01002020010020E4060020D80700204601002008806FF063005849086140F215
:20D780001A404861564AD17B564A127A012383EAD21002F0E3FF5349097A4FF47A72514345
:20D7A0004843401400904E480089C1114E4A009804F054FD4D4908804D4A117B484AD08869
:20D7C0004C4A128801F0F4FB07464A48078001231A4649480188384601F042FD4649088070
:20D7E000404A517A3E4A907D01F0D0FB83463D4A527A0F3A91B23A4A507D01F0C7FB019046
:20D8000001980BFB00F0810A0291029988B201231A463A49098801F023FD38490880384854
:20D82000B0F900003449098848438612334800887043861233480078B0B933480068301A37
:20D84000022805DD30480068801C2F49086018E02D480068301A10F1030F12DA2A48006868
:20D86000C01E294908600CE027480068132805DD2548006810382449086002E000202149B2
:20D8800008702148006810F1C80F03DA6FF0C7001D4908601D48008818B91D4802F0C7FFBB
:20D8A00002E01B4802F0B6FF174800680F49B1F900100844401000B2ADF8100001208DF8FA
:20D8C000120004208DF80C000398C8F800000498C8F8040009B0BDE8F08F0000E4060020DF
:20D8E000DC080020B00A0020C006002048010020F00A00204A0100204C0100204E0100209A
:20D900004601002044010020400100203C010020000100202DE9FF4F87B0824616461F4638
:20D92000FE4903C9CDE90501002004900390BE4203DA07FB07F0C01202E006FB06F0C0127E
:20D94000F749488008464088B0F5006F02DD4FF4006001E0F2484088F14948809DF8200079
:20D96000C0F3400000287CD0149803287AD004DC012807D0022876D149E0042874D03328DA
:20D98000F9D1D7E0E748007A002801DC012001E0E448007A0490E348407A0390E0484088B4
:20D9A000E049C9884843C00A04B2DE48C088A04202DADC48C08800E0204604B2D948408964
:20D9C000D949097A48434FF47A714843401400EBC00101EB00104FF6FF7101EA8005012319
:20D9E0000522D2480188284601F03AFCCF490880CC48C0884042CE49086100204861C948F0
:20DA0000C0888002404288610020C861DFE0C548007D002801DC012001E0C248007D04901D
:20DA2000C048407D0390BE484088BE49498A4843C00A04B2BB48408AA04202DAB948408A85
:20DA400000E0204604B2B748C08AB749097A48434FF47A714843401400EBC00101EB0010BE
:20DA600003E0B5E01DE0ADE063E04FF6FF7101EA800501230522AD480188284601F0F0FB29
:20DA8000AA490880A748408A4042A949086100204861A448408A8002404288610020C861C0
:20DAA00095E0A04890F82000002801DC012002E09C4890F8200004909A4890F8210003901B
:20DAC000974840889749C98B4843C00A04B29548C08BA04202DA9348C08B00E0204604B258
:20DAE0009048408C9049097A48434FF47A714843401400EBC00101EB00104FF6FF7101EA46
:20DB000080050123052289480188284601F0A8FB864908808348C08B404285490861002093
:20DB200048618048C08B8002404288610020C8614DE000BF7B4890F82C00002801DC01206A
:20DB400002E0784890F82C000490764890F82D000390734840887349498D4843C00A04B2B5
:20DB60007048408DA04202DA6E48408D00E0204604B26C48C08D6C49097A48434FF47A71F1
:20DB80004843401400EBC00101EB00104FF6FF7101EA80050123052264480188284601F0FA
:20DBA0005FFB624908805F48408D404260490861002048615B48408D80024042886100208A
:20DBC000C86104E0002004900390002400BF4DE09DF82000C0F34000F0BB524890F8380034
:20DBE000002801DC012002E04E4890F8380004904C4890F82D000390494840884949498D96
:20DC00004843C00A04B24748408DA04202DA4548408D00E0204604B24248C08D4249097AA4
:20DC200048434FF47A714843401400EBC00101EB00104FF6FF7101EA8005012305223B48B1
:20DC40000188284601F00CFB384908803548408D40423749086100E008E00020486131480D
:20DC6000408D8002404288610020C861314890F90E00322805DC2F4890F90E0010F1320F06
:20DC800002DA00202B4988732A4890F90F00322805DC284890F90F0010F1320F02DA00208E
:20DCA0002449C873244800780521B1EBD00F63DB224AD17B1C4A1279012383EAD21002F0EB
:20DCC0007BFD194909791B4A92F9102011449DF8202001EBD201083101EB8101154A92F94E
:20DCE0000E2002EB41014843C0F38F2014490880124AD17B0C4A1279012383EAD21002F007
:20DD00005BFD094909790B4A92F9102011449DF8202001EBD2010A3114E0000050780108DE
:20DD2000F0000020E40B0020B00A00205201002008070020D00A0020B9010020DC08002070
:20DD40005601002001EB8101BA4A92F90F2002EB410116314843C0F38F20B74908800846E7
:20DD60000088B6490988401AC01E4FF4806191FBF0F0B34908804CE0B24AD17BB24A127944
:20DD8000012383EAD21002F017FDAF490979A94A92F9102011449DF8202001EBD2011739A9
:20DDA00001EB8101A34A92F90E2002EB41014843C0F38F20A1490880A24AD17BA24A127912
:20DDC000012383EAD21002F0F7FC9F490979994A92F9102011449DF8202001EBD2011539AC
:20DDE00001EB8101934A92F90F2002EB410116314843C0F38F2090490880084600888F49AC
:20DE00000988401AC01E4FF4806191FBF0F08C4908808E480078C0F3800078B98C4800883E
:20DE200000908748008803B28448028800210846F9F7F4FE6043800A04B20EE0844800887A
:20DE400000907F48008803B27C480288FF213C20F9F7E4FE6043800A04B27E488480B0F93C
:20DE60000400002802DC00207A4988807848008872490988884220DD7648B0F90400754929
:20DE8000B1F90610401A022806DD7248C088401C00B27049C88033E06E48B0F904006D491E
:20DEA000B1F90610401AB0F1FF3F29DA6948C088401E00B26749C88022E000BF6548B0F94E
:20DEC00004006449B1F90610401A022807DD6148C1880498084400B25E49C88010E05D4859
:20DEE000B0F904005B49B1F90610401AB0F1FF3F06DA5848C1880398081A00B25549C880BA
:20DF00005448B0F90600062801DA062002E05148B0F906004F49C8804D4800884649098840
:20DF2000884208DD01204B4908700020C8804A4802F07DFC02E0484802F06CFC474A117BB7
:20DF4000404AD088464A128801F032F881464448A0F8009001231A4642480188484601F009
:20DF60007FF940490880384A517A364A907D01F00DF80290344A527A0F3A91B2314A507D98
:20DF800001F004F80190DDE9011048434FEA902B1FFA8BF001231A463349098801F060F93E
:20DFA00031490880274AD17B274A127A012383EAD21002F0D3FB2D4909884843642190FBD0
:20DFC000F1F0801200B200901E480089C111284A009804F043F9274908801E48B0F9060084
:20DFE0002049098848434FEAA0281F48008808FB00F04FEAA0281F48B0F9000040444FEAEB
:20E000006008B8F1000F01DA002000E0404600B2ADF8160001208DF81A0004208DF8140095
:20E020000598CAF800000698CAF804000BB0BDE8F08F0000D00A0020580100205601002054
:20E040005A010020DC080020B00A0020B9010020E4030020F000002000010020F00A00203B
:20E060005C0100205E010020600100205201002008070020500100202DE9FF4F8BB08146AA
:20E080008A46FE4903C9CDE909014FF0000B0020089005900490FA48A0F802A0F94800886D
:20E0A000C82801DA642002E0F648008840100690F34841880698814204DBFCF715FEF249FE
:20E0C000086020E0F148B0F90200C82807DDEF48B0F90200EE4991FBF0F086B201E04FF43F
:20E0E0009666B6F5FA7F02DA4FF4FA7000E030460646FCF7F9FDE4490968401AB04202D927
:20E100000120DF490870E14800883C2814DDDD480088C82801DA96200CE0DA480088B0F5CF
:20E120002F7F02DD40F20D2004E0D648008800EB40008010079010E0D2480088C82801DABA
:20E14000962009E0CF480088B0F52F7F02DD40F20D2001E0CB4800880790C9484188079864
:20E16000814202DB0020C6490870CA484078012802D0C848807810B90120C1490870C04817
:20E18000007801283ED1BE48B0F90610C2484079002801DA032007E0BF484079052801DD6F
:20E1A000032001E0BC484079401EBC4A105C81420CDC0020B249C880B94802F038FB012079
:20E1C000B84908700020B8490880B6E3AC48B0F90610B1484079002801DA032007E0AE481C
:20E1E0004079052801DD032001E0AB484079401EAA4A105C081A00B2A149C880A84802F005
:20E2000009FB9AE39E490E984880A048B0F90200B0F5FA7F23DD9F4800780F281FDB084699
:20E220004088C8281BDD9948B0F90200642148439849097890FBF1F09C4908609C4800682B
:20E240000968C0EB01309A49096801EBA0209849086008460068C0F30F30964908800D9874
:20E2600003287DD004DC012807D0022879D160E0042877D03328F9D198E18F48007A002808
:20E2800001DC012001E08C48007A83468A48407A0890DFF8ECC1BCF80230DFF81CC2BCF891
:20E2A0000220BCF80010BCF800C04FEA6C00F7F797F9734949884843800A04B27E488088BB
:20E2C000A04202DD7C48808800E0204604B27A48C088A04202DA7848C08800E0204604B2E9
:20E2E000754840896C49097A48434FF47A714843401400EBC00101EB00104FF6FF7101EA80
:20E300008005012305226D480188284600F0A8FF6A4908806848C0884042694908610020FA
:20E3200048616548C0888002404288610020C861ABE16148007D002801DC012001E05E48AA
:20E34000007D83465C48407D0890DFF834C1BCF80230DFF864C1BCF80E20BCF80C1002E03C
:20E3600047E08CE1C7E0BCF80CC04FEA6C00F7F737F9434949884843800A04B24E48008AD7
:20E38000A04202DD4C48008A00E0204604B24A48408AA04202DA4848408A00E0204604B232
:20E3A0004548C08A3C49097A48434FF47A714843401400EBC00101EB00104FF6FF7101EA9E
:20E3C0008005012305223D480188284600F048FF3A4908803848408A4042394908610020D8
:20E3E00048613548408A8002404288610020C8614BE1314890F82000002801DC012002E0A2
:20E400002D4890F8200083462B4890F821000890DFF86CC0BCF80230DFF89CC0BCF81A2058
:20E42000BCF81810BCF818C04FEA6C00F7F7D8F8134949884843800A04B21F48808BA042C5
:20E4400002DD1D48808B00E0204604B21A48C08BA04202DA1848C08B00E0204604B2164801
:20E46000408C0D49097A48434FF47A714843401414490978484385B2012325E068780108AD
:20E48000F00000201204002068010020DC08002020550300B4030020B00A0020010100205E
:20E4A0000001002071010020720100207C01002080010020FA010020E40B00206E0100201F
:20E4C00008070020EE0000200522FE480188284600F0C6FEFB490880FB48C08B4042FB49C7
:20E4E000086100204861F848C08B8002404288610020C861C9E0F44890F82C00002801DC8B
:20E50000012002E0F04890F82C008346EE4890F82D000890DFF8B8C3BCF80230DFF8A8C346
:20E52000BCF82620BCF82410BCF824C04FEA6C00F7F756F8E64949884843800A04B2E2488B
:20E54000008DA04202DDE048008D00E0204604B2DD48408DA04202DADB48408D00E02046D6
:20E5600004B2D948C08DDB49097A48434FF47A7148434014D8490978484385B20123052289
:20E58000D0480188284600F06BFECE490880CE48408D4042CD49086100204861CA48408DE8
:20E5A0008002404288610020C8616EE0C64890F83800002801DC012002E0C34890F8380036
:20E5C0008346C14890F839000890C1484088B0F5FF7F15DADFF8F8C2BCF80230DFF8E8C235
:20E5E000BCF80E20BCF80C10BCF80CC04FEA6C00F6F7F6FFB64949884843800A04B207E0E0
:20E60000B34840884043B049498EB0FBF1F004B2AD48808EA04202DDAB48808E00E0204697
:20E6200004B2A948C08EA04202DAA748C08E00E0204604B2A448408FA649097A48434FF4F3
:20E640007A7148434014A4490978484385B2012305229C480188284600F002FE9949088040
:20E660009948C08E404299490861002048619648C08E8002404288610020C86105E04FF04F
:20E68000000B00200890002400BF00BF934890F90E00322805DC914890F90E0010F1320FB6
:20E6A00002DA00208D4988738C4890F90F00322805DC8A4890F90F0010F1320F02DA00203E
:20E6C0008649C873864AD17B824A1279012383EAD21002F071F87F490979804A92F9102020
:20E6E000114401EB81017D4A92F90E2002EB41014843C0F38F207B490880794AD17B754AA1
:20E700001279012383EAD21002F056F871490979724A92F91020114401EB81016F4A92F901
:20E720000F2002EB410116314843C0F38F206E490880084600886B490988401AC01E4FF472
:20E74000806191FBF0F0694908806948008800900846008803B26348028800210088F9F710
:20E760005DFA6043800A04B259488480B0F90400002802DC0020564988805D480088594971
:20E780000988884220DD5248B0F904005049B1F90610401A022806DD4D48C088401C00B22F
:20E7A0004B49C880ABE04A48B0F904004849B1F90610401AB0F1FF3F05DA4548C088401E17
:20E7C00000B24349C8809AE000BF4A480078012857D140484078032805D1002046490880A7
:20E7E000444908708BE03B484078012805D14FF4967005901E20049003E0642005900A2099
:20E8000004903D480088401C3B49088008460188059881422FDC2E48B0F904002C49B1F96B
:20E820000610401A022814DD33480188049891FBF0F0C0F10A003049098891FBF0F200FB13
:20E84000121068BB2248C088584400B22049C88055E01F48B0F904001D49B1F90610401AF9
:20E86000B0F1FF3F4BDA1A48C1880898081A00B21749C88043E000201F4908801D490870BC
:20E880003DE01348B0F904001149B1F90610401A022806DD0E48C088584400B20C49C88049
:20E8A0002DE00B48B0F904000949B1F90610401AB0F1FF3F23DA0648C1880898081A00B2F8
:20E8C00003491BE06E010020E40B002008070020F0000020B00A0020EE000020D00A002032
:20E8E000DC080020840100208601002088010020E40300207101002072010020C8804A4819
:20E90000B0F90600062801DA062002E04648B0F906004549C8804548008845490988884226
:20E9200008DD0120404908700020C880414801F07EFF02E03F4801F06DFF3F4A117B3F4A0D
:20E94000D0883F4A128800F033FB80463C48A0F8008001231A463B480188404600F080FC3A
:20E9600038490880384A517A344A907D00F00EFB0290354A527A0F3A91B2304A507D00F01D
:20E9800005FB0190DDE901104843810A0391039988B201231A462D49098800F061FC2B4943
:20E9A0000880264AD17B284A127A012383EAD21001F0D4FE264909884843642190FBF1F063
:20E9C000801200B200901D480089C111214A009803F044FC204908801348B0F90600194910
:20E9E00009884843871219480088784387121A48B0F9000038444710002F01DA002000E03D
:20EA0000384600B2ADF8260001208DF82A0002208DF824000998C9F800000A98C9F8040097
:20EA20000FB0BDE8F08F0000F0000020E40300208601002000010020F00A0020DC080020F6
:20EA40007401002076010020B00A0020780100206E010020080700206C0100202DE9FF5F58
:20EA600082460E468C4903C9CDE90201002700BF0025002E40D1A9468848C07F08B9872070
:20EA800001E08648C07F8146854840680A21C1EB4911884205D282484068401C804948603B
:20EAA00010E07F4840680A2101EB4911884205D97B484068401E7A49486003E04FEA491035
:20EAC00077494860774AD17B744A127A012383EAD21001F043FE7149097A4FF4FA72514352
:20EAE0004843401400906F480089C1116E4A009803F0B4FB044655E06C484088400141F234
:20EB0000883190FBF1F0C5B2012D01DA012000E02846054665484088400165490978484326
:20EB2000642190FBF1F00A385D494968884205D95B48406828445A49486026E05B48408830
:20EB400040015B4909784843642190FBF1F00A305349496888420DD251484068A84205D99A
:20EB60004F484068401B4E4948600EE000204C4948600AE04D48408840014D490978484347
:20EB8000642190FBF1F046494860464A1289D111424A127A4FF47A735A43D011424A03F0FB
:20EBA0005DFB04463F4AB2F902103D4A5268520910B2404A03F052FB0746381907B236BBFD
:20EBC0004FF000093548807F08B93C2001E03348807F814633480088A9F105018AB20090C3
:20EBE00088B280230021F9F719F87843800A07B22C480088484506DD0020294948602E48FC
:20EC000001F015FE02E02C4801F004FE02E02A4801F000FE254A117B224AD088274A12889A
:20EC200000F0C6F980462548A0F8008001231A4623480188404600F013FB21490880174A8B
:20EC4000517A184A907D00F0A1F9019001231A461C480188019800F003FB1A49088018481C
:20EC6000008878434FEAA02B084600880BFB00F04FEAA02B0FFA8BF0ADF80C0001208DF8A2
:20EC80000E008DF808000298CAF800000398CAF80400BDE8FF9F000058780108B00A002026
:20ECA000F8000020DC080020C0060020F00A0020CF010020E406002000010020620100209A
:20ECC000640100206601002070B504460D461646FCF70AF83C490968401A642870D3FCF703
:20ECE00003F8394908603948006828443749086037480078401C36490870084600780828B2
:20ED00000ADB32480068C0F3CF003249088000202F4908702D490860462C0BDA2D48008865
:20ED200041F27071884205DD2B480088401C2A49088002E0002028490880462C05DC254806
:20ED4000008841F28831884207DA962E05DA23480088401C2149088002E000201F490880BE
:20ED60001D480088B0F5967F05DD00201A49088001201B49087019480088642804DD00208C
:20ED8000164908801649087015480078012814D1462C0EDA04F11E001249087008460078CC
:20EDA000642801DD642001E00E4800780D49087006E064200B49087002E064200949087082
:20EDC0000848007870BD0000A4000020A8000020AC000020AE000020B0000020B200002076
:20EDE000B4000020B50000202DE9FF4385B0074615469846DDE9109408EA090000F00103FE
:20EE0000BDF81A10554800782A46049001F060FC06462078B04223D05148007800BB0526ED
:20EE200001204F4908702078042819D14D480068142806DD04260020087001204A490870E9
:20EE40000EE00020494908604949086049490880444908604449087005260120404908704F
:20EE6000062E68D2DFE806F06733574B03683B48007800F0010078B905F00F03BDF81A20AD
:20EE8000364800780146029003A8FEF733FA039820600498606016E03048007800F0010088
:20EEA00088B105F00F000090BDF81830BDF81A202A4800780146029003A8FEF72BFD039873
:20EEC00020600498606000202549087041E02A480078012807D12948B0F902004001264978
:20EEE000486000200870394603A8FFF7B7FD039820600498606000201949087029E0294615
:20EF000003A8FEF7DDF903982060049860600020134908701DE01A480389BDF818102A46D8
:20EF200003A8FFF7A9F8039820600498606000200B4908700DE000BF124801F078FC124867
:20EF4000F6F7FCFD052020700020A0716080A08000BF00BF09B0BDE8F0830000B9010020BC
:20EF60008A010020400100204401002008010020200100203C010020F8000020DC0800203D
:20EF8000B4030020000100208C01002010B502464FF480608A4208DD01FB01F4A302B3FBA7
:20EFA000F2F4B4FBF2F4A0B201E04FF4806010BDF0B503460E461546002100244FF48060AE
:20EFC000182E04D0242E12D0302E34D121E0E721FC2401EBC10707EB0117B3EB870F02DD86
:20EFE0004FF4806701E0B3FBF1F73A4625E04FF4A5714FF4B47401EBC10707EB0117B3EBCB
:20F00000870F02DD4FF4806701E0B3FBF1F73A4613E040F2AD114FF4EA7401EBC10707EB30
:20F020000117B3EB870F02DD4FF4806701E0B3FBF1F73A4601E0642200BF00BF02FB02F7A9
:20F040004FF0640CB7FBFCF75743B7FBFCF75743BF0242F2107CB7FBFCF2B2F54D7F02D21B
:20F060004FF44D7700E017463A46AA4201D290B200E0284604EBC40707EB0417B3EB870F82
:20F0800001DD4FF48060F0BD2DE9F04105460E4617461C46002F7DD1552D66D147480078E0
:20F0A00020BBFBF721FE45494968401AB0F57A7F15D901204149087000202070404800786C
:20F0C000C043404908703E484078C04348703E48007820F00200801C3B49087018E03A4811
:20F0E000007820F002003849087011E00020207033480078C0433349087031484078C043CE
:20F1000048703148007820F00200801C2E490870AA2E06D12C48007820F004002A4908700F
:20F1200023E02A480078C8B9FBF7DEFD27494968401AB0F57A7F0AD9012024490870224828
:20F14000007820F00400001D1F4908700DE01E48007820F004001C49087006E01A480078AA
:20F1600020F00400001D1849087019480078E0B9FBF7BAFD16494968401A41F2883188424A
:20F180000CD90120124908700F48007820F00100401C00E010E00C4908700DE00A48007806
:20F1A00020F001000849087006E00748007820F00100401C04490870BDE8F081D801002087
:20F1C000DA000020DC000020B0010020E0010020E801002001201349087000204860012080
:20F1E00011490870002048808880C8800F4908600F4908600F4908600F4908600F49086045
:20F200000F4908600F4908600F4908620F4908620F4908620F4908620F4908620F490862E2
:20F2200070470000F8000020F000002004000020080000200C000020100000201400002013
:20F24000180000201C00002078060020540600209C06002008070020E4060020C006002041
:20F2600070B504461546661A32B2002A06DDAA4202DB4E19B0B20CE020460AE0002A07DA7A
:20F2800056429E4202DBCE1AB0B202E0204600E0204670BD10B5FBF727FD2E490968401AF7
:20F2A000642855D3FBF720FD2A4908602A4800782A4908702A480078487000208870C870E9
:20F2C0002848008800B288802748008800B2C880264840880881254800884881244800881A
:20F2E000888123484088C88122480089088222480068801200B2488220480068801200B218
:20F30000888215480078022803D113484088C8821EE011480078012804D10F4880880F491F
:20F32000C88215E00C48007804280ED11448007800F0010020B9084880880849C88207E03F
:20F34000054840880549C88202E000200349C88210BD000084000020DE000020FC080020D5
:20F360003000002004000020080000202C00002032050020B4030020100000200C0000201B
:20F38000B901002070B505460E46144608216748FBF798FC664908704FF400416548FBF7CD
:20F3A00091FC6549087062480078644909784840634908705E480078604908705E48007841
:20F3C000604909784840604908705B4800785D490870574800785849097848405B49087044
:20F3E000FBF782FCB0F57A7F0CD2FBF77DFC58490860FBF779FC57490860FBF775FC56493C
:20F40000086070BD2088C0F38030002878D1B5F5966F7CDD462E7ADD4948007800BBFBF752
:20F4200063FC4B490968401A42F2107188421BD9206820F4804000F5804020600120474959
:20F4400048800846F8F72CF900204549087045484088401C43494880022043490870D0E77A
:20F46000FBF742FC3A4908603748007800BBFBF73BFC38490968401A41F2883188421BD9A0
:20F48000206820F4804000F5804020600220334948800846F8F704F90020314908703148B0
:20F4A0004088401C2F49488002202F490870A8E7FBF71AFC274908602448007810BBFBF7C6
:20F4C00013FC25490968401A41F2883188422AD9206820F4804000F58040206003201F490F
:20F4E00048800846F8F7DCF800201D4908701D484088401C1B49488002201B49087080E71B
:20F5000011E004E0FBF7F0FB134908600BE0FBF7EBFB0F490860FBF7E7FB0E490860FBF76D
:20F52000E3FB0D49086000BF6BE70000000C0140C802002000080140C9020020B1020020E0
:20F54000B0020020B9020020B8020020C0020020B4020020BC020020C402002098070020E9
:20F5600091030020300B0020BA0100201FB53948007890B93848807E55280ED1374A3848B0
:20F5800000783849498889B2CDE9010200913649887836490EC900F0A9FE3049344A304841
:20F5A0000078CDE902210190304880680090314801782E480CC8304800F030FF27480190A6
:20F5C0002E488088ADF80000264B5B889AB2254B1989234B9879294B1C6802949B88ADF881
:20F5E0000C30234600F0A2FD1E4A917D507D1B4A00F01EFD20490839088A184900F076FA27
:20F600001E48016802918088ADF80C00134ADDE9020100F0D3FB114800F03EF80F48134AB8
:20F62000009011780F4A528890B2154A12680392144A1388039A00F095FC0848124900907C
:20F64000CA8912490878124B1249098800F010FB1FBD0000D8000020B00A00208C010020DD
:20F66000DE000020DC080020E4030020B403002010040020DA000020E41E002042050020F3
:20F6800032050020FA010020F21E0020D0010020E3070020CC01002010B50446FBF724FBC0
:20F6A00041F2883188420CD2FBF71EFBEE490860FBF71AFBED490860FBF716FBEC490860C7
:20F6C00010BD2068C0F3804000286FD14FF40041E848FBF7F7FA00BBFBF706FBE349096818
:20F6E000401A41F2883188421BD9206820F4802000F5802020600120DF4948800846F7F768
:20F70000CFFF0020DD490870DD484089401CDC4948810220DB49087003E0FBF7E5FAD34997
:20F720000860D9480088002847D1D8480078012843D1D748007805283FD0D5488079012891
:20F740003BD1D348B0F90400C82804DCD048B0F90200C82831DDCF48807A40BBCE48008999
:20F76000C82825DAFBF7C0FAC1490968401A41F28831884225D9206820F4802000F5802094
:20F7800020600220BC494880BF48008888800846F7F786FF0020B9490870B9484089401CE2
:20F7A000B74948810220B74908700AE08DE0FFE7FBF79AFAAE49086003E0FBF795FAAC496B
:20F7C0000860FBF791FAA8490968401A14287CD3FBF78AFAA4490860B048C088B049096888
:20F7E0000844AF490860AF480088AF4909680844AD490860AB484088AC4909680844AB496A
:20F800000860A8488088AA4909680844A8490860A8480078401CA749087008460078202845
:20F820007EDB002008709E4800684FF4FA71B1EB501F2FD89A480068C900B1EB501F29D3AF
:20F840009948006841F28831B1EB501F22D8964800684EF66021B1EB501F1BD39348006827
:20F8600041F28831B1EB501F14D8904800684EF66021B1EB501F0DD38D48006841F288318C
:20F88000B1EB501F06D88A4800684EF66021B1EB501F16D2206820F4802000F5802020603C
:20F8A0000320754948800846F7F7FAFE00207349087073484089401C7149488102207149D8
:20F8C00008707D480068C82100E0C2E0B1EBA02F36DA7A48008872490968C0EB51101928DA
:20F8E0002AD277480078401C75490870084600780A2828DD206820F4802000F580202060F5
:20F9000004205D49488066480068C0F34F1088800846F7F7C5FE002058490870584800E06D
:20F920001AE04089401C5649488102205549087000206349087006E000206149087002E0BA
:20F9400000205F4908700020554908605649086056490860564908604F48407B00287AD167
:20F960004D484088002876D1FBF7BEF955490968401A41F28831884274D94848C088524933
:20F98000524A127821F812004648008850494F4A127821F81200434841884E484B4A127810
:20F9A00020F812103F4881884B48484A127820F8121046480078401C444908700846007867
:20F9C00032284FDB0020087032213F48F8F744FE4249086032213E48F8F73EFE4049086018
:20F9E00032213C48F8F738FE3E49086032213A48F8F732FE3C49086038480068B0F5FA7F35
:20FA00000DD83748006842F6E061884207D835480068884203D834480068884222D920683D
:20FA200020F4802000F5802020600520124948802A48008888800846F7F732FE00200F49CF
:20FA400008700F484089401C0D49488102200D49087007E0FFE700201C490870FBF744F9AA
:20FA60001849086000BF2BE654020020580200205C020020001001409807002091030020BB
:20FA8000300B0020BA010020C401002030000020DE000020D8070020DC080020F21E0020CA
:20FAA000640200202A050020680200206C02002070020020600200200C00002048050020AC
:20FAC00061020020880200205413002074020020B81300201C140020801400207802002053
:20FAE0007C02002080020020840200207047000013B50C465448007860B9FBF7F5F85349A7
:20FB000008609DF8012006215148F3F7DAFF01204D4908702078C0F3C01000287ED19DF8EE
:20FB2000000018B19DF80000072821D1FBF7DCF846490968401AB0F57A7F1DD9206820F0FA
:20FB40008000803020600120424948809DF8000088800846F7F7A4FD00203F4908703F4860
:20FB6000C08A401C3D49C88201203D4908701CBDFBF7BAF8354908609DF800009DF8011052
:20FB800088425FD09DF80010364802780078401C344B18702E48815418460078062851DB79
:20FBA00000201946087006212948F5F7E3FC28B92D480068401C2C49086006E000202A497B
:20FBC0000860FBF791F82949086027480068322838D9FBF789F82549096801F5FA718842A9
:20FBE00030D9206820F08000803020600220194948801748007800021549497800EB011074
:20FC0000134989780844134988801148C07800020F49097900EB01100D4900E012E0497984
:20FC200008440C49C8800846F7F73AFD00200A4908700A48C08A401C0849C8820120084978
:20FC4000087094E700BF92E79A0200209C020020A40200209807002091030020000B00209B
:20FC6000BA010020AA020020AC020020A00200202DE9F04105460E4614469846069FFBF798
:20FC800033F8B0F57A6F01D2BDE8F081FBF72CF842F21071884220D23868C0F38040002800
:20FCA0007CD1FBF721F83E490968401A142875D3FBF71AF83A49086098F80000A8BB0DB176
:20FCC000C82E0BDD40F2C270844207DD40F63E00844203DA0020334908705FE031480078DD
:20FCE000401C3049087008460078FA2856DB00200870386820F4802000F58020386008205D
:20FD00002949488005EB860088800846C480F7F7C7FC00202549087025484089401C2449E3
:20FD2000488102202349087038E0FFE70DB1C82E03DD002088F8000030E040F68B608442CB
:20FD400002DCB4F5BA7F26DA1B480078401C1A49087008460078FA2820DB002008703868B6
:20FD600020F4802000F58020386009200E49488005EB860088800846C480F7F791FC0020AF
:20FD80000A4908700A484089401C0949488102200849087002E000200749087000BF73E738
:20FDA00094020020980200209807002091030020300B0020BA0100209902002037B5144629
:20FDC0006048007801280CD0FAF78EFF5E490860FAF78AFF5D490860FAF786FF5C49086066
:20FDE0003EBD2068C0F30040002875D1BDF90000002801DB014600E0414244F6206291422C
:20FE000028DDFAF771FF50490968401AB0F57A7F24D9206820F4803000F5803020600120EB
:20FE20004C494880BDF90000002801DB014600E04142484A91801046F7F732FC002046493D
:20FE400008704648C088401C4449C880022044490870C5E7FAF748FF3B490860BDF9020074
:20FE6000002801DB014600E0414244F62062914228DDFAF739FF35490968401AB0F57A7F30
:20FE800024D9206820F4803000F580302060022030494880BDF90200002801DB014600E0AE
:20FEA00041422C4A91801046F7F7FAFB00202A4908702A48C088401C2849C8800220284992
:20FEC00008708DE7FAF710FF20490860BDF90400002802DB014601E031E0414244F620622E
:20FEE000914228DDFAF700FF19490968401AB0F57A7F24D9206820F4803000F58030206001
:20FF0000032014494880BDF90400002801DB014600E041420F4A91801046F7F7C1FB0020A7
:20FF20000D4908700D48C088401C0C49C88002200B49087054E7FAF7D7FE0549086000BFF9
:20FF40004EE70000300000203C02002040020020440200209807002091030020300B002028
:20FF6000BA0100202DE9FF4105460E461F460A9C2068C0F3805000284BD1FAF7B5FE264944
:20FF80000968401A142844D3FAF7AEFE22490860B5F5FA7F3ADD0F2E38DBBDF80800C8289C
:20FFA00034DDBDF80A00322830DA40F2DC50874228DD1A480088401C1849088008460088DC
:20FFC000FA2826DB00200880206820F4800000F580002060002012494880BDF8080088803D
:20FFE000BDF80A00C8800846F7F75AFB00200D4908700D480089401C0B49088102200B49EE
:020000040801F1
:20000000087006E000200549088002E0002003490880BDE8FF8100008C0200209002002031
:200020009807002091030020300B0020BA01002070B504460E461546FAF756FE41F28831C8
:20004000884201D35A2C08DDFAF74EFE31490860FAF74AFE2F49086070BD2888C0F340206F
:20006000002855D1052C01DBBE2C22DDFAF73CFE28490968401A41F2883188421DD9286899
:2000800020F4007000F50070286001202249488008468480C680F7F703FB00201F49087017
:2000A0001F48408B401C1E49488301201D490870D2E7FAF719FE17490860052E01DBBE2EFD
:2000C00022DDFAF711FE18490968401A41F2883188421DD9286820F4007000F50070286048
:2000E00002200D49488008468480C680F7F7D8FA00200A4908700A48408B401C08494883E8
:20010000012008490870A7E7FAF7EEFD0649086000BFA1E7340200209807002091030020C4
:20012000000B0020BA010020380200200FB42DE9F04105460E4617460B9C2088C0F3002037
:20014000002877D1012D76D141F28830864272DDB7F5FA7FFBDDBDF92400002801DB014696
:2001600000E04142B1F5967F2CDAFAF7BDFD58490968401A41F28831884227D9206820F4F2
:20018000807000F580702060012052494880BDF92400002801DB014600E041424D4A918056
:2001A0001046F7F77DFA00204B4908704B48008B401C4A490883012049490870BDE8F001FF
:2001C0005DF814FBFAF790FD41490860BDF92600002801DB014600E04142B1F5967F2BDA01
:2001E000FAF782FD3F490968401A41F28831884226D9206820F4807000F580702060022074
:2002000034494880BDF92600002801DB014600E04142304A91801046F7F742FA00202E496D
:2002200008702E48008B401C2C49088301202C490870C3E73CE03CE0FAF756FD29490860DB
:20024000BDF92800002801DB014600E04142B1F5967F29DAFAF748FD23490968401A41F2B4
:200260008831884231D9206820F4807000F580702060032017494880BDF92800002801DBD3
:20028000014600E04142134A91801046F7F708FA0020114908701148008B401C0F490883EB
:2002A00001200F49087089E7FAF71EFD0E4908600BE0FAF719FD06490860FAF715FD094914
:2002C0000860FAF711FD0849086000BF76E70000280200209807002091030020000B0020FA
:2002E000BA0100202C020020300200202DE9FF410646DDE90A870C9C00252078C0F3401022
:20030000002878D1052F08D1FAF7EEFC3B490860FAF7EAFC3A4908606DE0012F01D0042F55
:2003200032D1B8F1320F2ADD4EBB364890FBF8F085B242F21070854200DA00E028460546AA
:20034000FAF7D2FC2D490968401AA84253D9206820F020002030206001202B494880084654
:20036000F7F79EF90020294908702948408A401C27494882012027490870BDE8FF81FAF7FE
:20038000B3FC1E49086036E09DF8040005282EDB9DF8050058BB56BB9DF804001E4991FBB0
:2003A000F0F085B242F21070854200DA00E028460546FAF799FC12490968401AA8421AD9AF
:2003C000206820F020002030206002200E4948800846F7F765F900200C4908700C48408AAF
:2003E000401C0B49488201200A490870C5E7FAF77BFC0349086000BFBFE700001C0200202C
:200400002002002048F13E009807002091030020000B0020BA010020D8B805000FB42DE93C
:20042000F84305460E46DDE90D840F9FFAF75CFC41F28831884207D35E480078012803D0EA
:200440005C480078022819D1FAF74EFC5A490860FAF74AFC58494860FAF746FC5649086468
:20046000FAF742FC54494864FAF73EFC5249C1F88000FAF739FC5049C1F88400FAF734FCE8
:200480004E490968401A142847D3FAF72DFC4B490860222E27D006F00F0020B39DF82800B2
:2004A0001E2820DD9DF82900E8B9B8F1020F1AD100949DF8283028883F4A012100F088F8A9
:2004C00000949DF8283068883B4A4032022100F07FF800949DF82830A888374A8032032122
:2004E00000F076F819E0FAF7FFFB33490860FAF7FBFB31494860FAF7F7FB2F490864FAF715
:20050000F3FB2D494864FAF7EFFB2B49C1F88000FAF7EAFB2849C1F884003878C0F38010CC
:20052000F0BB207800F001002178C1F3400108442178C1F380010844022838DD386820F0A4
:20054000400040303860207800021D4948801A48418FB0F87A0001EB80011748B0F8BA0009
:2005600001EB0010164949880843154948801248818F90F87C0001EB0020114988800E48AC
:20058000B0F8BC00C8800846F7F78AF800200D4908700D48808A401C0B498882012000E0E9
:2005A00005E00A490870BDE8F8035DF814FB00BFF9E70000D80000209412002024020020E4
:2005C0009807002091030020000B0020BA0100202DE9F0470546884614469946089E002736
:2005E00008E004F10800791C30F8111020F81710781C87B2182FF4D32587192104F108003B
:20060000F8F72AF8E063E06B0A2812D2FAF76CFB2168401A43F6982188420DD93078A8F107
:20062000010101228A401043307001206087BDE8F087FAF759FB2060322D03DB40F6D2703A
:20064000854210DDFAF750FB6168401AB0F57A7F0CD93078A8F1010101228A4010433070E1
:2006600002206087E3E7FAF73FFB606000BFDEE710B51149487B01F00BFD0F49487B05F04D
:200680009DFB0E4803F09AFC0C48F5F757FA0C4801890C4804F0BAFE094841890A4804F013
:2006A000B5FE07488189094804F0B0FE01F0F0FE012001F019FF10BDB00A00208C010020DE
:2006C000DC1E0020F01500200A160020241600202DE9FF410E4615461F461D48006850BBFF
:2006E00025B3012F22D1FAF7FFFA40F6B83188421CD9C82E0BDD9DF80000552807D09DF8DB
:200700000000F82801D1012411E004240FE0642E0DDA222D01D1012409E005F0F00018B164
:20072000332D01D0032402E0022400E00524012001F0DAFE08E00524002006490870084620
:200740000078C04304490870204604B0BDE8F0818C010020DA000020DC00002010B5024679
:200760004FF480630AB9184610BD022902DC4FF480731FE0062906DC881E4FF4807404EB4A
:20078000801083B216E0162908DC881F00EB40004FF4007404EBC00083B20BE01E2907DCF9
:2007A000A1F116004FF4607404EB001083B201E04FF480631846D7E710B502464FF48063F0
:2007C0000AB9184610BD022902DC4FF400731FE0062906DC881E4FF4007404EB401083B28B
:2007E00016E0162908DC881F00EB80004FF4207404EB800083B20BE01E2907DCA1F1160096
:200800004FF4707404EBC00083B201E04FF480631846D7E710B50446207838B9F6F7DEFE49
:20082000FBF7DAFFF7F772F80120207010BD10B5044601F04DFFF7F757F8FEF7CBFC0020B2
:20084000207010BD2DE9F04107460D46144605EB4500C0F34F06207800F0010050BBB74230
:2008600003DAFAF741FA1C490860FAF73DFA1A490968401A41F2883188422AD9206820F0FB
:200880000100401C206002201449488008468680F6F706FF00201249087012480089401CBC
:2008A00010490881012010490870FAF71DFA0F4908600EE0FAF718FA0C490968401A41F258
:2008C0008831884205D90A48006820F0010008490860BDE8F0810000FC0200209807002040
:2008E00091030020000B0020BA010020000300208C0100201CB52C492C48808BC0F30B00EB
:2009000010B940F6B83001E02848808B284CCDE90001237B274C247814B9274C248801E0EF
:20092000264CE4882246254CE17B224C207800F0FFF92248008941F2883188420DDA1C4AC0
:20094000117B2246127812B91B4A128801E01B4AD2881046144A00F0FFF8194A917A174A45
:200960001089114A00F060F90F48104C0090A37A124CA27D617DE07D00F04EF822461189EA
:20098000D088094A00F0ACFA084A127A02EB4203C3EBC2124FF6FF7303EAC201224610891C
:2009A000014AFFF74FFF1CBD8C010020B00A0020F00A0020E80100207C090020DC0800207C
:2009C000D807002070B504460D46207868B900200F4908700F480078C0B90E480078401C3B
:2009E0000C490870F6F7E0FD10E000200949087007480078012802DB0020207001E0F6F73B
:200A000003FB03480078401C0149087070BD000004030020050300202DE9F04180460E461A
:200A200017461C46069DFAF75FF940F6B831884207D2FAF759F940490860FAF755F93F494E
:200A400008602878C0F3001000283DD13C48C07A58B9A4F11900B04215DD2330874212DA2C
:200A6000FAF742F9344908600DE0A4F11900B04209DD2330874206DA1E38404503DDFAF74A
:200A800033F92D490860FAF72FF92B490968401A41F2883188424CD9FAF726F92749086031
:200AA000286820F01000103028602648F6F7F8FD0020254908702548008A401C234908821F
:200AC00001202349087034E01D48C07AB8B9A4F12300B0422DDD0F30B8422ADDFAF704F90B
:200AE00016490968401A1B49884222D9286820F010002860FAF7F8F80F49086019E0A4F13C
:200B00002D00B04215DD1930B84212DD0A3840450FDDFAF7E9F809490968401A0D498842D0
:200B200007D9286820F010002860FAF7DDF802490860BDE8F0810000EC020020F0020020EE
:200B4000D80700209807002091030020000B0020BA010020E09304002DE9F04105460E46C0
:200B600014460027182E04D0242E05D0302E09D105E047F60C3707E04AF6C87704E04EF28C
:200B8000844701E02F4600BF00BF2078C0F3800030BBBD4203DCFAF7A7F81D490860FAF7D3
:200BA000A3F81B490968401A41F28831884212D9206820F00400001D20601648F6F770FDD9
:200BC00000201549087015488089401C13498881012013490870FAF787F81249086014E0DC
:200BE000A7F5FA70A84203DAFAF77EF80D490860FAF77AF80B490968401A41F288318842CB
:200C000003D9206820F004002060BDE8F0810000D80200209807002091030020000B00202E
:200C2000BA010020DC02002070B505460E4614462078C0F3C000002849D1012E08D1FAF777
:200C400053F831490860FAF74FF83049086014E040F6C410854208DAFAF746F82A4908609D
:200C6000FAF742F82949086007E041F64C50854203DAFAF739F825490860FAF735F8224990
:200C80000968401A41F28831884208D8FAF72CF81E490968401A40F6B831884232D9206830
:200CA00020F00800083020601948F6F7F9FC0020184908701848C089401C1749C881012059
:200CC00016490870FAF710F8154908601AE0FAF70BF813490968401A41F28831884211D9C9
:200CE0001048007870B9104800880A280ADA0E4840880A2806DA0D48807818B9206820F01F
:200D00000800206070BD0000E0020020E40200209807002091030020000B0020BA0100209D
:200D2000E8020020DA00002032050020B40300202DE9F0478046894615469A46DDE9086432
:200D400000270120B0EBE63F4ED12078C0F34000A0BBB9F1010F03DBF9F7C6FF5A4908602E
:200D6000F9F7C2FF58490968401AC6F3023101EB8101052202EB410101EB4102C2EBC111F8
:200D8000B0EBC10F15D9206820F00200801C20604E484580A0F80480F6F782FC00204C49AD
:200DA00008704C484089401C4A49488101204A490870F9F799FF4949086082E0FFE7B9F106
:200DC000050F03DAF9F790FF44490860F9F78CFF42490968401A41F28831884271D9206855
:200DE00020F0020020606CE0BAF1180F06D0BAF1240F08D0BAF1300F12D10AE0C6F30B003C
:200E0000C0EBC0070EE0C6F30B0000EB8000470008E0C6F30B0000EB800101EBC00701E050
:200E20002F4600BF00BF2078C0F3400098BBBD4203DBF9F759FF24490860F9F755FF224938
:200E40000968401AC6F3023101EB8101052202EB410101EB4102C2EBC111B0EBC10F15D910
:200E6000206820F00200801C206018484580A0F80480F6F715FC0020154908701548408961
:200E8000401C14494881012013490870F9F72CFF1249086015E0FFE707F57A70854203DA98
:200EA000F9F722FF0D490860F9F71EFF0B490968401A41F28831884203D9206820F002000B
:200EC0002060BDE8F0870000D00200209807002091030020000B0020BA010020D402002015
:200EE0002DE9F0410746884614460026F9F7FCFE2B490968401A642850D3002507E02949BA
:200F0000681C31F8100021F81500681C85B2092DF5D3244847820A21F7F79EFB0646206872
:200F2000C0F3404090BBB8F1320F2BDAB6F57A7F28D91D480078322830DD206820F400308F
:200F400000F500302060C6F30F20184948800A211448F7F7F5FA154988800A211148F7F79F
:200F600000FB1249C8800846F6F79AFB00201049087010480089401C0E49088102200E497C
:200F800008700BE000200849087007E0FFE7B6F57A7F03D8206820F400302060BDE8F08157
:200FA000F402002050070020F80200209807002091030020300B0020BA01002010B5F9F72C
:200FC00093FEA2490968401AC8287DD3F9F78CFE9E4908609E480088C01268B99D480089F2
:200FE000FA2148439C49097A4FF47A725143B0FBF1F09849888016E095480088C0F30A0093
:2010000093490988012202EBE121484340119149098948439049097A4FF47A725143B0FBB4
:20102000F1F08C4988808B488088142801DA002001E088488088874988808848407808734C
:20104000874800881C2190FBF1F08249C8728548007848738348407888738348007800F0DA
:20106000010040B17A48037B0846C27B7F498048F3F7DCFB01E07F48407A7649C8737A4844
:20108000007800F0010010B14EF6EE6001E07A48C08A704908827048807EEE2815D17748F3
:2010A0008078012823D1754880684FF44821B1FBF0F07349096808447149086008460068ED
:2010C000000B6E49C86012E0BFE06348807EAA280DD1624840686049897948435E49C979CB
:2010E000B0FBF1F03221B0FBF1F06449C8605A48007B594991F91B10084442F2107191FBAF
:20110000F0F15E48C0685F4A1268801A814206D801205D4908705948C0685A4908605A480D
:20112000007801283ED100205749087057480068401C564908605648406A401C5449486272
:2011400052488068401C51498860084680685149884203D900204D498860C8603D48008BE3
:20116000401C3C490883494800680A21B0FBF1F03849488248480078401C4749087008464E
:2011800000781E280EDB424B30226921434803F0A8F83E4B1022AD21404803F0A2F8002063
:2011A0003D4908702B4800881E281ADB3C480078401C3B49087008460078052814DB0020A5
:2011C000087038480088401C364908802148408B401C2049488334480078401C3249087025
:2011E00002E000202E4908702F4800783C2811DB00202D49087025484068401C234948602C
:201200002348C06A401C2249C8622048C068401C1E49C86023480088B0F5167F0EDB002097
:20122000204908801A4B302269211C4803F059F8164B1022AD21194803F053F80E48808A74
:201240000A2190FBF1F00349087510BD6C000020F00A0020DC080020B00A0020B403002006
:2012600032050020DA000020B0010020B4090020280300207C09002008030020E40300204D
:201280007C0000207000002074000020200C0020000B00209F8601008000002040040020ED
:2012A00075000020780000207600002010B50446F9F71AFD10490968401A4EF660218842A2
:2012C00018D3F9F711FD0C4908602068401C20600A480078401C09490870084600780A281C
:2012E00008DB074B30226921064802F0FAFF00200249087010BD0000C0000020C400002030
:20130000000B00204004002010B50446022C1BD1F9F7EAFC0F490968401AC82818D30E4BE8
:201320004FF481520C214FF4E26003F079F80B4B4BF620220C2140F2157003F071F8F9F778
:20134000D3FC0449086003E0F9F7CEFC0149086010BD000090000020DC080020FC08002015
:2013600001B511480078022800D108BD0098A0B1F9F7BAFC0D490968401AB0F5FA7F10D96F
:20138000F9F7B2FC094908606B4641F204120C214FF4E26003F044F803E0F9F7A5FC03495A
:2013A000086000BFE1E700005D0000208800002010B50446012C13D1F9F796FC0B490968B2
:2013C000401AC82810D30A4B4FF481520C214FF4E26003F025F8F9F787FC0449086003E0A8
:2013E000F9F782FC0149086010BD00008C000020DC08002010B5FBF701FAFBF7EDF9F3F7DC
:20140000F5FE03F099F9FBF7D3FC0A4801890A4804F05EF807484189084804F059F8054820
:201420008189074804F054F80248018A0548F6F703FD10BDDC1E0020F01500200A160020B8
:2014400024160020880400201CB50446F9F74CFC40490968401AB0F5FA7F7AD33E48008866
:20146000401C3D49088008460088142837DB3B48007800F0010010B900203949487437484C
:201480000088C0F3002010B900203549087433480078C0F3801010B90020314908812F4875
:2014A0000078C0F3C01010B900202D4948812B480078C0F3001010B9002029498881274888
:2014C0000078C0F3401010B900202549C8814FF480512448F9F7FEFB00201F49088022480E
:2014E000007868B900204FF408430C2240F2FF7100901E4802F0E0FF01201B49087024E00D
:2015000019480078012820D100200190184801780078401C164A107005290CDC01A841F2A8
:201520000133162240F2FF710090104802F0C4FF0A20F9F7F3F841F214030C2240F2FF71E1
:201540000A48009402F0B8FF00BFF9F7CDFB014908601CBD9C000020A0000020C401002099
:20156000D00B0020001001405D00002000060020A200002070B504464D48007880BB0821DA
:201580004C48F9F79FFB4C4908704FF400414B48F9F798FB4A49087080214A48F9F792FBCB
:2015A000494908704FF480714648F9F78BFB474908704FF400514348F9F784FB444908704E
:2015C00004214448F9F77EFB43490870002020816081A081E081207460740120344908704B
:2015E0003E48C08860803D488088A0804FF40060E0803A480089208008212E48F9F762FBF6
:2016000005462D480078A84202D02089401C2081294805704FF400412848F9F753FB0546CD
:2016200027480078A84202D06089401C60812448057080212348F9F745FB05462248007897
:20164000A84202D0A089401CA0811F4805704FF480711C48F9F736FB05461C480078A84282
:2016600002D0E089401CE081184805704FF400511448F9F727FB054615480078A84202D0BF
:20168000207C401C20741248057004211148F9F719FB054610480078A84202D0607C401C5E
:2016A00060740D4805704FF47A70608270BD00009A000020000C014094000020000801404C
:2016C00095000020001001409600002097000020980000200014014099000020F21E0020A1
:2016E00010B5F9F701FB42F21071884204D2F9F7FBFA4149086010BDF9F7F6FA3E49096868
:20170000401A41F28831884274D3F9F7EDFA3A4908603A48407D3A4991F82310884207DA87
:201720003648407D364981F823000020354908703248407D324991F82210884207DD2F48AB
:20174000407D2F4981F8220000202E4908702B48807D2B4991F82910884207DA2748807DED
:20176000274981F829000020264908702348807D234991F82810884207DD2048807D20493F
:2017800081F8280000201F4908701C48C07D1C4991F82B10884207DA1848C07D184981F8BC
:2017A0002B000020174908701448C07D144991F82A10884207DD1148C07D114981F82A000C
:2017C00000201049087010480088401C0E490880084600880C280DDD0A48007850B9002016
:2017E0000880012007490870054B30226921074802F077FD00BF7EE7C8000020DC08002087
:20180000000B0020CE000020CC0000204004002010B50748007850B9F9F766FA044949687C
:20182000401AB0F5FA6F02D901200149087010BDD001002000B587B001200390032004906D
:2018400003A90E48F9F7B0F80D480068806820F001000B4909688860002000900A20019020
:201860000720029069460648F7F7ACF920B140F2123104A004F0B4FF07B000BD00080140D1
:20188000081F00202E2E5C436F72655C5372635C6164632E630000000EB55F485F490860AD
:2018A00081155E4881600021C16041614FF46021C1610020594948600B2158480161F7F7BB
:2018C000EBFD18B15A2156A004F08AFF0A200090012001900720029069465048F7F772F9A4
:2018E00018B164214EA004F07BFF0B200090022001900720029069464848F7F763F918B1C5
:201900006E2147A004F06CFF0C200090032001900720029069464148F7F754F918B17821F4
:201920003FA004F05DFF0D200090042001900120029069463948F7F745F918B1822138A0B3
:2019400004F04EFF0520009001900120029069463248F7F737F918B18C2131A004F040FF8C
:2019600004200090062001900120029069462B48F7F728F918B1962129A004F031FF0F207C
:201980000090072001900120029069462348F7F719F918B1A02122A004F022FF072000901A
:2019A000082001900720029069461C48F7F70AF918B1AA211AA004F013FF0E200090092076
:2019C00001900120029069461448F7F7FBF818B1B42113A004F004FF102000900A20019014
:2019E0000220029069460D48F7F7ECF818B1BE210BA004F0F5FE112000900B20019007207F
:201A0000029069460548F7F7DDF818B1C82104A004F0E6FE0EBD000000240140081F0020D0
:201A20002E2E5C436F72655C5372635C6164632E6300000000B589B0234824490860811508
:201A4000224881600021C1604161C16100201F49486001211D480161F7F71EFD18B1DC214D
:201A60001BA004F0BDFE01200190029003200590002003904FF48050089000200790069055
:201A8000049001A91148F6F793FE18B1EB2110A004F0A6FE02200190029001A90B48F6F7E5
:201AA00087FE18B1F4210AA004F09AFE03200190029001A90548F6F77BFE18B1FD2104A05F
:201AC00004F08EFE09B000BD00280140381F00202E2E5C436F72655C5372635C6164632EB9
:201AE0006300000010B50F480F4908601220486000210D488160C1604FF4A02101610021CE
:201B0000416181610121C1610021016241628162C162F8F707F918B1592104A004F060FEA8
:201B200010BD000000640040442400202E2E5C436F72655C5372635C63616E2E63000000C8
:201B400008B500BF0A48406940F00100084948610846406900F00100009000BF00BF0222C9
:201B600011460B20F9F78FF90B20F9F77FF908BD0010024000B585B000BF3A48806940F07D
:201B80001000384988610846806900F01000009000BF00BF00BF0846806940F02000886157
:201BA0000846806900F02000009000BF00BF00BF0846806940F0040088610846806900F096
:201BC0000400009000BF00BF00BF0846806940F0080088610846806900F00800009000BF5E
:201BE00000BF002289142048F9F778F84FF4634001900320029001A91B48F8F7D5FE40F66E
:201C0000087001900320029001A91848F8F7CCFE4EF6024001900320029001A91448F8F782
:201C2000C3FE4FF480500190124802900020039001A90F48F8F7B8FE4FF480500190012035
:201C400002900220049001A90748F8F7ADFE002211462820F9F717F92820F9F707F905B0FB
:201C600000BD0000001002400010014000080140000C01400000211010B50848084908606F
:201C80000320486040F2E24105488160F9F732F818B13A2103A004F0A3FD10BD0030004044
:201CA000040800202E2E5C436F72655C5372635C697764672E63000000B595B031483249AD
:201CC00008600020486020212F4881604FF41661C1600021016101214161F9F7C3FF4FF424
:201CE0008050119011A92848FAF764F82648FAF795FA70200F90802010900FA92248F9F78D
:201D00003AFF4FF4006008904010099000200A9039200B9000200C900D900E9008A91A48AE
:201D2000F9F7EAFE6FF08000174909680861602001904FF4966002900020039004900590FA
:201D400006900790002201A90F48FAF7E3F9042201A90D48FAF7DEF9082201A90A48FAF762
:201D6000D9F96020019040F65F10029000200390082004900C2201A90348FAF7CBF915B03D
:201D800000BD0000002C01401C1E002000B587B000200390049005900690019002904FF0FF
:201DA000804019490860002048600021164881604FF6FF71C1600021016141618161F9F7A4
:201DC00051FF18B17E2111A004F00AFD4FF400500390002004900590069003A90A48F9F7AC
:201DE000E9FF18B1862109A004F0FAFC00200190029001A90448F9F7BEFE18B18C2103A0FA
:201E000004F0EEFC07B000BD5C1E00202E2E5C557365725C5372635C74696D2E63000000C4
:201E200000B589B01C481D4908600020486000211A4881604721C1600021016180218161C7
:201E4000FAF7ECF920B14FF48F7115A004F0C8FC00200790089007A91048F9F78CFE20B189
:201E600040F225110EA004F0BBFC6020009024200190002002900490002269460748FAF765
:201E800049F920B14FF4977105A004F0A9FC0348FAF7F6F809B000BD000400409C1E0020E8
:201EA0002E2E5C557365725C5372635C74696D2E6300000010B50C480C4908604FF4165091
:201EC0004860002109488160C16001610C21416100218161C161FAF7DFFB18B1462104A0F1
:201EE00004F07EFC10BD000000480040882600202E2E5C436F72655C5372635C7573617275
:201F0000742E630000BFFEE730B504460A460021002329480078401C274D2870284600781E
:201F20000F2841DB0020287024480089244D2D88411B002907DA214800894FF6FF752844FE
:201F40001F4D2D88411B44F62060814200DD00211A4800891A4D28804FF47A70414319487D
:201F60000068081A174D2D6805EB2020154D2860284600680314C3EB031040F35C0000B2D5
:201F8000114D28800D488089104D2D68C5EB80200E4D2D6805EB60100C4D28602846006894
:201FA000C0F38F20054DE88112B90020064D28800548B0F9000030BDA2030020D807002077
:201FC000A4030020A8030020B0030020AC0300202DE9F04107460C46154629462046F6F7CA
:201FE00025FA8046002606E0701C34F8100024F81600701C86B2681EB042F5DC24F810704D
:202000004046BDE8F081704702480068C0F30220704700000CED00E010B5002807DA0A0777
:20202000140E054A00F00F031B1FD45403E00A07130E024A135410BD18ED00E000E400E08D
:2020400010B5F8F751FE40F6B831884216D90C480078012812D10020094908700948C07A58
:20206000AA280BD133200849087008460078C0430649087004484078C043487010BD00007A
:20208000CF000020B00A0020DA000020DC00002010B50446012C06D0022C23D0032C40D00F
:2020A000042C7DD15CE024224E494F48F1F7F7FC24224E494E48F1F7F2FC24224D494E485C
:2020C000F1F7EDFC24224D494D48F1F7E8FC24224C494D48F1F7E3FC24224C494C48F1F764
:2020E000DEFC7CE024224B493F48F1F7D8FC242249493F48F1F7D3FC242248493E48F1F732
:20210000CEFC242246493E48F1F7C9FC242245493D48F1F7C4FC242243493D48F1F7BFFCF2
:202120005DE0242241493048F1F7B9FC242240492F48F1F7B4FC24223E492F48F1F7AFFCC8
:2021400024223D492E48F1F7AAFC24223B492E48F1F7A5FC24223A492D48F1F7A0FC3EE006
:20216000242238492048F1F79AFC242236492048F1F795FC242235491F48F1F790FC242227
:2021800033491F48F1F78BFC242232491E48F1F786FC242230491E48F1F781FC1FE0FFE7ED
:2021A000242210491048F1F77AFC24220F491048F1F775FC24220F490F48F1F770FC2422EC
:2021C0000E490F48F1F76BFC24220E490E48F1F766FC24220D490E48F1F761FC00BF00BF10
:2021E00010BD000058720108540600207C72010878060020A07201089C060020C472010814
:20220000C0060020E8720108E40600200C7301080807002030730108547301087873010844
:202220009C730108C0730108E4730108087401082C740108507401087474010898740108E9
:20224000BC740108E074010804750108287501084C75010870750108947501082DE9F043AD
:2022600004460D46601B06B2B2F9000000FB06FC908810B90020106212E0B2F9040000FBD7
:2022800006F7106AC319D069984202DAD069106206E09069984202DD9069106200E01362F9
:2022A00050889CFBF0F0B2F80690D2F8208098FBF9F800EB0801002906DA1069884203DD81
:2022C000108A00B2BDE8F083002905DD5069884202DC908A00B2F5E708B2F3E72DE9F34F9A
:2022E00083B00C46204603F003F900901D4800990160BDF90C001B49B1F9001000FB01F742
:20230000FF13BDF90E001749B1F9021000FB01F84FEAE8380FFA87FB0FFA88F00190019848
:20232000ABEB000000B2ADF80800BDF90C000D49B1F9021000FB01F5ED13BDF90E000949CD
:20234000B1F9001000FB01F6F6130FFA85F90FFA86FA09EB0A0000B2ADF80A00029805B00A
:20236000BDE8F08F4C0000207047000030B50246B2F900303F4CB4F90040A34202DD138837
:202380003C4C2380B2F902303B4CB4F90040A34202DD5388384C2380B2F90430374CB4F9EC
:2023A0000040A34202DD9388344C2380344B1B885B1C1BB2324C23802346B3F90030B3F567
:2023C000FA7F56DB2B4BB3F900000023294C2380031E01DB1C4600E05C42B5256C43294D1A
:2023E0002D68C5EB8404274D2D6805EB6414254D2C602B461B689B121BB20B801E4BB3F993
:20240000000000231C4C2380031E01DB1C4600E05C42B5256C431C4D2D68C5EB84041A4D8B
:202420002D6805EB6414184D2C602B461B689B121BB24B80114BB3F9000000230F4C23804C
:20244000031E01DB1C4600E05C42B5256C430F4D2D68C5EB84040D4D2D6805EB64140B4D3E
:202460002C602B461B689B121BB28B800023044C238030BD7C0500207E050020800500206B
:202480008205002084050020880500208C05002000B585B000BF1148806940F004000F4917
:2024A00088610846806900F00400009000BF00BF002289140A48F8F711FC4FF48050019049
:2024C000012002900220049001A90548F8F76CFA00200449087005B000BD0000001002409E
:2024E000000801408604002010B50446012C0BD10C480078A8B9012211030B48F8F7EEFB42
:202500000120084908700CE05CB906480078012807D1002201030448F8F7E0FB0020014963
:20252000087010BD860400200008014010B5044619480078012816D1B4F5D16F0FDB174839
:202540000088401C80B21549088047F23051884220DD0020114908800F4908701AE0002012
:202560000E49088016E0B4F5BC6F10DA0C480088401C80B20A4908803C280BDDF4F744FD0B
:2025800001200549087000200649087002E000200349088010BD000094050020900500205C
:2025A00092050020FF01002038B50446002034490870F020487008460078C0433149087075
:2025C0002F484078C04348702D4840782E4B0090DA79997958792D4B1B78FAF725FD2C4813
:2025E000007810BB2B4800682B4908602948406848602848806888602648C068C8602748B3
:20260000406808612548406A48612448C06A88612822234801F002FE042222A12048083833
:2026200001F0FCFD01201A49087020A341F205320C214FF4E26001F0F3FE04B938BDF8F752
:2026400053FB1C49086000201B49087012E0F8F74BFB18490968401A64280BD9F8F744FB72
:202660001449086014480078401C134908701348F8F768FB104800780A28E8DB00BFDDE79C
:20268000DA000020DC000020D00A002050040020B6000020200C0020900B0020000B0020CE
:2026A00008E80108464C4147000000005245414459000000B8000020BC00002004080020B2
:2026C00010B50248F9F767FB10BD00001C1E002010B500210B48F9F7F5FD04210948F9F7F1
:2026E000F1FD08210748F9F7EDFD00210548F9F789FA04210348F9F785FA08210148F9F778
:2027000081FA10BD1C1E002008B508490968C9084FF47A72B1FBF2F14143009100BF00BF76
:2027200000994A1E00920029F9D108BD000000202DE9F04705460E4617469846F8F7D4FA4A
:2027400084490968401A052801D2BDE8F087F8F7CBFA804908600FFA88F07F4948807F4808
:202760000088281AC8810846007801287ED1F8F7BBFA7949C969401AB0F5FA6F06D9F8F73A
:20278000B3FA7549C8610120887601E0744886607148407E01281BD100206F4948760024BD
:2027A00005E000206F4921F81400601CC4B2192CF7DB00206C4908806C4908606C4908707F
:2027C0006548408A20B16448408A0002694908606148C0890A2849DB604805605E48807E26
:2027E00000286FD15E4886600774C068002869D05B4880895A490989401A00B25E490880C5
:202800000846B0F90000002803DD0846B0F9000000E00020584908800846B0F900001E285C
:2028200003DA0846B0F9000000E01E20524908800846008818B94A48007C642842D049489F
:202840004949098830F8110048490968081A47490860084600684849B1F900100844434927
:2028600008604548008881B23F4800E06FE002880088401C3C4B18803A4820F8121018464B
:202880000088192807DB002019460880012038490870314908763548006840B334480078A8
:2028A000012810D1314800684FF47A7148436421484329498989FA225143B0FBF1F0264935
:2028C000088217E03FE02848008800EB80004100214880894143254800684FF47A72504327
:2028E00064225043B0FBF1F01B49088202E00020194908821C480088A0B91748B0F810906B
:202900001C480068C0EB09201E2190FBF1F01949096808441749086008460068C0F30F20ED
:202920000D4948820C48408A002808DD0C4880680949898AB0FBF1F00749C88203E04FF65D
:20294000FF700549C882064880680549C86000BFFBE600006C0300200803002070030020D7
:2029600028030020640700205C030020600300206403002068030020660300202DE9F0419D
:2029800004460D4617469846069E00201349086088601348008848600020C8600DB9084608
:2029A000866000200F49087048800520888000208860084684810020C881088248824FF6EF
:2029C000FF70C88200200876487601208876F8F78BF90449C861BDE8F08100002803002079
:2029E000B4090020080300202DE9F04106460F4606F00F0000287DD0052FFCD001206F4994
:202A000008700846007E012864D1002008760846408A6B49098888425CD06848408A002881
:202A200054D06648408A67490988401A642100FB01F56448008895FBF0F004B214F11E0F5D
:202A400044DBB4F5E47F41DA04F164005D4909884843642190FBF1F0584988825A4805884A
:202A600004F164006843642190FBF1F0574908805548458804F164006843642190FBF1F0DA
:202A8000524948805048858804F164006843642190FBF1F04D4988804B48C58804F1640062
:202AA0006843642190FBF1F04849C8804648058904F164006843642190FBF1F0434908817B
:202AC0000B461022CD21424801F00BFC3B48408A3B4908803F480078864203D13E48007811
:202AE000874265D0032E1DD005DC012E08D0022E33D10EE054E0042E1DD0332E2DD123E0FB
:202B0000324800882D4948822F4800882D49088029E02E484088294948822B484088294946
:202B2000088020E02948808824494882264880882449088017E02548C088204948822248A9
:202B4000C088204908800EE0204800891B4948821D4800891B49088005E000201749488226
:202B60001849088000BF00BF1448408A144908801248408A114988820846408A002807DD37
:202B800016488068898AB0FBF1F00C49C88203E04FF6FF700949C88201200849487607E067
:202BA000002006490870488288824FF6FF70C8820848067008480770BDE8F081080300208E
:202BC0007603002078030020E4790108300C00204004002074030020750300202803002021
:202BE0002DE9F047074689461546AD10002414E057F82460300E144A02F82400C6F30741AE
:202C0000A000401C1154C6F30721A000801C1154A000C01C1654601CC4B2AC42E8DB57F8F9
:202C200025A0A1000848F2F7C5FA8046BAEB080007D1AA0004494846F0F731FF0020BDE88A
:202C4000F0874FF0FF30FAE77C17002010B5B0F900205243B0F9023003FB03210C4A9142B2
:202C600014D909163939CBB20A4C34F81320B0F9003003FB02F1CB131BB20380B0F90230D1
:202C800003FB02F1CB131BB2438000BF10BD0000400AC139B87501082DE9F14181B0BDF9A0
:202CA0000400DFF86880B8F9008000FB08F1C913BDF90600DFF85480B8F9028000FB08F2C1
:202CC000D2130EB217B2F01900B2ADF80000BDF90400DFF83880B8F9028000FB08F3DB13C6
:202CE000BDF90600DFF82480B8F9008000FB08F4E4130FFA83FC25B2CCF10000284400B244
:202D0000ADF802000098BDE8FC8100004C00002010B504462078012808D10B4B302269210B
:202D20000A4801F0DEFA002020700AE02078022807D1074B10229B21044801F0D2FA0020DB
:202D40002070002010BD0000000B002040040020300B00204FF055301F4A106040001F4AC6
:202D600010601D480168B1F1553F01D0002070471A480168B1F1AA3F01D00020F7E74FF0D3
:202D8000AA30154A10604008144A106012480168B1F1AA3F01D00020E9E710480168B1F102
:202DA000553F01D00020E2E74FF055300A4A106040000A4A106008480168B1F1553F01D079
:202DC0000020D4E705480168B1F1AA3F01D00020CDE70120CBE700000008002010080020FF
:202DE00001200C490968B1F1EE3F00D0002009494968B1F1CC3F00D0002006498968B1F1AB
:202E0000BB3F00D000200349C968B1F1DD3F00D000207047102B002010B5214800780D28B0
:202E20002FD2DFE800F0070A0D101316191C1F2225282B00F0F7C2F924E0F0F7F3F921E01B
:202E4000F0F72FFA1EE0F0F771FA1BE0F0F7B4FA18E0F0F7F8FA15E0F0F73CFB12E0F0F7C5
:202E600080FB0FE0F0F7C5FB0CE0F0F70BFC09E0F0F74CFC06E0F0F78DFC03E0F0F7CEFC65
:202E800000E000BF00BF06480078401C04490870084600780C2801DD0020087010BD0000B0
:202EA0001006002010B5F0F789F9F0F7BBF9F0F7F8F9F0F73BFAF0F77FFAF0F7C4FAF0F733
:202EC00009FBF0F74EFBF0F794FBF0F7DBFBF0F71DFCF0F75FFCF0F7A1FC10BD10B53B48B0
:202EE0000068B0F1AA3F70D138480068384909684840401C002866D136490860C043364919
:202F0000086034480068801C32490860FFF784FF31480068801E304908602E4800680D30F2
:202F20002C490860FFF75CFF08B9F4F743FE2A4800680D3828490860264800680B302549FF
:202F4000086000F0C5FC044634B1012C0AD0032C04D0042C05D100E007E006E0F4F72AFE59
:202F600003E000BFF4F726FE00BF00BF1A4800680B381949086017480068C01C15490860E2
:202F800000F044F808B9F4F715FE13480068C01E114908600F480068401D0E490860FFF712
:202FA000D9FE08B9F4F706FE0B480068401F0A490860222003F0B4FD08B9F4F7FBFD00200B
:202FC0000249086001E0F4F7F5FD10BDD8260020FC260020C8260020EC26002010B500F05E
:202FE00047FC00F055FC00F001F810BD4FF0EE30054908604FF0CC3048604FF0BB3088608F
:203000004010C86070470000102B0020F0B55527552F01D00020F0BDAA27AA2F01D0002048
:20302000F9E74FF05531B1F1553F01D00020F2E74FF0AA31B1F1AA3F01D00020EBE74FF440
:203040007A714A008C1840F6B830844201D00020E1E74FF0FF3102228C18012C01D00020A5
:20306000D9E74FF47A73F94D5E1916F57A7F01D00020D0E76FF0004301255E19B6F1004FC2
:2030800001D00020C7E76FF0004302255E19981C864201D00020BEE76FF0004303255E19FE
:2030A000D81C864201D00020B5E74FF4FA614A108C1AB4F57A7F01D00020ACE74FF4FA6165
:2030C0004A1C8C1A601C08B10020A4E7002101228C1A601C08B100209DE74FF47A735D00B4
:2030E0005E1B16F57A7F01D0002094E7002301255E1B701C08B100208DE74FF000430125A4
:203100005E1B581E864201D0002084E74FF47A71491C0846814201D000207CE74FF0FF3135
:20312000491C09B1002076E70021491C012901D0002070E74FF47A735B1C1846834201D060
:20314000002068E700235B1C012B01D0002062E76FF000435B1CB3F1004F01D000205AE7C2
:203160004FF000435B1C1846834201D0002052E74FF47A71491E0846814201D000204AE741
:203180000021491E481C00B145E74FF0FF31491E881C00B13FE74FF47A735B1E1846834249
:2031A00001D0002037E74FF000435B1E1846834201D000202FE76FF000435B1E184683429D
:2031C00001D0002027E700235B1E581C00B122E764210A2201FB02F4B4F57A7F01D00020F0
:2031E00019E76FF07041112201FB02F49848844201D000200FE74FF0FF31012201FB02F489
:20320000601C08B1002006E76421002201FB02F40CB10020FFE64FF47A710A22B1FBF2F425
:20322000642C01D00020F6E601210A22B1FBF2F40CB10020EFE600210A22B1FBF2F40CB103
:203240000020E8E64FF47A710022B1FBF2F40CB10020E0E64FF0FF310122B1FBF2F4601C5B
:2032600008B10020D7E602214C00042C01D00020D1E602210C02B4F5007F01D00020CAE677
:203280000221CC070CB10020C5E64FF6FF714C084810844201D00020BDE64FF6FF710C0A2A
:2032A000FF2C01D00020B6E64FF6FF71CC0F0CB10020B0E6012109B90020ACE6002109B1E2
:2032C0000020A8E6FF2109B90020A4E664210A22914201D800209EE664216422914201D9FB
:2032E000002098E60A216422914201D9002092E64FF0FF310022914201D800208BE66FF00D
:203300000043DD07AB4201DC002084E60A216422914201D300207EE664216422914201D2A5
:20332000002078E664210A22914201D2002072E600214A1E914201D300206CE64FF000431C
:203340005D1EAB4201DB002065E664210A22914201D200205FE664216422914201D2002031
:2033600059E60A216422914201D3002053E64FF0FF310022914201D200204CE66FF0004332
:20338000DD07AB4201DA002045E60A216422914201D900203FE664216422914201D90020BB
:2033A00039E664210A22914201D8002033E600214A1E914201D900202DE64FF000435D1EF2
:2033C000AB4201DD002026E664216422914201D0002020E64FF0FF310A46914201D000209E
:2033E00019E600210022914201D0002013E64FF000431D46AB4201D000200CE600230025D1
:20340000AB4201D0002006E66FF000431D46AB4201D00020FFE564216422914201D000204C
:20342000F9E54FF0FF310A46914201D00020F2E500210022914201D00020ECE54FF00043FA
:203440001D46AB4206D00020E5E5000030F8FFFFEFFFFF0F00230025AB4201D00020DAE555
:203460006FF000431D46AB4201D00020D3E50121002221B9022904D0032906D103E0921C00
:2034800004E0121D02E0083200E000BF00BF022A01D00020BFE502210022012904D0022970
:2034A00004D0032906D103E0921C04E0121D02E0083200E000BF00BF042A01D00020AAE569
:2034C00003210022012904D0022904D0032906D103E0921C04E0121D02E0083200E000BF47
:2034E00000BF082A01D0002095E504210022012904D0022904D0032906D103E0921C04E0B4
:20350000121D02E0083200E000BF00BF0AB1002081E50021002211B10AB100207BE501B9C7
:203520000AB1002077E50021012211B10AB1002071E511B90AB900206DE50121012201B127
:203540000AB9002067E511B90AB9002063E50121FF2201B10AB900205DE511B90AB9002080
:2035600059E50021FF2211B10AB1002053E511B90AB900204FE54FF055310A4681EA02048F
:203580000CB1002047E54FF055314A0081EA0204601C08B100203EE50021002281EA020476
:2035A0000CB1002037E54FF0FF310A4681EA02040CB100202FE500214A1E81EA0204601C7B
:2035C00008B1002027E54FF05531CC43B4F1AA3F01D000201FE5E443B4F1553F01D000205E
:2035E00019E50021CC43601C08B1002013E5E4430CB100200FE501200DE5000008B500BFC9
:203600007148806940F004006F4988610846806900F00400009000BF00BF00BF0846806904
:2036200040F0080088610846806900F00800009000BF00BF00BF0846806940F0100088610D
:203640000846806900F01000009000BF00BF00BF0846806940F0200088610846806900F0CF
:203660002000009000BF00BF5848F4F7F7FA08B9002008BD5648F4F7F1FA08B90020F8E7C6
:203680005448F4F7EBFA08B90020F2E75248F4F7E5FA08B90020ECE74B48806920F004005C
:2036A000494988610846806920F0080088610846806920F0100088610846806920F02000B0
:2036C00088614648F1F720F800BF3F48C06940F000703D49C8610846C06900F0007000904E
:2036E00000BF00BF3E48F1F71FFD08B90020C0E73548C06920F000703349C86100BF084662
:20370000406940F0010048610846406900F00100009000BF00BF3348F2F7A0FA08B9002051
:20372000A7E72948406920F001002749486100BF0846806940F4007088610846806900F409
:203740000070009000BF00BF00BF0846806940F4806088610846806900F48060009000BF9E
:2037600000BF2148F0F7E8FE08B9002081E71F48F0F7E2FE08B900207BE71348806920F442
:203780000070114988610846806920F48060886100BF0846806940F40060886108468069B8
:2037A00000F40060009000BF00BF114801F089FB08B900205DE70448806920F400600249C0
:2037C0008861012055E700000010024000080140000C0140001001400014014000000140D4
:2037E00000640040080002400024014000280140002C014010B5002419480068194909681B
:203800004840401C48BB164800681749884210D316490846F0F73AF8012801D1042400E025
:20382000032411484B380E490860C0430D49086014E00E490A480068F0F728F801280AD1F5
:203840000748006810300649086008460068C0430449086002E0032400E00124204610BD0B
:2038600044060020480600207B0000202406002004480549086008460068C043034908601C
:203880007047000030000020440600204806002010B50A480A490860C0430A4908600A4867
:2038A0000A4908600846F6F764FD08480068806840F0010005490968886010BD0030000834
:2038C000E426002008270020003002401806002010B502241F4800681F4909684840401C48
:2038E000002834D11B4800681C49884223D2002006E01849096851F82010194A1160401C2B
:2039000018498908174A9209B1FBF2F18142F0D814498908134A9209B1FBF2F10D4A126859
:2039200002EB81010B4A116011460968C9430A4A116000240CE00A48006808490968884263
:2039400001D1042400E00324FFF7A2FF00E00124204610BDE426002008270020808F010806
:2039600000300240805F010070B50A2050490870F7F7FCF900F0E2FF00204E490860C043BF
:203980004D4908604B480068801C4A490860FFF789FA49480068801E47490860EFF7C2FBEC
:2039A0000C2043490870434800680B304149086042484349086008460068806840F001006A
:2039C000096888603E48F6F7D4FC002405E03D4951F8240039490860641C3B48B4EB900F24
:2039E000F5D33648056839480068854201D0F4F7E1F8314800680B382F4908600E202C4928
:203A000008702C480068C01C2A490860FFF7FEFA08B9F4F7CFF828480068C01E26490860AD
:203A200010202349087023480068401D21490860FFF790F908B9F4F7BDF81F480068401F62
:203A40001D49086012201A4908701A480068C01D18490860FFF7D2FD08B9F4F7ABF81420D3
:203A600013490870FFF7CAFD08B9F4F7A3F812480068C01F1049086016200D4908701C20CC
:203A800003F04EF808B9F4F795F81820084908704FF400510804EFF772FF08B9F4F78AF88E
:203AA00000F0B6FFAA2005490871EFF71FFB70BD14060020C8260020EC26002000300240B7
:203AC0001806002000300008805F0100808F010810B5124800780A281EDB00200F490870C6
:203AE0004FF0AA300E49086040080E49086072B6FFF780FE044662B634B1012C08D0032CD0
:203B000005D0042C02D100E005E004E000BF00BFF4F750F800BF00BF10BD000059000020AF
:203B2000D8260020FC260020002107E041F64C5100BF0A00A1F1010399B2FAD10200A0F141
:203B4000010398B2F2D17047002106E0072100BF0A00A1F1010399B2FAD10200A0F1010362
:203B600098B2F3D1704770472DE9F143BDF9000044F2F30100FB01F9BDF902004FF4165148
:203B80004843C0F10008444608EB09004710A8EB09004610002F0FDA002E03DA0520F7498A
:203BA000088018E0002C03DC0420F449088012E00320F24908800EE0002E03DB0220EF4965
:203BC000088008E0002C03DC0620EC49088002E00120EA4908800020E9490870E748008848
:203BE00007287BD2DFE800F07A044D97E0FCFB0004F51650801B4FF4966101EBA040E1492F
:203C000008800846008800EB6640488008464088A0EB6440888008460088C0F5166080B26D
:203C2000E22803DD40F65F10C88029E0D5480088D4494988401A85B2B5F58B7F05DBD148D3
:203C400000883338CF49C8801AE0CE480088C0F5166080B28A2813DDCA480088E230C949BC
:203C6000C8800846C088B0F5166F09DB0120C4490870C448C088C0F59650401EC149C88013
:203C800074E107F51650801B4FF4966101EBA040BC4908800846008800EB664048800846C2
:203CA0000088A0EB6740888008464088C0F5166080B2E22803DD40F65F10C8802AE0B148F5
:203CC0004088B0490988401A85B2B5F58B7F06DBAC4840883338AB49C8801BE045E1A948F7
:203CE0004088C0F5166080B28A2813DDA5484088E230A449C8800846C088B0F5166F09DB5D
:203D000001209F4908709F48C088C0F59650401E9C49C8802AE1C4F5165038444FF49661ED
:203D200001EBA0409749088008460088A0EB674088800846808800EB64404880084640887C
:203D4000C0F5166080B2E22803DD40F65F10C88029E08C4840888B498988401A85B2B5F56A
:203D60008B7F05DB8748408833388649C8801AE084484088C0F5166080B28A2813DD8148EA
:203D80004088E2307F49C8800846C088B0F5166F09DB01207A4908707A48C088C0F5965094
:203DA000401E7849C880E1E004F51650801B4FF4966101EBA040734908800846008800EBD6
:203DC0006640488008464088A0EB6440888008468088C0F5166080B2E22806DD01E078E04F
:203DE0002EE040F65F10C88029E06648808865494988401A85B2B5F58B7F05DB61488088B4
:203E000033386049C8801AE05E488088C0F5166080B28A2813DD5B488088E2305949C880F8
:203E20000846C088B0F5166F09DB0120544908705448C088C0F59650401E5249C88095E073
:203E400007F51650801B4FF4966101EBA0404D4908800846008800EB66404880084600883C
:203E6000A0EB6740888008468088C0F5166080B2E22803DD40F65F10C88029E041488088E4
:203E800040490988401A85B2B5F58B7F05DB3D48808833383B49C8801AE03A488088C0F5E6
:203EA000166080B28A2813DD36488088E2303549C8800846C088B0F5166F09DB012030491C
:203EC00008703048C088C0F59650401E2D49C8804CE0C4F5165038444FF4966101EBA04026
:203EE0002849088008460088A0EB674088800846808800EB6440488040F65F10C8800846D1
:203F00000088C0F5166080B2E22803DD40F65F10C88029E01B4800881A498988401A85B2EC
:203F2000B5F58B7F05DB1748008833381549C8801AE014480088C0F5166080B28A2813DD18
:203F400010480088E2300F49C8800846C088B0F5166F09DB01200A4908700A48C088C0F5F0
:203F60009650401E0749C88000E000BF00BF0448007848B9002000F003FB08E034000020F8
:203F80003600002038000020022000F0F9FA40F64C100949C880088800F0DAFA06494888CF
:203FA00000F0DCFA0449888800F0DEFA0249C88800F0E0FABDE8F883380000202DE9F041F2
:203FC0000446002500260027F3F75EF8A84618E000BF334800780128FBD100203049087047
:203FE0003048008805442F48408806442D48808807440C212C48F8F745F908F101001FFA46
:2040000080F8B8F10A0FE3DB0A20B5FBF0F0274908800A20B6FBF0F048800A20B7FBF0F0B7
:2040200088800846008846F2A81188421DDB1F48008849F64041884217DC1C48408846F21F
:20404000A811884211DB1948408849F6404188420BDC1648808846F2A811884205DB1348FB
:20406000808849F64041884216DD206820F4802000F58020206006200D4948800846F3F7EE
:204080000FFB00200B4908700B484089401C0A494881022009490870F2F7F6FFBDE8F081B6
:2040A00030050020240500201C1E0020360500209807002091030020300B0020BA01002004
:2040C00008B50020009053480088072870D2DFE800F0933362630405320000BF4E48008885
:2040E000404201B211F5004F04DA4FF40040ADF8000009E0B1F5004F04DB47F6FF70ADF822
:20410000000001E0ADF8001043484088404201B211F5004F04DA4FF40040ADF8020009E03B
:20412000B1F5004F04DB47F6FF70ADF8020001E0ADF8021061E000BF37484088404201B244
:2041400011F5004F04DA4FF40040ADF8020009E0B1F5004F04DB47F6FF70ADF8020001E011
:20416000ADF802102C488088BDF80220801A01B2B1F5004F04DB47F6FF70ADF8000009E0DA
:2041800011F5004F04DA4FF40040ADF8000001E0ADF8001031E000BF1F480088404201B23A
:2041A000B1F5004F05DB47F6FF70ADF800000AE022E011F5004F04DA4FF40040ADF8000092
:2041C00001E0ADF8001014488088BDF80020801A01B211F5004F04DA4FF40040ADF8020066
:2041E00009E0B1F5004F04DB47F6FF70ADF8020001E0ADF8021000E000BF00BFBDF9000003
:204200000011ADF80000BDF902000011ADF80200009808BD340000203C0500202DE9F04719
:2042200081460D4616463046F11706EB9171C1F38707002415E015F824000106A000401C08
:20424000285C01EB0041A000801C285C01EB0021A000C01C285C08440A4941F82400601C68
:20426000C4B2BC42E7DB31462846F0F7A3FF8046044840F827807A1C01464846F3F70EFB4B
:20428000BDE8F0877C1800202DE9F04190B080460D4616463046F11706EB9171C1F387079F
:2042A000002414E0A000C01C285C0106A000801C285C01EB0041A000401C285C01EB002066
:2042C00015F8241008444DF82400601CC4B2BC42E8DB3A4669464046F3F7E0FA10B0BDE857
:2042E000F0812DE9F84381460D4616461F46002000908046002420E02819C1B26A46484695
:20430000F3F71AF8401C18B94FF0FF30BDE8F883385D9DF8001088420DD0385D009028199F
:20432000C1B29DF800204846F3F75CF8401C10B94FF0FF30EAE7601CC4B2B442DCDB31460F
:204340003846F0F71FFF80464FEA28200090A819C1B29DF800204846F3F744F8401C10B941
:204360004FF0FF30D2E708F0FF000090A819401CC1B29DF800204846F3F734F8401C10B981
:204380004FF0FF30C2E70020C0E7000070B505460C46002C33D11E4800691E4948600B461E
:2043A000302269212846FFF79CFF401C28B9194B302269212846FFF794FF1548006816498A
:2043C00008601348406848601148806888601048C068C8600E4840690E4948620C488069BC
:2043E000C8620D4B1022AD212846FFF77AFF401C28B9094B1022AD212846FFF772FF0648AA
:2044000000680A21B0FBF1F004494882002070BD900B0020000B0020200C0020DC080020E3
:204420002DE9F04706468846174699460025FCB255201F490870AA204870084680F80280E7
:20444000A01CC870380A08710846447122464946801DEFF724FB552016490870AA20487043
:2044600030128870CE70221D1149891C1148001DEFF715FB04F108010E48F0F79BFE0546FB
:20448000280EA11D0A4A5054C5F30741E01D1154C5F30721401C1154401C1554F021401CFB
:2044A0001154421C02493046F0F7A0FDBDE8F0873E0E00203D0F00202DE9F04781460E4698
:2044C00090461F46DDF820A00025FCB255201E490870AA204870300A8870CE70084680F82D
:2044E0000480A01C4871380A88710846C471224651460830EFF7D3FA04F108021249134866
:20450000EFF7CDFA04F108011048F0F753FE0546280E04F108010C4A5054C5F3074104F1F2
:2045200009001154C5F30721401C1154401C1554F021401C1154401CC2B20349484601F03A
:20454000A2F9BDE8F08700003C100020D210002001490968486370471C1E00200149096804
:20456000886370471C1E002001490968C86370471C1E002001490968086470471C1E002010
:2045800008490968096A21F40051064A1268116204490968096A41EA0031024A126811627D
:2045A000704700001C1E002010B51048007801281BD10F4A32210F4800F048F90446EFF7DC
:2045C0006DFC0D49086008460068EFF78AFC0B490860002005490870084800681E2804DA14
:2045E0000348008800B20649088010BD100100201C0100201408002014010020180100207A
:204600000C0100202DE9F04705460C4616461F46DDE90889F6F768FB19490968401A322894
:204620002BD3F6F761FB1649086005FB06F090FBF7F000FB08F000EBC000000142F21071B0
:2046400090FBF1F0208020880E49096808440D4908600D480078401C0B4908700846007819
:2046600008280ADB0020087006480068C0F3CF00A9F80000002003490860BDE8F0870000C4
:20468000FC030020040400200004002070B504460D461646F6F728FB24490968401A3228EF
:2046A00041D3E07828B9F6F71FFB214908600120E070F6F719FB1E490968401AB0F57A6FA2
:2046C00004D90020A0704FF6FF70A060208980B24FF6FF71884202D10020A07001E00120BA
:2046E000A070A078012812D1A06810B94FF0FF30A0604FF4B4707043A168B0FBF1F02080F8
:2047000020880A220B49FDF763FC288007E00020208028800A210748F0F77DF870BDF6F737
:20472000E3FA0249086000BFF8E70000080400200C040020DC15002000B585B000BF1048DD
:20474000806940F020000E4988610846806900F02000009000BF00BF0420019009480290F3
:204760000120039001A90848F6F71EF9002202210820F6F788FB0820F6F778FB05B000BDB0
:204780000010024000001110001401402DE9F04104460D4617461E46F6F7A6FA284909683D
:2047A000401A32284AD3E07828B9F6F79DFA254908600120E070F6F797FA22490968401A70
:2047C0004FF47A6191FBF6F1884201D90020A070A078012822D1A06810B94FF0FF30A06001
:2047E0004FF4B4707843B0FBF6F0A168B0FBF1F0208020880A221449FDF7EAFB2880F6F732
:2048000073FA6168411AA068B1EB400F12D940F20E41A0684843800AA0600BE000202080E0
:2048200028800A210848EFF7F6FF4FF0FF30A060BDE8F081F6F758FA0149086000BFF7E768
:20484000F4030020F8030020C81500202DE9F74F88B0044689464FF0000BDA46002006905C
:2048600000210F4688460D460E4600BF0FE034F81B00EFF729FB3A464346CDE90401EFF7A4
:20488000F7F9074688460BF1010000F0FF0BCB45EDDB4846EFF718FB02460B46CDE9020165
:2048A00038464146EFF78BFACDE90401EFF791FB06900698EFF72EFB81B20A9801804FF083
:2048C000000A23E034F81A00EFF7E8FA00900699EFF796F9029034F81A00EFF7DFFA0090F2
:2048E0000699EFF78DF901900299EFF78FF90390EFF75CFB2A463346CDE90401EFF7B8F908
:2049000005460E460AF1010000F0FF0ACA45D9DB2846314602F0C8FBCDE90201EFF72DFBDF
:2049200080B20590EFF7D0FA05460E4628463146EFF723FB80B20BB0BDE8F08F10B594B05E
:2049400009200A904FF480300B9000200C9001200E90109002201190C10312914FF4E0118D
:2049600013910AA8F6F76EFD18B1CD211AA001F037FF0F20059002200690002007904FF47B
:204980008060089000200990022105A8F6F718FC18B1DB2110A001F023FF02200190800357
:2049A000039001A8F6F774FB18B1E2210AA001F017FFF6F7D7FC4FF47A71B0FBF1F42046FE
:2049C000F7F77AF80420F6F75DFF00221146501EF6F759FA14B010BD2E2E5C53656C6654BC
:2049E000657374557365725C7372635F6D6964646C6577617265735C73746D3332667878CD
:204A00005F535455737461727475702E6300000010B590B00220069001200A9010200B9054
:204A200000200D9006A8F6F70DFD20B140F2031114A001F0D5FE0F20019000200290039080
:204A40004FF48060049000200590002101A8F6F7B7FB20B140F211110AA001F0C1FEF6F715
:204A600081FC4FF47A71B0FBF1F42046F7F724F80420F6F707FF00221146501EF6F703FAA3
:204A800010B010BD2E2E5C53656C6654657374557365725C7372635F6D6964646C657761BE
:204AA0007265735C73746D33326678785F535455737461727475702E6300000003461804DD
:204AC0004843B0FBF2F0704710B5F6F743F9F7F70DF803480078401C0149087010BD000078
:204AE0005900002010B594B009200A904FF480300B9000200C9001200E9010900220119005
:204B0000C10312914FF4E01113910AA8F6F79AFC20B14FF4CA711CA001F062FE0F20059001
:204B200002200690002007904FF48060089000200990022105A8F6F743FB20B14FF4D17141
:204B400011A001F04DFE022001908003039001A8F6F79EFA20B140F2A9110BA001F040FEDA
:204B6000F6F700FC4FF47A71B0FBF1F42046F6F7A3FF0420F6F786FE00221146501EF6F730
:204B800082F914B010BD00002E2E2F436F72652F5372632F6D61696E2E6300001148006878
:204BA00040F001000F490860084640680E4908400C494860084600680C4908400949086065
:204BC0000846006820F4802008600846406820F4FE0048604FF41F008860C8030449086089
:204BE00070470000001002400000FFF8FFFFF6FE08ED00E010B50248F7F776F910BD0000B5
:204C00001C1E002000220268184B984208D0B0F1804F05D0164B984202D0164B984203D138
:204C200022F070024B681A43104B984208D0B0F1804F05D00E4B984202D00E4B984203D182
:204C400022F44072CB681A4322F080024B691A4302608B68C3620B688362044B984201D18A
:204C60000B6903630123436170470000002C0140000400400008004030B50023012404FAB7
:204C800001F3046A9C430462046A02FA01F52C43046230BD30B50023042404FA01F3046ABB
:204CA0009C430462046A02FA01F52C43046230BD30B50C460021816821F47F4142EA032523
:204CC00025432943816030BD0A460021816821F0700142F0070319438160704730B500241D
:204CE00000220023056A25F001050562026A4368846924F0700424F003040D682C4322F0E1
:204D000002028D682A430D4DA84206D100BF22F00802CD682A4322F00402084DA84207D166
:204D200023F4807323F400734D692B438D692B43436084614D684563026230BD002C0140B4
:204D400030B5002400220023056A25F010050562026A4368846924F4E04424F440740D6884
:204D600044EA052422F020028D6842EA05120F4DA84207D100BF22F08002CD6842EA051287
:204D800022F04002094DA84209D123F4806323F400634D6943EA85038D6943EA8503436078
:204DA00084614D688563026230BD0000002C014030B5002400220023056A25F48075056281
:204DC000026A4368C46924F0700424F003040D682C4322F400728D6842EA05220E4DA842F3
:204DE00007D100BF22F40062CD6842EA052222F48062094DA84209D123F4805323F40053B6
:204E00004D6943EA05138D6943EA05134360C4614D68C563026230BD002C014030B50022F2
:204E200000230024056A25F480550562036A4468C26922F4E04222F440720D6842EA05225B
:204E400023F400538D6843EA0533074DA84204D124F480444D6944EA85144460C2614D68A6
:204E60000564036230BD0000002C014030B50B46144600210022026A056A25F001050562DA
:204E8000816921F0F00141EA041122F00A021A438161026230BD30B50B4614460021002265
:204EA000056A25F0100505628169026A21F4704141EA043122F0A00242EA0312816102623B
:204EC00030BD0146002240F205100860086882B240F20510824201D00020704740F28A209A
:204EE0000860086882B240F28A20824201D00020F3E70020086045F255504860486882B24B
:204F000045F25550824201D00020E6E742F6A8204860486882B242F6A820824201D00020F2
:204F2000DBE70020486045F255508860886882B245F25550824201D00020CEE74AF6A220B7
:204F40008860886882B24AF6A220824201D00020C3E70020886045F25550C860C86882B274
:204F600045F25550824201D00020B6E742F6AA20C860C86882B242F6AA20824201D00020BE
:204F8000ABE70020C86045F255508861886982B245F25550824201D000209EE74AF6AA202D
:204FA0008861886982B24AF6AA20824201D0002093E70020886145F25550C861C86982B237
:204FC00045F25550824201D0002086E74AF6AA20C861C86982B24AF6AA20824201D000207C
:204FE0007BE70020C86141F255500862086A82B241F25550824201D000206EE742F6AA203A
:205000000862086A82B242F6AA20824201D0002063E70020086245F255504862486A82B289
:2050200045F25550824201D0002056E74AF6AA204862486A82B24AF6AA20824201D0002049
:205040004BE70020486245F255508862886A82B245F25550824201D000203EE74AF6AA20A8
:205060008862886A82B24AF6AA20824201D0002033E70020886245F25550C862C86A82B2D1
:2050800045F25550824201D0002026E74AF6AA20C862C86A82B24AF6AA20824201D0002019
:2050A0001BE70020C86255200863086B82B2552A01D0002011E7AA200863086B82B2AA2A05
:2050C00001D0002009E70020086345F255504863486B82B245F25550824201D00020FCE683
:2050E0004AF6AA204863486B82B24AF6AA20824201D00020F1E60020486345F255508863EC
:20510000886B82B245F25550824201D00020E4E64AF6AA208863886B82B24AF6AA20824223
:2051200001D00020D9E60020886345F25550C863C86B82B245F25550824201D00020CCE603
:205140004AF6AA20C863C86B82B24AF6AA20824201D00020C1E60020C86345F255500864BA
:20516000086C82B245F25550824201D00020B4E64AF6AA200864086C82B24AF6AA20824270
:2051800001D00020A9E60020086441F215508864886C82B241F21550824201D000209CE688
:2051A00040F60A208864886C82B240F60A20824201D0002091E600208864086101208CE6E7
:2051C0002DE9F04104460E461746984627480078012812D1264801780078401C244A107013
:2051E000244820F811601046007832281CDB00201E4908701146087016E032221D493046A7
:20520000FCF7E6FE05462088A84209DDF5F76CFD19490968401AB0F57A7F05D9258003E06E
:20522000F5F762FD1449086040F634007843642190FBF1F0C0F580502188884203DBF5F786
:2052400053FD0E490860F5F74FFD0C490968401A42F21071884206D90948007820F00100AF
:20526000401C07490870BDE8F081000015040020160400203E1600201C0400201804002091
:20528000100400202DE9F04104460E461746984627480078012812D1264801780078401C0C
:2052A000244A1070244820F811601046007832281CDB00201E4908701146087016E03222D4
:2052C0001D493046FCF784FE05462088A84209DDF5F70AFD19490968401AB0F57A7F05D91E
:2052E000258003E0F5F700FD1449086040F634007843642190FBF1F0C0F58050218888426A
:2053000003DBF5F7F1FC0E490860F5F7EDFC0C490968401A42F21071884206D909480078FB
:2053200020F00200801C07490870BDE8F08100002004002021040020A21600202804002034
:2053400024040020100400202DE9F04104460E461746984627480078012812D126480178D7
:205360000078401C244A1070244820F811601046007832281CDB00201E4908701146087089
:2053800016E032221D493046FCF722FE05462088A84209DDF5F7A8FC19490968401AB0F5AF
:2053A0007A7F05D9258003E0F5F79EFC1449086040F634007843642190FBF1F0C0F58050A8
:2053C0002188884203DBF5F78FFC0E490860F5F78BFC0C490968401A42F21071884206D955
:2053E0000948007820F00400001D07490870BDE8F08100002C0400202D04002006170020F7
:205400003404002030040020100400202DE9F04704460F46E7824FF0090841462046F3F730
:2054200005F8C01B0FFA80F919F1780F41DDB9F1780F3EDA002606E0701C34F8100024F82A
:205440001600701CC6B2A8F10100B042F4DC24F8107041462046F3F773F805B2608AA8426D
:2054600000DA658241462046F3F77BF805B2A08AA84200DDA5821148844206D123461822B9
:2054800015210F48FEF72DFF16E00E48844206D12346182232210A48FEF723FF0CE00A48D8
:2054A000844209D1234618224F210548FEF719FF02E0002005490870BDE8F087F0150020D6
:2054C000400400200A160020241600201404002003B564220276002106E000EB4102BDF8F6
:2054E000043013804A1CD1B20C29F6D30CBD000008B5024602F5004081B20846CB1701EBAA
:20550000936399114FF6FE70014001F4407038B3B0F5807F36D0B0F5007F03D0B0F5407F62
:2055200040D10DE0C8B2214B33F81000ADF80200C8B2C0F1FF0033F81000ADF8000032E089
:20554000C8B2C0F1FF00194B33F81000ADF80200C8B233F81000404200B2ADF8000022E04B
:20556000C8B2124B33F81000404200B2ADF80200C8B2C0F1FF0033F81000404200B2ADF800
:20558000000010E0C8B2C0F1FF00084B33F81000404200B2ADF80200C8B233F81000ADF82E
:2055A000000000E000BF00BF009808BD4676010870B505466C6A0020E085E0842046F6F7E9
:2055C000C4FF70BD2DE9F04106460D461446002025490870F5F788FB2349486005F0FF0816
:2055E000A5F50040083830B1A0F6FA70B8B1B0F5545F2DD108E0424621461C48EEF74FFA88
:2056000000201B4908702BE023462A46314640F21560FEF705FF01201649087020E0217802
:20562000627801EB02218FB2002007E0124931F81010B94200DD03E0411CC8B20B28F5D308
:2056400000BF00F14601CAB20C4981F8272007E023462A46314640F21560FEF7E1FE00BF51
:2056600000BFBDE8F0810000D0010020C4010020CE0100205D0000200C7A01081C0900203F
:2056800010B50A46C37893421EDBC3681B68DB6823F02003C4682468E360C3789B1AC370A7
:2056A000C3681B68DB6843F02003C4682468E360114683780B4499B203788B4202DC03781B
:2056C000CB1A99B281701BE0C3681B68DB6823F02003C4682468E360C1780023C370C368D2
:2056E0001B68DB6843F02003C4682468E3608378194403788B4202DC0378CB1A99B2817079
:2057000010BD0168C96821F490710268D1600168496921F0010102685161202180F83A1024
:20572000704710B504462068C06820F040002168C860202084F839002046F7F74CF8002045
:2057400010BD00BFC27803789A42FBD0C2681268D26822F08002C3681B68DA60C2788AB98A
:20576000C26812681268C2F3C0125AB1C26812685160C2681268D26842F08002C3681B68E4
:20578000DA60704743788268D1544278521CD2B2427003789A4201D100224270C278521C4B
:2057A000C270C2681268D26842F08002C3681B68DA6000BFE5E710B502460B461946D478A9
:2057C0009C4209DB94780C44A1B214788C4204DC14780C1BA1B200E000219468605C10BD92
:2057E00070B5044694F83A0022284AD1A068B0F5805F13D1A56A206940B920684068C0F32B
:2058000008002880A06A801CA06219E020684068C0B22880A06A401CA06211E0206938B91A
:2058200020684068C1B2A26A501CA062117007E02068406800F07F01A26A501CA062117048
:20584000E08D401E80B2E085C8B92068C06820F020002168C8602068C06820F48070216897
:20586000C8602068406920F0010021684861202084F83A002046F6F7ADFF002070BD00202A
:20588000FCE70220FAE7F0B507460D461646002405E0295D3846FFF754FF601CC4B2B44243
:2058A000F7DBF0BD2DE9F041044600252068006920F44050E1680843216808612169A06806
:2058C00008436169084305432068C06841F20C61884328432168C8602068406920F44070F4
:2058E000A1690843216848615F49206888425CD1F5F74EFD00EBC00101EB001061688900C9
:20590000B0FBF1F6F5F744FD00EBC00101EB001061688900B0FBF1F06421B0FBF1F000EB46
:20592000C00101EB0010A6EB8000322101EB00106421B0FBF1F000F0F006F5F729FD00EB56
:20594000C00101EB001061688900B0FBF1F06421B0FBF1F006EB0016F5F71AFD00EBC001E5
:2059600001EB001061688900B0FBF1F7F5F710FD00EBC00101EB001061688900B0FBF1F0C7
:205980006421B0FBF1F000EBC00101EB0010A7EB8000322101EB00106421B0FBF1F000F0EC
:2059A0000F003044216888605BE0F5F7E1FC00EBC00101EB001061688900B0FBF1F6F5F777
:2059C000D7FC00EBC00101EB001061688900B0FBF1F06421B0FBF1F000EBC00101EB0010B5
:2059E000A6EB8000322101EB00106421B0FBF1F000F0F006F5F7BCFC00EBC00101EB001004
:205A000061688900B0FBF1F06421B0FBF1F006EB0016F5F7ADFC00EBC00101EB001061688A
:205A20008900B0FBF1F7F5F7A3FC00EBC00101EB001061688900B0FBF1F06421B0FBF1F028
:205A400000EBC00101EB0010A7EB8000322101EB00106421B0FBF1F000F00F003044216830
:205A60008860BDE8F081000000380140014691F8390021282CD18868B0F5805F0FD10A6A98
:205A80001088C0F308000B685860086918B9086A801C086209E0086A401C086205E00B6A53
:205AA000581C086218780B685860C88C401E80B2C88458B90868C06820F080000B68D86039
:205AC0000868C06840F040000B68D860002070470220FCE710B5054800F00EF8044800F0F3
:205AE00040F80448F6F732FD10BD0000F0050020000600208826002008B5C2681268126855
:205B0000C2F3401262B3C26812685268D1B2C268126812680022B2B943788268D154427859
:205B2000521CD2B2427003789A4201DB00224270C278521CD2B2C27003789A4203DD0278AB
:205B4000C2700122027100BF00220092C268126812680092C26812685268009200BF00BFEC
:205B600008BDC16809680968C1F3C01139B3C1680968C96801F0800109B36FF08001C268E1
:205B800012681160C17891B1C178491EC17082788168895CC268126851608178491CC9B2D8
:205BA0008170027891420ADB0021817007E0C1680968C96821F08001C2681268D1607047E0
:205BC00010B50248F3F784FF10BD00004424002010B54FF4FA71024800F004F810BD00007E
:205BE000F00500202DE9F34F83B00398C0780D2873DB00210398FFF7DEFD01906B49019844
:205C0000087001210398FFF7D6FD8146674981F80190019855287DD1B9F1AA0FFBD102214F
:205C20000398FFF7C8FD6149887003210398FFF7C2FD5E49C87004210398FFF7BCFD06465E
:205C40005A490E71112E03D0162E01D00C2E7DD105210398FFF7AFFD074654484771072147
:205C60000398FFF7A8FD834606210398FFF7A3FD0BEB00201FFA80F84FEA18204B49887128
:205C800081F8078007210398FFF795FD0446381B02287AD10398C17807F10B0081421DDA16
:205CA00043480078012806D1F5F71EF84149086000203F490870F5F717F83E490968411A7F
:205CC0000498814206D9F5F70FF83A49086001203749087005B0BDE8F08F64E001203449D4
:205CE000087000250FE005F10800C1B20398FFF762FD314948550846415D05F108002B4A41
:205D00001154681C85B2A542EDDB04F10800C1B2039800E043E0FFF74EFD4FEA006B04F1CC
:205D20000900C1B20398FFF746FD0BEB004B04F10A00C1B20398FFF73EFD0BEB002B04F17E
:205D40000B00C1B20398FFF736FD00E022E05844029004F108011548EFF72CFA8246029828
:205D6000B0EB0A000CD1144A41463046FFF72AFC07F10B00C1B20398FFF782FCAAE704E030
:205D800001210398FFF77CFC0DE001210398FFF777FC08E001210398FFF772FC03E00121B7
:205DA0000398FFF76DFC00BF94E70000FE110020180200201402002068110020012806D078
:205DC00002282AD003284ED0042873D173E0FE49FE4A13680B6053684B6092688A60FC4A8E
:205DE0001368CB6053680B6192684A61F94A13688B615368CB6192680A62F74A13684B62D1
:205E000053688B629268CA620A46F4490B6813634B6853638968916373E0EB4AF0490B68BC
:205E200013604B685360896891601146ED4A1368CB6053680B6192684A61EB4A13688B610B
:205E40005368CB6192680A62E84A13684B6253688B629268CA62E64A13680B6353684B634B
:205E600092688A634DE0D849E24A13680B6053684B6092688A60E04A1368CB6053680B619A
:205E800092684A61DD4A13688B615368CB6192680A620A46DA490B6853624B68936289684E
:205EA000D1621146D74A13680B6353684B6392688A6326E024E0C449D34A13680B60536829
:205EC0004B6092688A60D14A1368CB6053680B6192684A61CE4A13688B615368CB61926846
:205EE0000A62CC4A13684B6253688B629268CA62C94A13680B6353684B6392688A6300E0FE
:205F000000BF00BFC549897B78290DDCC349897B502909DBAC490988C04A927B5143642243
:205F200091FBF2F1A84A1180BC49097C78290DDCBA49097C502909DBA3498989B74A127CE9
:205F40005143642291FBF2F19F4A9181B349897C78290DDCB149897C502909DB9A49098B5F
:205F6000AE4A927C5143642291FBF2F1964A1183AA49097D78290DDCA849097D502909DB47
:205F80009149898CA54A127D5143642291FBF2F18D4A9184A149897D78290EDC9F49897DB6
:205FA00050290ADB8849498E9C4A927D5143642291FBF2F18AB284494A869849C97B5A29DC
:205FC00005DC8149097A491E7F4A117208E09349C97B6E2904DB7C49097A491C7A4A11726E
:205FE0008E49497C5A2906DC7749097D491ECAB275490A7509E08949497C6E2905DB724988
:20600000097D491CCAB270490A758449C97C5A2908DC6D4991F82010491ECAB26A4981F8EA
:2060200020200BE07D49C97C6E2907DB664991F82010491CCAB2644981F820207749497D7C
:206040005A2908DC604991F82C10491ECAB25E4981F82C200BE07149497D6E2907DB5A4995
:2060600091F82C10491CCAB2574981F82C206B49C97D5A2908DC544991F83810491ECAB263
:20608000514981F838200BE06449C97D6E2907DB4D4991F83810491CCAB24B4981F8382091
:2060A0005F49C97C78290DDC5D49C97C502909DB4549C9885A4AD27C5143642291FBF2F1C7
:2060C000414AD1805649497D78290EDC5449497D50290ADB3C49498A514A527D5143642257
:2060E00091FBF2F18AB238494A824D49C97D78290EDC4B49C97D50290ADB3349C98B484AA7
:20610000D27D5143642291FBF2F18AB22E49CA834349497E78290EDC4149497E50290ADB1A
:206120002949498D3E4A527E5143642291FBF2F18AB225494A853A49C97E78290EDC3849E7
:20614000C97E50290ADB2049C98E354AD27E5143642291FBF2F18AB21B49CA863049897C14
:2061600078290DDC2E49897C502909DB164949892B4A927C5143642291FBF2F1124A518151
:206180002749097D78290EDC2549097D50290ADB0D49C98A224A127D5143642291FBF2F1FF
:2061A0008AB20949CA821E49897D78293DDC1C49897D502939DB0449498C194A927D5143BE
:2061C000642291FBF2F12DE0E40B0020227A01082E7A01083A7A0108467A0108527A0108FD
:2061E0005E7A01086A7A0108767A0108827A01088E7A01089A7A0108A67A0108B27A010847
:20620000BE7A0108CA7A0108D67A0108E27A0108EE7A0108FA7A0108067B0108B00A0020E0
:20622000D00A00208AB214494A841449097E78290EDC1249097E50290ADB0F49C98D0F4A47
:20624000127E5143642291FBF2F18AB20A49CA850A49897E78290EDC0849897E50290ADBAC
:206260000549498F054A927E5143642291FBF2F18AB201494A877047E40B0020D00A0020F9
:2062800000BFFEE700B587B00020C6490860C6490880C64908700720C54908701821C548C6
:2062A000EDF716FC1821C448EDF712FC1821C348EDF70EFC1022C249C248EDF7F0FBC2485F
:2062C000C2490A680260496841601022C0A1C548EDF709FC1022C4A1C2481030EDF703FC40
:2062E0002E21C048203880F83F102022C3A1CC48EDF7F9FB00BFCBA207CA04AB07C3CCA2B2
:2063000007CA01AB07C39DF81A0030389DF81910303901EB810100EB4100C1498876032231
:20632000C6A104A8EDF701FC18B90120BC49C87670E00322C2A104A8EDF7F7FB18B90220E7
:20634000B749C87666E00322BEA104A8EDF7EDFB18B90320B249C8765CE00322BAA104A828
:20636000EDF7E3FB18B90420AD49C87652E00322B6A104A8EDF7D9FB18B90520A849C876FB
:2063800048E00322B2A104A8EDF7CFFB18B90620A349C8763EE00322AEA104A8EDF7C5FB00
:2063A00018B907209E49C87634E00322AAA104A8EDF7BBFB18B908209949C8762AE00322AE
:2063C000A6A104A8EDF7B1FB18B909209449C87620E00322A2A104A8EDF7A7FB18B90A2090
:2063E0008F49C87616E003229EA104A8EDF79DFB18B90B208A49C8760CE003229AA104A800
:20640000EDF793FB18B90C208549C87602E000208349C8769DF8151030399DF814002028E1
:2064200001D1002002E09DF81400303800EB800001EB40007A4908779DF8051030399DF8F6
:206440000400202801D1002002E09DF80400303800EB800001EB4000714948779DF808105E
:2064600030399DF80700202801D1002002E09DF80700303800EB800001EB400068498877B0
:206480009DF80B1030399DF80A00202801D1002002E09DF80A00303800EB800001EB40008A
:2064A0005F49C87700BF7148007828B930214D48203880F82A1036E06C480078012805D1F3
:2064C00031214848203880F82A102CE067480078022805D132214348203880F82A1022E0B3
:2064E00062480078052805D132213E48203880F82A1018E05D480078032805D133213948A9
:20650000203880F82A100EE058480078042805D134213448203880F82A1004E030213148E0
:20652000203880F82A10102251A12E482038EDF7DAFA102253A12B481038EDF7D4FA0822EA
:2065400055A15848EDF7CFFA082257A155480830EDF7C9FA082257A152481030EDF7C3FABD
:206560005748584B0ECB0EC000F0D8F800F0B0F85548007B544991F91B1008445249897987
:206580004843C0EB001001034F48C07941F2C6125043B1FBF0F04D49888108468089C88178
:2065A00007B000BD8C010020C401002010040020B00100208C090020980A0020800A0020AF
:2065C00070780108A4090020B10100204C7901082020202020202020343820202020202031
:2065E000000000003C0900205637723272335F323032333131313843000000005443303134
:20660000313030302D4D53303030302D563072312E20202020202020202020200000000048
:206620005C09002041756720203120323032340031383A31313A3531000000004A616E00A1
:20664000466562004D617200417072004D6179004A756E004A756C00417567005365700026
:206660004F6374004E6F760044656300F80100205047383058582026205053583058582E7E
:206680000000000030303030303030303030303030303030000000004D4F54494E4F56418D
:2066A00000000000400B0020575548414E2E202000000000323032313039303100000000EF
:2066C000B80B0020E8F7FF1FB00A00200402002010B5302209490A48EDF7E1F910220949DD
:2066E0000948EDF7DCF90948094C1ECC1EC0102208490948EDF7D3F910BD0000A4790108AB
:20670000000B0020D4790108300B0020200C0020F4790108E4790108300C002010B50C2226
:206720001AA11E48EDF7DFF91D4801891D48FEF7CFFE1B4841891C48FEF7CAFE18488189AE
:206740001A48FEF7C5FE1A481A490A680260496841604FF4B87018490880202217491848DE
:20676000EDF79DF91648007816490870202216491648EDF794F9102215491648EDF78FF928
:20678000CC2215491548EDF78AF910BD30303030303030303030303000000000C40B0020ED
:2067A000DC1E0020F01500200A16002024160020BB010020047A0108120400205479010891
:2067C000B00A0020B901002074790108D00A002094790108F00A002080780108B409002007
:2067E00088B004460D4631E01948FAF720F80020FBF77AFEF0F708FC20216846EDF768F9A0
:206800002046EDF77CF90646324621466846EDF746F92046EDF773F9694608440DA10A88CC
:206820000280897881702046EDF769F969460844C0F803506B464FF620720C214FF4E260F8
:20684000FDF7EEFDC820F3F769FF00BFCCE7000000010020202C200008B52B4988420DD147
:2068600000BF2A49896941F00401284A91611146896901F00401009100BF43E02449884271
:206880000DD100BF2149896941F008011F4A91611146896901F00801009100BF32E01D495F
:2068A00088420DD100BF1949896941F01001174A91611146896901F01001009100BF21E0EC
:2068C000154988420DD100BF1049896941F020010E4A91611146896901F02001009100BF61
:2068E00010E00E4988420DD100BF0849896941F04001064A91611146896901F040010091E7
:2069000000BF00BF08BD00000008014000100240000C01400010014000140140001801404D
:2069200070B504460E46A1882068F4F7CBF928B9A07908B9012506E0002504E0A07908B98A
:20694000002500E00125012E04D1207A68402840E07102E0207A6840E071257270BD10B50F
:206960000446A18801222068F4F7B8F910BD00BF704702E008C8121F08C1002AFAD17047C2
:206980007047002001E001C1121F002AFBD1704700F0010181F31388704700000149086035
:2069A0007047000020060020F0B504460E4619681F683D14A54206DA31440814A04212DD15
:2069C000204601040FE0A5420CDD02EB04473DB2A94202DA2046010405E0891A081410B9C7
:2069E000002100E020461960F0BD000010B50A46437993421EDB1E4B1B685B6923F00203A3
:206A00001B4C2468636143799B1A4371184B1B685B6943F00203164C246863611146037933
:206A20000B4499B283788B4202DC8378CB1A99B201711BE00E4B1B685B6923F002030C4C6E
:206A400024686361417900234371094B1B685B6943F00203064C246863610379194483780C
:206A60008B4202DC8378CB1A99B2017110BD00004424002010B502460B46194654799C4211
:206A800009DB14790C44A1B294788C4204DC94780C1BA1B200E000219468605C10BD00001C
:206AA0007FB50646002404E0305D18490855601CC4B2082CF8DB3823154A02A9304600F03F
:206AC0008DFB00241EE0002504E002A800F0AEFA681CC5B20F48005DA842F6DC40230E4A9B
:206AE000694602A800F07AFB002507E01DF805000A4901EBC4014855681CC5B2082DF5DB11
:206B0000601CC4B2102CDEDB7FBD000089030020D27B0108AA7E01080A7C0108E414002078
:206B200001460120064A12688A4206D1044A1268044B1B685A40521C02B100207047000054
:206B4000C8260020EC2600202DE9F04F87B082460F469046994600250AE0785D3A49495D8A
:206B6000884203D03846FFF79BFF0725681CC5B2082DF2DB4023354A05A9504600F02EFB02
:206B8000012536E0002405E005A8005D03A90855601CC4B2082CF7DBB8F1000F04D1681E92
:206BA0002B4901EBC00B04E0C5F11000284901EBC00B002406E003A9201D085C05A9085576
:206BC000601CC4B2042CF6DB01AA05A9584600F043F8002409E003A8005D01A9095D4840F3
:206BE00005AA211D5054601CC4B2042CF3DB681CC5B2112DC6DB9DF814609DF818008DF8FF
:206C000014008DF818609DF815609DF819008DF815008DF819609DF816609DF81A008DF8D4
:206C200016008DF81A609DF817609DF81B008DF817008DF81B604023064A494605A800F008
:206C4000CDFA07B0BDE8F08F89030020127B0108E4140020527B0108F0B587B005460E46E7
:206C600017464023104A05A9304600F0B7FA002410E005A8005D295D484000F03F0003A92E
:206C800008550A4800EB8410095D405C01A90855601CC4B2082CECDB2023054A394601A816
:206CA00000F09CFA07B0F0BD4A7C0108AA7C01088A7C01081CB5F6F717F8F6F71DF8B7490E
:206CC0000870F4F753F8FDF70DFFF6F74FF9FAF751FFFAF7F1FFFBF759F8FBF7A1F8FAF7F0
:206CE0002FFFFAF7D9FDFAF7A5FEFAF7FBFEFBF7E1F8FCF773F9EDF7EBFB1420F3F70EFD04
:206D0000A748F5F739F8FFF7BDFAFAF7B5FFFAF771FBA448F0F720FAF0F7C4FBA148F0F755
:206D2000D3F9F0F70BFCA0490870084601789D48FDF72CFB9D499E48F0F7DEFBF9F798FC61
:206D4000F1F702F900209B49087026E19A480078401C9949087008460078C82801DD002009
:206D6000087096480088F1F771FBFBF769F9EEF7A5FBFEF72DFF924A5178924AD07A924B3F
:206D8000924A1278F8F780F9FAF742FDF0F706F98C48807EAA2841D18D48007BC0B18C48C4
:206DA000B0F902000B2190FBF1F084B288498548007B844A92F91B20104480B2CDE9000170
:206DC0008048C379827983492046FDF71BFC46E07F48B0F902000B2190FBF1F07C49897A7F
:206DE000884206DD7A48B0F902000B2190FBF1F001E07748807A84B275497248007B714A63
:206E000092F91B20104480B2CDE900016D48C379827970492046FDF7F5FB20E06948807ED1
:206E2000EE280AD16748007B6649C97E0844C2B267496848FDF72AFC11E06248007B614947
:206E4000C97E0844C2B25F48007E08B9012001E05C48007E03465E495E48FDF797FC5E485E
:206E6000F1F7D6FA5D48EDF743FE00BF5C48007818BB5C48007828B1F3F736FF42F2107119
:206E8000884229D95248C0880A2190FBF1F084B2554880884B4A0090127B4A4D95F91B5090
:206EA0002A4490B2514A137B4E4A11782246FBF765FD01204A4908700EE0454C23894A4C2F
:206EC000627AA188434CE068FBF732FC484A11783D4A1078FBF788FD00BFFAF76FF8F8F70F
:206EE000D9F94448FAF7E2F9FAF7FAFB384B9A7D1989987AF7F7E8FE3F4908703C488079E3
:206F000010B93E48F0F7EEFA3948807930B93C493C48F0F789FB3C48FBF7FAFE3B48007813
:206F2000E8B93B4800683B4908603948406848603748806888603648C068C8602D48001F57
:206F40004068086128221A480830FDF767F9042231A11748FDF762F901202C490870F8F745
:206F600005FBF9F7C7FC2E480068FAF7F9F917480078FAF71DFA15480078FAF7C5F92948C9
:206F8000FAF762FAFDF710FBF1F73EF8FCF7A0FDFBF7A4FF2448F3F7D5FED7E6F801002063
:206FA0005C1E00204004002038040020FFEF010800E801085C0000205A000020FC0100207C
:206FC000B1010020B00A0020DA000020D8000020DC080020E403002051040020500400201F
:206FE0005B000020E80100207C090020F00A0020DE000020040B0020EE00002039040020B6
:207000009103002098070020BA010020FF010020200C0020900B0020464C414700000000E1
:207020008C010020D00B0020040800200CB5002104E0425C0DF801204A1CD1B20829F8DB05
:20704000002112E0425C5206120E425406290ADA4A1C1DF8022002F08002802A03D1425C31
:2070600042F0010242544A1CD1B20729EADB9DF8002002F0800222B1C27842F01002C270BB
:2070800003E0C27822F01002C2709DF8032002F0080222B1827942F00102827103E08279F5
:2070A00022F0010282710CBD2DE9F04106460F46EDF766F804000D4618BF0120284320F00B
:2070C0000040C0F17F6000F1E040C00F0ED0301C18BF0120384320F00040C0F17F6000F192
:2070E000E040C00F04BF0120FFF758FC20462946BDE8F08130B502460023002952D0334872
:20710000007890B13248334C247830F81400324C2468201A304C2060204600681044206003
:207120002B482C4C247820F814202A480078401C284C2070204600781E280FDB0020207074
:207140002248007818B90120204C207006E01F480078012802D102201C4C20701B480078A9
:20716000022806D11C4800681E24B0FBF4F083B211E01648007801280CD11648007808B9D8
:20718000134608E014480068124C2478B0FBF4F083B200E01346052093FBF0F0904212DD9F
:2071A000134610E0002005E00024094D25F81040441CE0B21E28F7DB0020064C2070064C3C
:2071C0002060024C2070184630BD0000E003002078150020D8030020DC0300202DE9F04115
:2071E00004461D46154E002000BF4FF000080746401C01F807800828F7DB002000BF12F845
:20720000013B04EBE3073F7803F0070C16F80CC007EA0C0767B101EBE0073F7800F0070C19
:2072200016F80CC047EA0C0701EBE00C8CF80070471C3846AF42E2DBBDE8F081BA7E01087E
:20724000000000000000000001020304060708090000000001020304204E00040300000483
:2072600000000004000000009CFFFFFFFF7F0000000000FE00FCFF0100000000204E000487
:207280000300000400000004000000000080FFFFFF7F0000000000FE00FCFF0100000000ED
:2072A000400000040300000400000004000000000000FCFF00000000000000F00000000094
:2072C00000000000307500012C0100040000000400000000CCF7FFFF000000000030DFFF04
:2072E0000000000000000000001000040100000400000004000000009CFFFFFF1A040000BA
:207300000070FEFF0068100000000000307500042C0100040000000400000000E6FBFFFFCB
:20732000000000000098EFFF0000000000000000204E00040300000400000004000000004A
:207340009CFFFFFFFF7F0000000000FE00FCFF0100000000204E000403000004000000049F
:20736000000000000080FFFFFF7F0000000000FE00FCFF01000000004000000403000004CC
:2073800000000004000000000000FCFF00000000000000F000000000000000003075000158
:2073A0002C0100040000000400000000CCF7FFFF000000000030DFFF0000000000000000C9
:2073C000001000040100000400000004000000009CFFFFFF1A0400000070FEFF00681000F4
:2073E00000000000307500042C0100040000000400000000E6FBFFFF000000000098EFFF4A
:207400000000000000000000204E00040300000400000004000000009CFFFFFFFF7F0000D8
:20742000000000FE00FCFF0100000000204E00040300000400000004000000000080FFFF57
:20744000FF7F0000000000FE00FCFF01000000004000000403000004000000040000000065
:207460000000FCFF00000000000000F00000000000000000307500012C0100040000000446
:2074800000000000CCF7FFFF000000000030DFFF0000000000000000001000040100000404
:2074A00000000004000000009CFFFFFF1A0400000070FEFF00681000000000003075000483
:2074C0002C0100040000000400000000E6FBFFFF000000000098EFFF000000000000000012
:2074E000204E00040300000400000004000000009CFFFFFFFF7F0000000000FE00FCFF01FE
:2075000000000000204E00040300000400000004000000000080FFFFFF7F0000000000FEF4
:2075200000FCFF0100000000400000040300000400000004000000000000FCFF0000000005
:20754000000000F00000000000000000307500012C0100040000000400000000CCF7FFFF9F
:20756000000000000030DFFF000000000000000000100004010000040000000400000000E0
:207580009CFFFFFF1A0400000070FEFF0068100000000000307500042C0100040000000471
:2075A00000000000E6FBFFFF000000000098EFFF0000000000000000657F367E107D807C45
:2075C000657B527A467940784177C476CE75DF74F47310739F72C271EA701770486F7D6E4F
:2075E0001A6E566D966CDA6B216B6D6A136A6469B8680F68696718677666D8653D65A464A3
:207600000E64C4633263A26215628A614561BE603960B55F345FB55E765EFA5D805D085D52
:20762000915C1C5CE25B705BFF5A905A235AED5981591859AF584858E357B1574D57EB56BE
:207640008A562B56CC550000C90092015B022403ED03B6047F0548061107D907A2086A0937
:20766000330AFB0AC40B8C0C540D1C0EE30EAB0F72103A110112C8128F1355141C15E2153E
:20768000A8166E173318F918BE19821A471B0B1CCF1C931D571E1A1FDD1F9F206121232284
:2076A000E522A62367242825E825A82667272628E528A329612A1F2BDC2B992C552D112E30
:2076C000CC2E872F4130FB30B5316E322633DF3396344D350436BA366F372438D9388C391F
:2076E000403AF23AA53B563C073DB83D683E173FC53F73402141CE417A422543D0437A4420
:207700002445CD4575461C47C34769480F49B449584AFB4A9D4B3F4CE04C814D204EBF4EF1
:207720005D4FFB4F97503351CE51685202539B533254C9546055F5558A561D57B057425835
:20774000D3586459F359825A0F5B9C5B285CB35C3E5DC75D4F5ED75E5D5FE35F6860EB6073
:207760006E61F0617162F1627063EE636C64E8646365DD655666CF664667BC673268A66810
:2077800019698B69FD696D6ADC6A4A6BB76B236C8E6CF86C616DC96D306E966EFB6E5E6F50
:2077A000C16F22708370E27040719D71F9715472AE7207735E73B5730A745F74B274047550
:2077C0005575A575F37541768D76D87622776B77B377FA773F788478C77809794A79897906
:2077E000C879057A417A7C7AB67AEE7A267B5C7B917BC57BF87B297C597C887CB67CE37C3A
:207800000E7D397D627D897DB07DD57DFA7D1D7E3E7E5F7E7E7E9C7EB97ED57EEF7E097F83
:20782000217F377F4D7F617F747F867F977FA67FB47FC17FCD7FD87FE17FE97FF07FF57F52
:20784000F97FFD7FFE7F0000050000000000000005000000000000000500000000000000A8
:2078600005000000000000000500000000000000A028240000000000000000000000000012
:20788000983A38100810F90FEE0FE60FE00FDB0FD70FD30FCF0FCB0FC70FC20FBC0FB50F2D
:2078A000AD0FA40F9B0F900F850F7A0F6F0F640F5A0F4F0F460F3D0F340F2B0F230F1B0FC1
:2078C000120F0A0F030FFA0EF20EE90EE10ED70ECE0EC40EB90EAF0EA40E990E8F0E840ECF
